:020000040000FA
:1000000000040020810A000015070000610A0000BA
:100010001F07000029070000330700000000000050
:10002000000000000000000000000000A50A000021
:100030003D070000000000004707000051070000D6
:100040005B070000650700006F07000079070000EC
:10005000830700008D07000097070000A10700003C
:10006000AB070000B5070000BF070000C90700008C
:10007000D3070000DD070000E7070000F1070000DC
:10008000FB070000050800000F0800001908000029
:10009000230800002D080000370800004108000078
:1000A0004B080000550800005F08000069080000C8
:1000B000730800007D080000870800009108000018
:1000C0009B080000A5080000AF080000B908000068
:1000D000C3080000CD080000D7080000E1080000B8
:1000E000EB080000F5080000FF0800000909000007
:1000F000130900001D090000270900003109000054
:100100003B0900001FB500F003F88DE80F001FBD8C
:1001100000F0ACBC40F6FC7108684FF01022401CA7
:1001200008D00868401C09D00868401C04D0086842
:1001300000F037BA9069F5E79069F9E7704770B554
:100140000B46010B184400F6FF70040B4FF0805073
:100150000022090303692403406943431D1B104621
:1001600000F048FA29462046BDE8704000F042BA47
:10017000F0B54FF6FF734FF4B4751A466E1E11E0DA
:10018000A94201D3344600E00C46091B30F8027B3B
:10019000641E3B441A44F9D19CB204EB134394B25D
:1001A00004EB12420029EBD198B200EB134002EBB2
:1001B000124140EA0140F0BDF34992B00446D1E952
:1001C0000001CDE91001FF224021684600F0F4FB58
:1001D00094E80F008DE80F00684610A902E004C8FB
:1001E00041F8042D8842FAD110216846FFF7C0FF7C
:1001F0001090AA208DF8440000F099F9FFF78AFFCB
:1002000040F6FC7420684FF01025401C0FD0206889
:1002100010226946803000F078F92068401C08D030
:100220002068082210A900F070F900F061F9A869AF
:10023000EEE7A869F5E74FF080500369406940F6A2
:10024000FC71434308684FF01022401C06D0086838
:1002500000F58050834203D2092070479069F7E788
:100260000868401C04D00868401C03D00020704778
:100270009069F9E70420704770B504460068C34DE3
:10028000072876D2DFE800F033041929631E250021
:10029000D4E9026564682946304600F062F92A46CE
:1002A0002146304600F031F9AA002146304600F0E0
:1002B00057FB002800D0032070BD00F009FC4FF46C
:1002C000805007E0201D00F040F90028F4D100F034
:1002D000FFFB60682860002070BD241D94E80700C3
:1002E000920000F03DFB0028F6D00E2070BDFFF715
:1002F000A2FF0028FAD1D4E901034FF0805100EBAE
:10030000830208694D69684382420ED840F6F8704E
:1003100005684FF010226D1C09D0056805EB8305B8
:100320000B6949694B439D4203D9092070BD55694A
:10033000F4E70168491C03D00068401C02D003E0C8
:100340005069FAE70F2070BD2046FFF735FFFFF731
:1003500072FF0028F7D1201D00F0F7F80028F2D135
:1003600060680028F0D100F0E2F8FFF7D3FE00F05B
:10037000BFF8072070BD10B50C46182802D0012028
:10038000086010BD2068FFF777FF206010BD41684E
:10039000054609B1012700E0002740F6F8742068FF
:1003A0004FF01026401C2BD02068AA68920000F065
:1003B000D7FA38B3A86881002068401C27D020688D
:1003C000FFF7BDFED7B12068401C22D026684FF051
:1003D0008050AC686D68016942695143A9420DD9EA
:1003E000016940694143A14208D92146304600F0E5
:1003F000B8F822462946304600F087F800F078F831
:100400007069D2E700F093F8FFF784FEF6E77069B1
:10041000D6E77669DBE740F6FC7420684FF01026DB
:10042000401C23D02068401C0CD02068401C1FD0EA
:100430002568206805F18005401C1BD027683879A5
:10044000AA2819D040F6F8700168491C42D001680A
:10045000491C45D00168491C3ED001680968491C07
:100460003ED00168491C39D000683EE0B069DAE747
:10047000B569DEE7B769E2E710212846FFF778FEA5
:100480003968814222D12068401C05D0D4F8001080
:1004900001F18002C03107E0B169F9E730B108CA63
:1004A00051F8040D984201D1012000E000208A4259
:1004B000F4D158B1286810B1042803D0FEE72846CB
:1004C000FFF765FF3149686808600EE0FFF722FE1C
:1004D00000F00EF87169BBE77169BFE7706904E06D
:1004E0004FF480500168491C01D000F0CBFAFEE7C0
:1004F000BFF34F8F26480168264A01F4E06111439B
:100500000160BFF34F8F00BFFDE72DE9F0411746B3
:100510000D460646002406E03046296800F054F8EF
:10052000641C2D1D361DBC42F6D3BDE8F08140F69B
:10053000FC700168491C04D0D0F800004FF48051D1
:10054000FDE54FF010208069F8E74FF080510A690F
:10055000496900684A43824201D810207047002050
:10056000704770B50C4605464FF4806608E0284693
:1005700000F017F8B44205D3A4F5806405F5805562
:10058000002CF4D170BD0000F40A0000000000202F
:100590000CED00E00400FA05144801680029FCD0C5
:1005A0007047134A0221116010490B68002BFCD0E0
:1005B0000F4B1B1D186008680028FCD0002010603D
:1005C00008680028FCD07047094B10B501221A605A
:1005D000064A1468002CFCD0016010680028FCD08A
:1005E0000020186010680028FCD010BD00E4014015
:1005F00004E5014070B50C46054600F073F810B9EB
:1006000000F07EF828B121462846BDE8704000F091
:1006100007B821462846BDE8704000F037B8000012
:100620007FB5002200920192029203920A0B000B06
:100630006946012302440AE0440900F01F0651F80C
:10064000245003FA06F6354341F82450401C8242F8
:10065000F2D80D490868009A10430860081D016827
:10066000019A1143016000F03DF800280AD00649C4
:1006700010310868029A10430860091D0868039A3F
:10068000104308607FBD00000006004030B50F4CED
:10069000002200BF04EB0213D3F800582DB9D3F8A1
:1006A000045815B9D3F808581DB1521C082AF1D3C3
:1006B00030BD082AFCD204EB0212C2F80008C3F8CD
:1006C00004180220C3F8080830BD000000E0014013
:1006D0004FF08050D0F83001082801D0002070473A
:1006E000012070474FF08050D0F83011062905D016
:1006F000D0F83001401C01D0002070470120704725
:100700004FF08050D0F830010A2801D00020704707
:100710000120704708208F490968095808471020B0
:100720008C4909680958084714208A4909680958FA
:100730000847182087490968095808473020854923
:100740000968095808473820824909680958084744
:100750003C20804909680958084740207D490968BC
:100760000958084744207B49096809580847482028
:1007700078490968095808474C207649096809589A
:10078000084750207349096809580847542071499F
:1007900009680958084758206E49096809580847E8
:1007A0005C206C4909680958084760206949096854
:1007B00009580847642067490968095808476820AC
:1007C00064490968095808476C2062490968095852
:1007D000084770205F4909680958084774205D4937
:1007E00009680958084778205A490968095808478C
:1007F0007C205849096809580847802055490968EC
:10080000095808478420534909680958084788202F
:1008100050490968095808478C204E490968095809
:10082000084790204B4909680958084794204949CE
:10083000096809580847982046490968095808472F
:100840009C204449096809580847A0204149096883
:1008500009580847A4203F49096809580847A820B3
:100860003C49096809580847AC203A4909680958C1
:100870000847B0203749096809580847B420354966
:10088000096809580847B8203249096809580847D3
:10089000BC203049096809580847C0202D4909681B
:1008A00009580847C4202B49096809580847C82037
:1008B0002849096809580847CC2026490968095879
:1008C0000847D0202349096809580847D4202149FE
:1008D000096809580847D8201E4909680958084777
:1008E000DC201C49096809580847E02019490968B3
:1008F00009580847E4201749096809580847E820BB
:100900001449096809580847EC2012490968095830
:100910000847F0200F49096809580847F4200D4995
:10092000096809580847F8200A490968095808471A
:10093000FC2008490968095808475FF48070054998
:10094000096809580847000003480449024A034B54
:100950007047000000000020000B0000000B0000AA
:1009600040EA010310B59B070FD1042A0DD310C82C
:1009700008C9121F9C42F8D020BA19BA884201D97E
:10098000012010BD4FF0FF3010BD1AB1D30703D0C6
:10099000521C07E0002010BD10F8013B11F8014B7C
:1009A0001B1B07D110F8013B11F8014B1B1B01D198
:1009B000921EF1D1184610BD02F0FF0343EA032254
:1009C00042EA024200F005B87047704770474FF0A6
:1009D00000020429C0F0128010F0030C00F01B800C
:1009E000CCF1040CBCF1020F18BF00F8012BA8BF1A
:1009F00020F8022BA1EB0C0100F00DB85FEAC17CDE
:100A000024BF00F8012B00F8012B48BF00F8012B90
:100A100070474FF0000200B51346944696462039C1
:100A200022BFA0E80C50A0E80C50B1F12001BFF4A7
:100A3000F7AF090728BFA0E80C5048BF0CC05DF80D
:100A400004EB890028BF40F8042B08BF704748BF5B
:100A500020F8022B11F0804F18BF00F8012B7047CF
:100A6000014B1B68DB6818470000002009480A4951
:100A70007047FFF7FBFFFFF745FB00BD20BFFDE719
:100A8000064B1847064A1060016881F308884068E1
:100A900000470000000B0000000B000017040000DE
:100AA000000000201EF0040F0CBFEFF30881EFF3ED
:100AB0000981886902380078182803D100E0000015
:100AC000074A1047074A12682C3212681047000084
:100AD00000B5054B1B68054A9B58984700BD0000B0
:100AE0007703000000000020F00A0000040000006E
:100AF000001000000000000000FFFFFF0090D00386
:10100000B81300201953020019C100007F520200DA
:1010100019C1000019C1000019C100000000000042
:10102000000000000000000000000000A5530200C6
:1010300019C100000000000019C1000019C1000022
:101040000D5402001354020019C1000019C1000020
:1010500019C1000019C1000019C1000019C1000028
:101060001954020019C1000019C100001F540200E8
:1010700019C10000255402002B5402003154020013
:1010800019C1000019C1000019C1000019C10000F8
:1010900019C1000019C1000019C1000019C10000E8
:1010A00019C100003754020019C1000019C1000025
:1010B00019C1000019C1000019C1000019C10000C8
:1010C0003D54020019C1000019C1000019C10000FF
:1010D00019C1000019C1000019C1000019C10000A8
:1010E00019C1000019C1000019C1000019C1000098
:1010F00019C1000019C1000019C1000019C1000088
:1011000019C1000019C1000000F002F824F0F3F842
:101110000AA090E8000C82448344AAF10107DA4552
:1011200001D124F0E8F8AFF2090EBAE80F0013F08D
:10113000010F18BFFB1A43F001031847EC470200E8
:101140000C4802000A444FF0000C10F8013B13F069
:10115000070408BF10F8014B1D1108BF10F8015B10
:10116000641E05D010F8016B641E01F8016BF9D103
:1011700013F0080F1EBF10F8014BAD1C0C1B09D15A
:101180006D1E58BF01F801CBFAD505E014F8016BCC
:1011900001F8016B6D1EF9D59142D6D3704700005E
:1011A0000023002400250026103A28BF78C1FBD870
:1011B000520728BF30C148BF0B6070471FB500F011
:1011C00003F88DE80F001FBD24F092B870B51A4CDB
:1011D00005460A202070A01C00F0D5F85920A080F8
:1011E00029462046BDE8704008F098B908F0A1B93A
:1011F00070B50C461149097829B1A0F160015E294A
:1012000008D3012013E0602804D0692802D043F2FB
:1012100001000CE020CC0A4E94E80E0006EB8000A2
:10122000A0F58050241FD0F8806E2846B04720607B
:1012300070BD012070470000080000201C00002045
:10124000805402003249884201D2012070470020B8
:10125000704770B50446A0F500002E4EB0F1786FCF
:1012600002D23444A4F500042948844201D2012565
:1012700000E0002500F043F848B125B9B44204D39A
:101280002548006808E0012070BD002070BD002DD9
:10129000F9D1B442F9D321488442F6D2F3E710B52C
:1012A0000446A0F50000B0F1786F03D21948044459
:1012B000A4F5000400F023F84FF0804130B1164847
:1012C000006804E08C4204D2012003E01348844209
:1012D000F8D2002080F0010010BD10B520B1FFF75A
:1012E000DEFF08B1012010BD002010BD10B520B1F7
:1012F000FFF7AFFF08B1012010BD002010BD084866
:1013000008490068884201D10120704700207047D9
:1013100000600200000000202000002008000020E3
:101320005C000020BEBAFECA10B5044600210120B0
:1013300000F042F800210B2000F03EF800210820C8
:1013400000F03AF80421192000F036F804210D20AD
:1013500000F032F804210E2000F02EF804210F20B6
:1013600000F02AF80421C84300F026F806211620D0
:1013700000F022F80621152000F01EF82046FFF7A5
:1013800025FF002010BD40F2011101807047FFF7DA
:101390002DBF1148704710487047104A10B51468A7
:1013A0000E4B0F4A08331A60FFF722FF0B48001D4F
:1013B000046010BD704770474907090E002804DB20
:1013C00000F1E02080F80014704700F00F0000F1F9
:1013D000E02080F8141D704703F900421005024018
:1013E00001000001FD48002101604160018170475A
:1013F0002DE9FF4F93B09B46209F160004460DD069
:101400001046FFF726FF18B1102017B0BDE8F08F87
:101410003146012001F0D3FE0028F6D101258DF8D8
:1014200042504FF4C050ADF84000002210A92846A9
:1014300006F0D6FC0028E8D18DF84250A8464FF4BB
:1014400028500025ADF840001C2229466846079523
:101450000CF0E7FF9DF81C000DF11C0A20F00F00B6
:10146000401C20F0F00010308DF81C0020788DF822
:101470001D0061789DF81E000DF1400961F34200E6
:1014800040F001008DF81E009DF8000008AA40F011
:1014900002008DF800002089ADF83000ADF8325020
:1014A0006089ADF83400CDF82CA060680E900AA9D0
:1014B000CDF82890684606F088FA0028A5D1606823
:1014C000FFF70BFF40B16068FFF710FF20B96078AD
:1014D00000F00300022801D0012000E00020BF4CF2
:1014E00008AA0AA92072BDF8200020808DF8428049
:1014F00042F60120ADF840009DF81E0020F00600E5
:10150000801C20F001008DF81E000220ADF8300094
:10151000ADF8340014A80E90684606F056FA00287C
:1015200089D1BDF82000608036B1211D304600F021
:101530005FF90028C2D109E0BBF1000F05D00CF023
:10154000EBFCE8BB0CF0E8FCD0BBA58017B1012F89
:1015500043D04AE08DF8428042F6A620ADF8400024
:1015600046461C220021684607950CF05AFF9DF85C
:101570001C00ADF8346020F00F00401C20F0F0009B
:1015800010308DF81C009DF81D0020F0FF008DF834
:101590001D009DF81E0020F0060040F00100801C98
:1015A0008DF81E009DF800008DF8446040F00200A8
:1015B0008DF80000CDE90A9AADF8306011A800E07E
:1015C00011E00E9008AA0AA9684606F0FEF9002864
:1015D000A6D1BDF82000E08008E00CF09DFC10B919
:1015E0000CF09AFC08B103200FE7E58000200CE71F
:1015F0003EB50446794D0820ADF80000A88828B112
:101600002046FFF726FE18B110203EBD06203EBD45
:101610002146012001F0D3FD0028F8D12088ADF843
:1016200004006088ADF80600A088ADF80800E088E6
:10163000ADF80A00A88801AB6A46002106F0CCFD8F
:10164000BDF800100829E2D003203EBD7FB5634DF0
:101650000446A88868B1002002900820ADF8080070
:10166000CDF80CD02046FFF7F4FD20B1102004B0D7
:1016700070BD0620FBE7A98802AA4FF6FF7006F0AE
:10168000EDFF0028F3D1BDF80810082901D0032090
:10169000EDE7BDF800102180BDF802106180BDF8B3
:1016A0000410A180BDF80610E180E0E701B582B02A
:1016B0000220ADF80000494802AB6A46408800218C
:1016C00006F08AFDBDF80010022900D003200EBDEF
:1016D0001CB5002100910221ADF800100190FFF728
:1016E000DEFD08B110201CBD3C486A4641884FF61B
:1016F000FF7006F0B3FFBDF800100229F3D00320FD
:101700001CBDFEB5354C06461546207A0F46C0076F
:1017100005D00846FFF79DFD18B11020FEBD0F2033
:10172000FEBDF82D01D90C20FEBD3046FFF791FD1E
:1017300018BB208801A905F04AFE0028F4D13078B2
:101740008DF80500208801A906F024FD0028EBD1C2
:1017500000909DF800009DF8051040F002008DF803
:101760000000090703D040F008008DF80000208831
:10177000694606F0ACFC0028D6D1ADF808502088A8
:101780003B4602AA002106F027FDBDF80810A94239
:10179000CAD00320FEBD7CB5054600200090019014
:1017A0000888ADF800000C4628460195FFF795FD26
:1017B00018B92046FFF773FD08B110207CBD15B1A4
:1017C000BDF8000060B105486A4601884FF6FF7019
:1017D00006F044FFBDF8001021807CBD24020020EB
:1017E0000C20FAE72F48C088002800D0012070475D
:1017F00030B5044693B000200D46014600901422F7
:1018000001A80CF00EFE1C22002108A80CF009FE15
:101810009DF80000CDF808D020F00F00401C20F00B
:10182000F00010308DF800009DF8010006AA20F0AD
:10183000FF008DF801009DF8200001A940F0020092
:101840008DF8200001208DF8460042F60420ADF806
:10185000440011A801902088ADF83C006088ADF8E4
:101860003E00A088ADF84000E088ADF842009DF849
:10187000020020F00600801C20F001008DF802001C
:101880000820ADF80C00ADF810000FA8059008A8CE
:1018900006F09BF8002803D1BDF81800288000202E
:1018A00013B030BD24020020F0B5007B059F1E461A
:1018B00014460D46012800D0FFDF0C2030803A206E
:1018C0003880002C08D0287A032806D0287B0128ED
:1018D00000D0FFDF17206081F0BDA889FBE72DE96C
:1018E000F0470D4686B095F80C900E991446B9F164
:1018F000010F0BD01022007B2E8A9046052807D0BE
:10190000062839D0FFDF06B0BDE8F0870222F2E7F3
:10191000E8890C2200EB400002EB400018803320E5
:101920000880002CEFD0E8896081002720E0009635
:10193000688808F1020301AA696900F097FF06EBC5
:101940000800801C07EB470186B204EB4102BDF89A
:1019500004009081F848007808B1012300E00023DA
:101960000DF1060140460E3212F0CDFE7F1CBFB2D3
:101970006089B842DBD8C6E734200880E889B9F12D
:10198000010F11D0122148430E301880002CBAD01C
:10199000E88960814846B9F1010F00D00220207328
:1019A00000270DF1040A1FE00621ECE70096688885
:1019B00008F1020301AA696900F058FF06EB08006C
:1019C000801C86B2B9F1010F12D007EBC70004EBFF
:1019D0004000BDF80410C18110220AF1020110304C
:1019E0000CF0F5FC7F1CBFB26089B842DED88AE7F4
:1019F00007EB470104EB4102BDF80400D0810AF176
:101A000002014046103212F0A0FEEBE72DE9F0474C
:101A10000E4688B090F80CC096F80C80378AF5898D
:101A20000C20DFF81493109902F10C04BCF1030FA1
:101A300008D0BCF1040F3DD0BCF1070F75D0FFDF1B
:101A400008B061E705EB850C00EB4C0018803120F5
:101A50000880002AF4D0A8F1060000F0FF0A5581A2
:101A600024E01622002101A80CF0DBFC009770880E
:101A7000434601AA716900F0F9FEBDF80400208018
:101A8000BDF80600E080BDF80800208199F800004C
:101A900008B1012300E00023A21C0DF10A01504609
:101AA00012F031FE07EB080087B20A346D1EADB2AA
:101AB000D7D2C5E705EB850C00EB4C00188032202F
:101AC0000880002ABCD0A8F1050000F0FF0A55816B
:101AD00037E000977088434601AA716900F0C6FE9E
:101AE0009DF80600BDF80410E1802179420860F3FA
:101AF000000162F34101820862F38201C20862F3CD
:101B0000C301020962F30411420962F3451182091B
:101B100062F386112171C0096071BDF80700208150
:101B200099F8000010B1012301E00EE000232246E5
:101B30000DF10901504612F0E6FD07EB080087B2EF
:101B40000A346D1EADB2C4D27AE7A8F1020084B2A5
:101B500005FB08FC0CF10E00188035200880002AD7
:101B6000A7D05581948100971FFA8CF370880E32AC
:101B7000716900F07BFE63E72DE9F84F1E460A9D70
:101B80000C4681462AB1607A00F58070D080E089E9
:101B9000108199F80C000C274FF000084FF00E0A46
:101BA0000D2872D2DFE800F09D070E1B272F374566
:101BB000546972727200214648460095FFF774FE20
:101BC000BDE8F88F207B9146082802D0032800D07A
:101BD000FFDF3780302009E0A9F80A80F0E7207B9A
:101BE0009146042800D0FFDF378031202880B9F1EA
:101BF000000FF1D1E4E7207B9146042800D0FFDFFD
:101C000037803220F2E7207B9146022800D0FFDFA8
:101C100037803320EAE7207B1746022800D0FFDF19
:101C20003420A6F800A02880002FC9D0A7F80A8089
:101C3000C6E7207B1746042800D0FFDF3520A6F832
:101C400000A02880002FBBD04046A7F80A8012E0F1
:101C5000207B1746052802D0062800D0FFDF102081
:101C6000308036202880002FAAD0E0897881A7F81C
:101C70000E80B9F80E00B881A2E7207B91460728B4
:101C800000D0FFDF37803720B0E72AE04FF01200A6
:101C900018804FF038001700288091D0E0897881B3
:101CA000A7F80E80A7F8108099F80C000A2805D034
:101CB0000B2809D00C280DD0FFDF81E7207B0A28F4
:101CC00000D0FFDF01200AE0207B0B2800D0FFDFDF
:101CD000042004E0207B0C2800D0FFDF05203873AF
:101CE0006EE7FFDF6CE770B50C46054601F0ABFB15
:101CF00020B10078222804D2082070BD43F20200EF
:101D000070BD0521284610F073FF206008B1002047
:101D100070BD032070BD30B44880087820F00F00FB
:101D2000C01C20F0F000903001F8080B1DCA81E8BB
:101D30001D0030BC07F073BC100000202DE9FF47E8
:101D400084B0002782460297079890468946123051
:101D50000AF033FA401D20F00306079828B907A9B6
:101D60005046FFF7C0FF002854D1B9F1000F05D04D
:101D70000798017B19BB052504681BE098F8000053
:101D8000092803D00D2812D0FFDF46E0079903256C
:101D90004868B0B3497B42887143914239D98AB2CD
:101DA000B3B2011D10F097FD0446078002E0079CC6
:101DB000042508340CB1208810B1032D29D02CE063
:101DC0000798012112300AF02AFAADF80C000246F9
:101DD00002AB2946504608F0B2FA070001D1A01C18
:101DE000029007983A461230C8F80400A8F802A0FA
:101DF00003A94046029B0AF01FFAD8B10A2817D25D
:101E000000E006E0DFE800F007091414100B0D14E1
:101E10001412132014E6002012E6112010E6082008
:101E20000EE643F203000BE6072009E60D2007E665
:101E3000032005E6BDF80C002346CDE900702A46D4
:101E40005046079900F022FD57B9032D08D1079895
:101E5000B3B2417B406871438AB2011D10F04FFD5F
:101E6000B9F1000FD7D0079981F80C90D3E72DE98D
:101E7000FE4F91461A881C468A468046FAB102AB4C
:101E8000494608F05CFA050019D04046A61C278890
:101E900010F0F3FF3246072629463B46009610F025
:101EA00000FC20882346CDE900504A465146404672
:101EB00000F0ECFC002020800120BDE8FE8F002017
:101EC000FBE710B586B01C46AAB104238DF800309C
:101ED0001388ADF808305288ADF80A208A788DF85A
:101EE0000E200988ADF80C1000236A462146FFF742
:101EF00025FF06B010BD1020FBE770B50D4605218B
:101F000010F076FE040000D1FFDF294604F1120034
:101F1000BDE870400AF06CB92DE9F8430D468046E3
:101F2000002607F079FB04462878102878D2DFE8ED
:101F300000F0773B345331311231313108313131D6
:101F400031312879001FC0B2022801D0102810D1E9
:101F500014BBFFDF35E004B9FFDF0521404610F078
:101F600047FE007B032806D004280BD0072828D082
:101F7000FFDF072655E02879801FC0B2022820D055
:101F800050B1F6E72879401FC0B2022819D01028B6
:101F900017D0EEE704B9FFDF13E004B9FFDF2879BB
:101FA00001280ED1172137E00521404610F020FE10
:101FB000070000D1FFDF07F1120140460AF0F5F8F3
:101FC0002CB12A4621464046FFF7A5FE29E0132101
:101FD000404602F021FD24E004B9FFDF0521404620
:101FE00010F006FE060000D1FFDF694606F1120080
:101FF0000AF0E5F8060000D0FFDFA988172901D212
:10200000172200E00A46BDF80000824202D90146CC
:1020100002E005E01729C5D3404600F047FCD0E7B1
:10202000FFDF3046BDE8F883401D20F0030219B100
:1020300002FB01F0001D00E000201044704713B5C2
:10204000009858B10024684610F0EFFB002C04D132
:10205000F749009A4A6000220A701CBD0124002042
:10206000F2E72DE9F0470C461546242200212046D0
:102070000CF0D7F905B9FFDFA87860732888DFF87E
:10208000B0A3401D20F00301AF788946DAF80400C0
:1020900010F0E9FB060000D1FFDF4FF000082660DA
:1020A000A6F8008077B109FB07F1091D0AD0DAF81C
:1020B000040010F0D8FB060000D1FFDF6660C6F810
:1020C000008001E0C4F80480298804F11200BDE812
:1020D000F0470AF05BB82DE9F047804601F11200A5
:1020E0000D4681460AF069F8401DD14F20F00302E9
:1020F0006E7B14462968786810F0E0FB3EB104FB63
:1021000006F2121D03D06968786810F0D7FB05202D
:1021100010F016FD0446052010F01AFD201A0128C3
:1021200002D1786810F094FB49464046BDE8F0477C
:102130000AF042B870B50546052110F059FD0400BB
:1021400000D1FFDF04F112012846BDE870400AF01B
:102150002CB82DE9F04F91B04FF0000BADF828B03E
:10216000ADF804B047880C4605469246052138462E
:1021700010F03EFD060000D1FFDF24B1A780A4F8D7
:1021800006B0A4F808B0297809220B20B2EB111F81
:1021900073D12A7A04F1100138274FF00C084FF060
:1021A00012090291102A69D2DFE802F068F2F1F018
:1021B0008008D3898EA03DDCF3EEB7B7307B0228D0
:1021C00000D0FFDFA88908EBC001ADF80410302172
:1021D000ADF82810002C25D06081B5F80E800027BE
:1021E0001DE004EBC709317C89F80E10F189A9F8CC
:1021F0000C10CDF800806888042305AA296900F036
:1022000035FBBDF81410A9F8101008F10400BDF852
:1022100016107F1C1FFA80F8A9F81210BFB260894F
:10222000B842DED80CE1307B022800D0FFDFE9891C
:1022300008EBC100ADF804003020ADF8280095F897
:102240000C90002CA9F10400C0B20F90EAD061817B
:10225000B5F81080002725E0CDF8008068884B464F
:1022600003AA696900F002FB08EB09001FFA80F875
:102270006F48007818B1012302E0DDE0DAE00023C6
:1022800004EBC702009204A90C320F9812F03BFA3B
:10229000009ABDF80C007F1C1082009ABDF80E0059
:1022A000BFB250826089B842D6D8C9E00AA800906F
:1022B00001AB224629463046FFF711FBC0E0307BD8
:1022C000082805D0FFDF03E0307B082800D0FFDFBF
:1022D000E8891030ADF804003620ADF82800002C55
:1022E0003FD0A9896181F189A18127E0307B09284C
:1022F00000D0FFDFA88901460C30ADF8040037207C
:10230000ADF82800002C2CD06181E8890090AB89C1
:10231000688804F10C02296955E0E88939211030F8
:1023200080B2ADF80400ADF82810002C72D0A98955
:102330006181287A0E280AD002212173E989E1817E
:10234000288A0090EB8968886969029A3BE001213C
:10235000F3E70AA8009001AB224629463046FFF772
:1023600055FB6DE0307B0A2800D0FFDFADF804900C
:10237000ADF828704CB3A9896181A4F810B0A4F815
:102380000EB0012020735BE020E002E030E038E096
:1023900041E0307B0B2800D0FFDF288AADF82870A1
:1023A0001230ADF8040084B104212173A989618140
:1023B000E989E181298A2182688A00902B8A6888CC
:1023C00004F11202696900F051FA39E0307B0C28FF
:1023D00000D0FFDFADF80490ADF828703CB30521C4
:1023E0002173A4F80AB0A4F80EB0A4F810B027E046
:1023F0000AA8009001AB224629463046FFF754FA5E
:102400001EE00AA8009001AB224629463046FFF79D
:10241000B3FB15E034E03B21ADF80400ADF8281023
:1024200074B30120E080A4F808B084F80AB007E093
:1024300010000020FFDF03E0297A012917D0FFDF19
:10244000BDF80400AAF800006CB1BDF82800208097
:10245000BDF804006080BDF82800392803D03C286E
:1024600001D086F80CB011B00020BDE8F08F3C21FF
:10247000ADF80400ADF8281014B1697AA172DFE755
:10248000AAF80000EFE72DE9F84356880F4680468A
:1024900015460521304610F0ABFB040000D1FFDFEC
:1024A000123400943B46414630466A6809F0F8FF12
:1024B000B8E570B50D46052110F09AFB040000D177
:1024C000FFDF294604F11200BDE8704009F082BE2A
:1024D00070B50D46052110F08BFB040000D1FFDF25
:1024E000294604F11200BDE8704009F0A0BE70B5A5
:1024F0000546052110F07CFB040000D1FFDF04F14C
:10250000080321462846BDE870400422AFE470B5B8
:102510000546052110F06CFB040000D1FFDF2146C9
:1025200028462368BDE870400522A0E470B5064641
:10253000052110F05DFB040000D1FFDF04F1120063
:1025400009F03BFE401D20F0030511E0011D00884D
:102550000322431821463046FFF789FC00280BD0A0
:10256000607BABB2684382B26068011D10F0FDF978
:10257000606841880029E9D170BD70B50E460546F6
:1025800007F04AF8040000D1FFDF012020726672D4
:102590006580207820F00F00C01C20F0F000303063
:1025A0002070BDE8704007F03AB8602801D00720DD
:1025B00070470878C54900F0010008700020704796
:1025C0002DE9F0438BB00D461446814606A9FFF76E
:1025D0008AFB002814D14FF6FF7601274FF42058CC
:1025E0008CB103208DF800001020ADF8100007A872
:1025F000059007AA204604A912F0A9F878B107208F
:102600000BB0BDE8F0830820ADF808508DF80E70CF
:102610008DF80000ADF80A60ADF80C800CE006986B
:10262000A17801742188C1818DF80E70ADF8085031
:10263000ADF80C80ADF80A606A4602214846069B58
:10264000FFF77CFBDCE708B501228DF8022042F69B
:102650000202ADF800200A4603236946FFF731FC69
:1026600008BD08B501228DF8022042F60302ADF83C
:1026700000200A4604236946FFF723FC08BD00B585
:1026800087B079B102228DF800200A88ADF80820C1
:102690004988ADF80A1000236A460521FFF74EFB72
:1026A00007B000BD1020FBE709B1072309E40720AC
:1026B000704770B588B00D461446064606A9FFF768
:1026C00012FB00280ED17CB10620ADF808508DF821
:1026D0000000ADF80A40069B6A460821DC813046BE
:1026E000FFF72CFB08B070BD05208DF80000ADF899
:1026F0000850F0E700B587B059B107238DF80030D6
:10270000ADF80820039100236A460921FFF716FB64
:10271000C6E71020C4E770B588B00C460646002511
:1027200006A9FFF7E0FA0028DCD106980121123053
:1027300009F075FD9CB12178062921D2DFE801F06E
:10274000200505160318801E80B2C01EE28880B2E4
:102750000AB1A3681BB1824203D90C20C2E7102042
:10276000C0E7042904D0A08850B901E00620B9E7E9
:10277000012913D0022905D004291CD005292AD00B
:102780000720AFE709208DF800006088ADF8080049
:10279000E088ADF80A00A068039023E00A208DF8D5
:1027A00000006088ADF80800E088ADF80A00A06875
:1027B0000A25039016E00B208DF800006088ADF824
:1027C0000800A088ADF80A00E088ADF80C00A06809
:1027D0000B25049006E00C208DF8000060788DF841
:1027E00008000C256A4629463046069BFFF7A6FAE4
:1027F00078E700B587B00D228DF80020ADF80810FD
:1028000000236A461946FFF799FA49E700B587B0F1
:1028100071B102228DF800200A88ADF8082049889D
:10282000ADF80A1000236A460621FFF787FA37E75A
:10283000102035E770B586B0064601200D46ADF88C
:1028400008108DF80000014600236A463046FFF765
:1028500075FA040008D12946304605F0D7FC00215E
:10286000304605F0F1FC204606B070BDF8B51C46B8
:1028700015460E46069F10F0EEFA2346FF1DBCB229
:1028800031462A4600940FF0D8FEF8BD30B4114608
:10289000DDE902423CB1032903D0002330BC08F03B
:1028A0002CBE0123FAE71A8030BC704770B50C4685
:1028B0000546FFF722FB2146284605F0B6FC2846D0
:1028C000BDE87040012105F0BFBC000010000020F1
:1028D0004FF0E0224FF400400021C2F88001BFF326
:1028E0004F8FBFF36F8F1748016001601649900248
:1028F00008607047134900B500220A600A60124B55
:102900004FF060721A60002808BF00BD0F4A104BDC
:10291000DFF840C001280CD002281CBFFFDF00BD3B
:10292000032008601A604FF4000000BFCCF80000DC
:1029300000BD022008601A604FF04070F6E700B555
:10294000FFDF00BD00F5004008F50140A4020020B3
:1029500014F5004004F5014070B50B2000F0BDF9FE
:10296000082000F0BAF900210B2000F0D4F9002172
:10297000082000F0D0F9F44C01256560A560002026
:10298000C4F84001C4F84401C4F848010B2000F029
:10299000B5F9082000F0B2F90B2000F091F925609C
:1029A00070BD10B50B2000F098F9082000F095F9E3
:1029B000E548012141608160E4490A68002AFCD1B0
:1029C0000021C0F84011C0F84411C0F848110B2094
:1029D00000F094F9BDE81040082000F08FB910B560
:1029E0000B2000F08BF9BDE81040082000F086B9FC
:1029F00000B530B1012806D0022806D0FFDF002044
:102A000000BDD34800BDD34800BDD248001D00BD65
:102A100070B5D1494FF000400860D04DC00BC5F8EB
:102A20000803CF4800240460C5F840410820C4359D
:102A300000F053F9C5F83C41CA48047070BD08B5B0
:102A4000C14A002128B1012811D002281CD0FFDF83
:102A500008BD4FF48030C2F80803C2F84803BB48F1
:102A60003C300160C2F84011BDE80840D0E74FF4A7
:102A70000030C2F80803C2F84803B448403001608F
:102A8000C2F84411B3480CE04FF48020C2F80803A8
:102A9000C2F84803AD4844300160C2F84811AD485F
:102AA000001D0068009008BD70B516460D4604462E
:102AB000022800D9FFDF0022A348012304F11001FE
:102AC0008B4000EB8401C1F8405526B1C1F840218C
:102AD000C0F8043303E0C0F80833C1F84021C0F85F
:102AE000443370BD2DE9F0411D46144630B1012834
:102AF00033D0022838D0FFDFBDE8F081891E0022E4
:102B000021F07F411046FFF7CFFF012D23D0002099
:102B1000944D924F012668703E61914900203C39E6
:102B200008600220091D08608D49042030390860C2
:102B30008B483D34046008206C6000F0DFF83004FE
:102B4000C7F80403082000F0BBF88349F007091F09
:102B500008602E70D0E70120DAE7012B02D00022B6
:102B6000012005E00122FBE7012B04D00022022016
:102B7000BDE8F04198E70122F9E774480068704722
:102B800070B500F0D8F8704C0546D4F84001002626
:102B9000012809D1D4F80803C00305D54FF48030CB
:102BA000C4F80803C4F84061D4F8440101280CD1EA
:102BB000D4F80803800308D54FF40030C4F80803A4
:102BC000C4F84461012012F089FDD4F848010128BD
:102BD0000CD1D4F80803400308D54FF48020C4F882
:102BE0000803C4F84861022012F078FD5E480560D1
:102BF00070BD70B500F09FF85A4D0446287850B16A
:102C0000FFF706FF687818B10020687012F066FDC3
:102C10005548046070BD0320F8E74FF0E0214FF401
:102C20000010C1F800027047152000F067B84B494A
:102C300001200861082000F061B848494FF47C1079
:102C4000C1F808030020024601EB8003C3F84025C9
:102C5000C3F84021401CC0B20628F5D37047410A92
:102C600043F609525143C0F3080010FB02F000F58F
:102C7000807001EB5020704710B5430B48F2376469
:102C800063431B0C5C020C60384C03FB0400384BA4
:102C90004CF2F72443435B0D13FB04F404EB402098
:102CA00000F580704012107008681844086010BD6C
:102CB0002C484068704729490120C1F8000270473C
:102CC000002809DB00F01F0201219140400980002B
:102CD00000F1E020C0F80011704700280DDB00F083
:102CE0001F02012191404009800000F1E020C0F85E
:102CF0008011BFF34F8FBFF36F8F7047002809DB40
:102D000000F01F02012191404009800000F1E02005
:102D1000C0F8801270474907090E002804DB00F153
:102D2000E02080F80014704700F00F0000F1E02070
:102D300080F8141D70470C48001F00680A4A0D49AE
:102D4000121D11607047000000B0004004B5004043
:102D50004081004044B1004008F50140008000403F
:102D6000408500403C00002014050240F7C2FFFFF0
:102D70006F0C0100010000010A4810B50468094900
:102D800009480831086012F03DFD0648001D046046
:102D900010BD0649002008604FF0E0210220C1F874
:102DA000800270471005024001000001FC1F004036
:102DB000374901200860704770B50D2000F049F8D0
:102DC000344C0020C4F800010125C4F804530D2040
:102DD00000F050F825604FF0E0216014C1F80001C8
:102DE00070BD10B50D2000F034F82A480121416073
:102DF0000021C0F80011BDE810400D2000F03AB8E5
:102E0000254810B504682449244808310860214940
:102E1000D1F80001012804D0FFDF1F48001D046025
:102E200010BD1B48001D00680022C0B2C1F800217F
:102E300013F0A1F9F1E710B5164800BFD0F8001162
:102E40000029FBD0FFF7DCFFBDE810400D2000F0AB
:102E500011B800280DDB00F01F020121914040094C
:102E6000800000F1E020C0F88011BFF34F8FBFF366
:102E70006F8F7047002809DB00F01F02012191408D
:102E80004009800000F1E020C0F880127047000087
:102E900004D5004000D000401005024001000001B0
:102EA0004FF0E0214FF00070C1F8800101F5C071D2
:102EB000BFF34F8FBFF36F8FC1F80001394B8022F2
:102EC00083F8002441F8800C704700B502460420C6
:102ED000354903E001EBC0031B792BB1401EC0B2A2
:102EE000F8D2FFDFFF2000BD41F8302001EBC00128
:102EF00000224A718A7101220A7100BD2A4A00210A
:102F000002EBC0000171704710B50446042800D3DD
:102F1000FFDF254800EBC4042079012800D0FFDF43
:102F20006079A179401CC0B2814200D060714FF03D
:102F3000E0214FF00070C1F8000210BD70B504250B
:102F4000194E1A4C16E0217806EBC1000279012ACD
:102F500008D1427983799A4204D04279827156F835
:102F6000310080472078401CC0B22070042801D373
:102F7000002020706D1EEDB2E5D270BD0C4810B57A
:102F800004680B490B4808310860064890F80004B3
:102F90004009042800D0FFDFFFF7D0FF0448001DE0
:102FA000046010BD19E000E0DC050020580000209E
:102FB00010050240010000010548064A01689142DF
:102FC00001D1002101600449012008607047000020
:102FD0005C000020BEBAFECA40E5014070B50C4658
:102FE000054609F0F9FB21462846BDE870400AF085
:102FF000DABC7047704770470021016081807047DC
:103000002CFFFFFFDBE5B151006002000101FFFF73
:103010008400000090D76A00773D4B16B620AFF9C8
:10302000F4D1D1B6F33F7AC76170DB6D30B5F84D9E
:103030000446062CA9780ED2DFE804F0030E0E0E2B
:103040000509FFDF08E0022906D0FFDF04E00329BD
:1030500002D0FFDF00E0FFDFAC7030BD30B50446CA
:103060001038EB4D07280CD2DFE800F0040C060CFA
:103070000C0C0C00FFDF05E0287E112802D0FFDFDA
:1030800000E0FFDF2C7630BD2DE9F04111F0CAFCE5
:10309000044612F0FDFE201AC5B206200FF050FDC6
:1030A000044606200FF054FD211AD94C207E122828
:1030B00018D000200F1807200FF042FD0646072009
:1030C0000FF046FD301A3918207E13280CD000204E
:1030D0000144A078042809D000200844281AC0B26E
:1030E000BDE8F0810120E5E70120F1E70120F4E7E8
:1030F000C74810B590F825004108C54800F12600E2
:1031000005D00DF02BFEBDE8104006F0A7B80DF07D
:1031100006FEF8E730B50446A1F120000D460A2866
:103120004AD2DFE800F005070C1C2328353A3F445B
:10313000FFDF42E0207820283FD1FFDF3DE0B448A8
:103140008178052939D0007E122836D020782428AD
:1031500033D0252831D023282FD0FFDF2DE0207851
:1031600022282AD0232828D8FFDF26E0207822280A
:1031700023D0FFDF21E0207822281ED024281CD075
:1031800026281AD0272818D0292816D0FFDF14E0C7
:103190002078252811D0FFDF0FE0207825280CD0DB
:1031A000FFDF0AE02078252807D0FFDF05E0207840
:1031B000282802D0FFDF00E0FFDF257030BD1FB5FB
:1031C00004466A46002001F0A7FEB4B1BDF8022013
:1031D0004FF6FF700621824201D1ADF80210BDF812
:1031E0000420824201D1ADF80410BDF808108142DC
:1031F00003D14FF44860ADF8080068460EF092F92C
:1032000006F02CF804B010BD70B514460D46064605
:10321000FEF71FF858B90DB1A54201D90C2070BDB9
:10322000002408E056F82400FEF713F808B1102037
:1032300070BD641CE4B2AC42F4D3002070BD2DE933
:10324000F04105461F4690460E4600240068FEF7F2
:103250004DF830B9A98828680844401EFEF746F8A2
:1032600008B110203CE728680028A88802D0B8429E
:1032700002D850E00028F5D0092031E72968085D20
:10328000B8B1671CCA5D152A2ED03CDC152A3AD28B
:10329000DFE802F03912222228282A2A313139396E
:1032A00039393939393939392200085D30BB641C64
:1032B000A4B2A242F9D833E00228DDD1A01C085CF8
:1032C00088F80000072801D2400701D40A2007E748
:1032D000307840F0010015E0C143C90707E001283C
:1032E00007D010E00620FBE60107A1F1805100297C
:1032F000F5D01846F4E63078810701D50B20EFE6CB
:1033000040F0020030702868005D384484B2A8881C
:10331000A04202D2B0E74FF4485382B2A242ADD8E5
:103320000020DDE610B5027843F2022354080122A2
:10333000022C12D003DC3CB1012C16D106E0032C88
:1033400010D07F2C11D112E0002011E080790324ED
:10335000B4EB901F09D10A700BE08079B2EB901F9B
:1033600003D1F8E780798009F5D0184610BDFF2019
:103370000870002010BD08B500208DF8000024481A
:1033800090F82E1049B190F82F0002280ED0032893
:103390000ED0FFDF9DF8000008BD1D4869462530AE
:1033A00001F009FE0028F5D0FFDFF3E7032000E07D
:1033B00001208DF80000EDE738B50C46054669465A
:1033C00001F0F9FD00280DD19DF80010207861F37F
:1033D0004700207055F8010FC4F80100A888A4F830
:1033E0000500002038BD38B51378A8B1022813D0E5
:1033F000FF281AD007A46D46246800944C7905EB89
:103400009414247864F347031370032809D00FE061
:10341000F00100200302FF0123F0FE0313700228D5
:10342000F3D1D8B240F0010005E043F0FE00107087
:10343000107820F0010010700868C2F80100888838
:10344000A2F8050038BD02210FF0D2BB38B50C46FA
:103450000978222901D2082038BDADF800008DF886
:10346000022068460DF0BCFC05F0F8FE050003D113
:1034700021212046FFF74EFE284638BD1CB500200E
:103480008DF80000CDF80100ADF80500FE4890F879
:103490002E00022801D0012000E000208DF8070056
:1034A00068460DF023FD002800D0FFDF1CBD002280
:1034B0000A80437892B263F3451222F040020A80F8
:1034C00000780C282BD2DFE800F02A06090E11162E
:1034D000191C1F220C2742F0110009E042F01D00C8
:1034E00008800020704742F0110012E042F0100006
:1034F00040F00200F4E742F01000F1E742F0010072
:10350000EEE742F0010004E042F00200E8E742F09A
:10351000020040F00400E3E742F00400E0E7072087
:1035200070472DE9FF478AB00025BDF82C60824620
:103530001C4690468DF81C50700703D56068FDF757
:1035400088FE68B9D04F4FF0010997F82E0058B1A6
:1035500097F82F00022807D16068FDF7C7FE18B161
:1035600010200EB0BDE8F087300702D5A089802872
:1035700016D8700705D4B8F1000F02D097F82400D0
:1035800070B1E07DC0F300108DF81B00617D072055
:1035900041B1012906D00229E3D00429E1D12CE070
:1035A0000720DEE749468DF81790F00609D4A27D82
:1035B000072032B1012A04D0022A05D0042AD0D132
:1035C0001BE08DF8191002E002208DF819008DF82B
:1035D00015806068B0B107A9FFF7A4FE0028C0D12C
:1035E0009DF81C00FF280AD0606850F8011FCDF834
:1035F0000F108088ADF8130008E00620B1E743F211
:103600000220AEE7CDF80F50ADF81350E07B002854
:10361000F3D1207C0028F0D1607C0028EDD1A07C83
:103620000028EAD1E07CC006E7D18DF800A0BDF803
:103630002C00ADF80200A0680190A068029004F18F
:103640000F0001F0ACFC8DF80C00FFF794FE8DF834
:103650000D009DF81C008DF80E008DF816508DF8A9
:103660001850E07D08A900F00F008DF81A00684698
:103670000EF0A0F805F0F2FD73E7F0B58FB000256D
:103680008DF830508DF814508DF8345006468DF872
:103690002850019502950395049519B10FC901AC05
:1036A00084E80F00784CA078052801D004280CD1BC
:1036B00001986168884200D120B90398E168884286
:1036C00003D110B108200FB0F0BD207DC00601D598
:1036D0001F2700E0FF273B460DAA05A903A8FFF717
:1036E000AEFD0028EFD1A08AC10702D0C00600D4E9
:1036F000EE273B460AAA0CA901A8FFF7A0FD002867
:10370000E1D19DF81400C00701D00A20DBE7A08AB0
:10371000410708D4A17D31B19DF82810890702D056
:1037200043F20120CFE79DF82810C90709D04007D0
:1037300007D4208818B144F25061884201D907208B
:10374000C1E78DF818508DF81960BDF80800ADF884
:103750001A000198079006A80EF038F805F07EFDD3
:103760000028B0D18DF820508DF82160BDF81000F0
:10377000ADF822000398099008A80EF049F805F06A
:103780006DFD00289FD101AD241D95E80F0084E850
:103790000F00002097E770B586B00D46040005D0F5
:1037A000FDF7A4FD20B1102006B070BD0820FBE796
:1037B0002078C107A98802D0FF2902D303E01F297E
:1037C00001D20920F0E780073BD4FFF75DFC38B158
:1037D0002178C1F3C100012804D0032802D005E0FC
:1037E0001320E1E7284890F82400C8B1C8074FF03B
:1037F00001064FF0000502D08DF80F6001E08DF852
:103800000F50FFF7B8FD8DF8000020786946C0F32F
:10381000C1008DF8010060788DF80250C20801D017
:103820000720C1E778B1C20701D08DF80260820796
:1038300005D59DF8022042F002028DF802204007D3
:1038400003D50620B0E78DF80260002022780B181F
:10385000C2F38002DA7001EB40026388D380401C1F
:10386000A388C0B253810228F0D3207A0028E8D17F
:10387000607A0028E5D1A07A0028E2D1E07A002819
:10388000DFD1207BC00601E0F0010020D9D104F196
:10389000080001F084FB8DF80E0068460DF0F3FB84
:1038A00005F0DCFC00288DD18DF810608DF81150EA
:1038B000E088ADF81200ADF8145004A80DF036FC05
:1038C00005F0CCFC00288CD12078C00701D0152051
:1038D00000E01320FFF7C2FB002065E72DE9FF475A
:1038E0000220FD4E8DF804000027708EADF8060012
:1038F000B84643F202094CE001A80FF0E0F80500D9
:1039000006D0708EA8B3A6F83280ADF806803EE0EF
:10391000039CA07F01072DD504F124000090A28E06
:10392000BDF80800214604F1360301F0CFFC050084
:1039300005D04D452AD0112D3CD0FFDF3AE0A07FC5
:1039400020F00801E07F420862F3C711A1778108E7
:1039500061F30000E07794F8210000F01F0084F884
:1039600020002078282826D129212046FFF7D2FBE5
:1039700021E014E040070AD5BDF8080004F10E016B
:1039800001F023FB05000DD04D4510D100257F1C13
:10399000FFB202200FF0D4F8401CB842ACD8052D7D
:1039A00011D008E0A07F20F00400A07703E0112DE3
:1039B00000D0FFDF0025BDF806007086052D04D07D
:1039C000284604B0CEE5A6F832800020F9E770B5AD
:1039D0000646FFF738FD054605F01EFE040000D13F
:1039E000FFDF6680207820F00F00801C20F0F000C0
:1039F000203020700320207295F83E006072BDE8F0
:103A0000704005F00CBE2DE9F04786B0040000D1EF
:103A1000FFDF2078B04D20F00F00801C20F0F00078
:103A20007030207060680178491F1B2933D2DFE8AD
:103A300001F0FC32323255FB320EFBFB42FA3232DD
:103A40003278FAFAF9F832FAFAF7F6FAFA00C68892
:103A50003046FFF7F8FC0546304607F044FCE0B17D
:103A60006068007A85F83E0021212846FFF752FB66
:103A70003046FEF75FFB304603F0ECFE3146012096
:103A800012F03EFEA87F20F01000A877FFF726FF77
:103A9000002800D0FFDF06B064E5207820F0F000B9
:103AA000203020700320207266806068007A607287
:103AB00005F0B5FDD8E7C5882846FFF7C4FC00B976
:103AC000FFDF60680079012800D0FFDF6068017ABD
:103AD00006B02846BDE8F04707F0EABDC688304684
:103AE000FFF7B1FC050000D1FFDF05F098FD60682D
:103AF00031460089288160684089688160688089D2
:103B0000A881012012F0FCFD0020A875A87F00F01C
:103B100003000228BFD1FFF7E1FE0028BBD0FFDF82
:103B2000B9E7007928B10228B5D03C28B3D0FFDF2F
:103B3000B1E705F074FD6668B6F806A0307A361D68
:103B4000012806D0687E814605F0F4FA070003D10B
:103B500001E0E878F7E7FFDF0022022150460FF08E
:103B60003EF8040000D1FFDF22212046FFF7D2FA01
:103B70003079012800D00220A17F804668F301013E
:103B8000A177308B2081708B6081B08BA08184F80D
:103B900022908DF80880B8680090F86801906A4615
:103BA000032150460FF01BF800B9FFDFB888ADF8CD
:103BB0001000B8788DF8120004AA052150460FF0C5
:103BC0000EF800B9FFDFB888ADF80C00F8788DF872
:103BD0000E0003AA042150460FF001F800B9FFDFE0
:103BE000062106F1120001F00EFA40B37079800749
:103BF00000D5FFDF7179E07D61F34700E075D6F80D
:103C00000600A0617089A083062106F10C0001F076
:103C1000FAF9F0B195F825004108607806E043E034
:103C20003BE072E05AE04FE031E045E061F34700ED
:103C30006070D5F82600C4F80200688D12E0E07DBF
:103C400020F0FE00801CE075D6F81200A061F08A1A
:103C5000D9E7607820F0FE00801C6070F068C4F83E
:103C60000200308AE080B8F1010F04D0B8F1020FF1
:103C700005D0FFDF0FE70320FFF7D8F90BE7287E19
:103C8000122800D0FFDF1120FFF7E8F903E706B0A4
:103C90002046BDE8F04701F0A5BD05F0C0FC15F8D1
:103CA000300F40F0020005E005F0B9FC15F8300FC8
:103CB00040F004002870EEE6287E132809D015286D
:103CC000D8D11620FFF7CAF906B0BDE8F04705F0D5
:103CD000A6BC1420F6E70000F0010020A978052911
:103CE00009D00429C6D105F09AFC022006B0BDE82F
:103CF000F047FFF79BB900790028BBD0E87801F0C6
:103D000035F905F08CFC0320F0E7287E122802D15B
:103D1000687E01F02BF91120D4E72DE9F05F05460C
:103D200000784FF000080009DFF8B4A891460C466F
:103D3000464601286ED002286DD007280BD00A28ED
:103D40006AD0FFDFA9F8006014B1A4F80080668093
:103D50000020BDE8F09F6968012704F108000B7896
:103D60004FF0020B5B1F4FF6FF721B2B7ED2DFE87A
:103D700003F0647D7D7D0E7D7D7D7D7D7D217D7D5E
:103D80007D2BFDFCFBFA7D14D2F9E7F8F700C8881B
:103D90004FF01208102621469AE14FF01C080A261F
:103DA000BCB38888A0806868807920726868C07910
:103DB0006072C7E74FF01B08142654B3032020722B
:103DC00068688088A080BDE70A793C2ABAD00D1DBA
:103DD0004FF010082C26E4B16988A180298B6182FC
:103DE000298B2182698BA182A98BE1826B790246A2
:103DF000A91D1846FFF7F7FA2979002001290CD0F0
:103E000084F80FB0FF212176E06120626062A06239
:103E100098E70FE03BE15EE199E1E77320760AF174
:103E2000040090E80E00DAF81000C4E90930C4E993
:103E3000071287E7A9F800608AE72C264FF01D08D3
:103E4000002CF7D0A28005460F1D897B008861F306
:103E500000002880B97A490861F341002880B97AC6
:103E6000890861F382002880B97A00E00CE1C90872
:103E700061F3C3002880B97AAA1C0911491C61F3B7
:103E8000041000F07F0028807878B91CFFF7ABFAA7
:103E9000387D05F1090207F11501FFF7A4FA387B17
:103EA00001F0C0F82874787B01F0BCF86874F87EE3
:103EB000A874787AE874387F2875B87B6875388A72
:103EC000E882DAF81C10A961B97A504697F808A080
:103ED000C1F34111012904D0008C504503D2824620
:103EE00009E0FFDF10E0022903D0288820F06000FD
:103EF00009E0504504D1288820F06000403002E0FD
:103F0000288840F060002880A4F824A0524607F1D9
:103F10001D01A8699BE011264FF02008002C89D0D4
:103F2000A280686804F10A02007920726868007B48
:103F3000607269688B1D48791946FFF754FA01E7EA
:103F40000A264FF02108002CE9D08888A0806868F4
:103F5000807920726868C07960729AF8301006E043
:103F600078E06BE052E07FE019E003E03AE021F016
:103F70000401A6E00B264FF02208002CCFD0C88801
:103F8000A0806868007920726868007A01F04AF8B9
:103F900060726868407A01F045F8A072D2E61C268B
:103FA0004FF02608002CBAD0A28068684079607271
:103FB0006868007AA0720AF1040090E80E00DAF84E
:103FC0001000C4E90530C4E90312686800793C2890
:103FD00003D0432803D0FFDFB4E62772B2E684F8AB
:103FE00008B0AFE610264FF02408002C97D0888840
:103FF000A0806868807920816868807A60816868BC
:104000000089A08168688089E0819BE610264FF0D6
:104010002308002C98D08888A0806868C0882081F8
:1040200068680089608168684089A08168688089C3
:10403000E0819AF8301021F0020142E030264FF082
:104040002508002C9AD0A2806968282249680AF0C5
:10405000BEF977E62A264FF02F08002C8ED0A280DA
:1040600069682222091DF2E714264FF01B08002C74
:1040700084D0A280686800790128B0D02772DAE97C
:104080000710C4E903105DE64A46214660E0287A3D
:10409000012803D0022817D0FFDF53E610264FF087
:1040A0001F08002CA2D06888A080A8892081E889F8
:1040B0006081288AA081688AE0819AF8301021F016
:1040C00001018AF830103DE64FF01208102668888A
:1040D00000F086FF36E6287AC8B3012838D00228D7
:1040E00036D0032801D0FFDF2CE609264FF0110857
:1040F000002C8FD06F883846FFF7A5F990F822A0E2
:10410000A780687A2072042138460EF083FD0521CD
:1041100038460EF07FFD002138460EF07BFD012170
:1041200038460EF077FD032138460EF073FD02216C
:1041300038460EF06FFD062138460EF06BFD072164
:1041400038460EF067FD504600F010FFFAE5FFE735
:104150002846BDE8F05F01F0CFBC70B5012803D060
:10416000052800D0FFDF70BD8DB22846FFF76BF940
:10417000040000D1FFDF20782128F4D005F04CFAAC
:1041800080B1017821F00F01891C21F0F00110317C
:1041900001700221017245800020A075BDE87040C9
:1041A00005F03DBA21462846BDE870401322FFF7CE
:1041B0004DB92DE9F04116460C00804600D1FFDFD5
:1041C000307820F00F00801C20F0F00010303070AC
:1041D0002078012804D0022818D0FFDFBDE8F08144
:1041E0004046FFF730F9050000D1FFDF0320A87536
:1041F00005F015FA94E80F00083686E80F00F84835
:1042000010F8301F41F001010170E7E74046FFF769
:104210001AF9050000D1FFDFA1884FF6FF700027D3
:10422000814202D1E288824203D0814201D1E088FA
:1042300040B105F0F4F994E80F00083686E80F0065
:10424000AF75CBE7A87D0128C8D17823002241466D
:1042500012F0ACF90220A875C0E738B50C46242846
:104260005ED008DC20280FD0212825D022284DD070
:10427000232806D14EE0252841D0262832D03F28D9
:1042800053D00725284638BD0021052012F00EFA2C
:1042900008B1112038BDA01C0DF097F904F0DEFF25
:1042A0000500EFD1002208231146052012F07EF907
:1042B0000528E7D0FFDFE5E76068FDF70EF808B1F5
:1042C000102038BD618820886A460DF032FC04F069
:1042D000C5FF0500D6D160680028D3D0BDF8001016
:1042E0000180CFE7206820B1FDF700F808B1102564
:1042F000C8E720460DF0ECFC1FE00546C2E7A078B9
:1043000000F0010120880DF045FC16E0086801F07E
:104310009FFEF2E7087800F001000CF0F3FC0CE0DF
:10432000618820880DF081FB07E0087800F001002B
:104330008DF8000068460CF0B0FF04F08FFFDCE75A
:1043400070B505460C460846FCF7A9FF08B11020D9
:1043500070BD202D07D0212D0DD0222D0BD0252D65
:1043600009D0072070BD2088A11C0CF09DFDBDE880
:10437000704004F073BF062070BD99482530704727
:1043800008B53422002196480AF04BF80120FEF7C8
:104390004DFE1120FEF762FE91496846263105F078
:1043A000D1F88F489DF8002010F8251F62F34701CF
:1043B00021F001010170002141724FF46171A0F8F8
:1043C000071002218172FEF793FE00B1FFDFFDF7B7
:1043D00009F801F0D0F908BD10B50C4640220021C3
:1043E00020460AF01EF8A07F20F00300A0772020CE
:1043F00020700020A07584F8230010BD70472DE9BF
:10440000FC410746FCF725FF10B11020BDE8FC81F8
:10441000734E06F12501D6F825000090B6F8295014
:10442000ADF8045096F82B408DF806403846FEF75C
:10443000C3FF0028EAD1FEF75BFE0028E6D0009912
:1044400046F8251FB580B471E0E710B50446FCF7C7
:1044500026FF08B1102010BD61486149224690F83E
:10446000250026314008FEF7BEFF002010BD3EB5F6
:1044700004460D460846FCF712FF08B110203EBD69
:1044800014B143F204003EBD55488078052803D09E
:10449000042801D008203EBD694602A80AF0C9FBE5
:1044A0002A4669469DF80800FEF79DFF00203EBDA4
:1044B000FEB50D4604004FF0000712D00822FEF7AB
:1044C000A3FE002812D1002609E000BF54F8260000
:1044D0006946FEF727FF002808D1761CF6B2AE42E7
:1044E000F4D30CF059FB10B143F20320FEBD3C4E57
:1044F00086F824700CB300271BE000BF54F8270097
:1045000002A9FEF70FFF00B1FFDF9DF808008DF84C
:10451000000054F8270050F8011FCDF801108088E2
:10452000ADF8050068460CF05CFB00B1FFDF7F1CB6
:10453000FFB2AF42E2D386F824500020FEBD2DE941
:10454000F0478AB01546894604001FD00F4608225E
:104550002946FEF759FE002811D1002614E000BFBD
:1045600054F826006946103000F025FD002806D1D9
:1045700047B157F82600FCF76CFE18B110200AB0BE
:10458000BDE8F087761CF6B2AE42E9D30026A5F16D
:1045900001081BE006F1010A0AF0FF0712E000BF64
:1045A00054F82600017C4A0854F827100B7CB2EB23
:1045B000530F05D106221130113109F0DBFE58B13D
:1045C0007F1CFFB2AF42EBD30AF0FF064645E1DBAA
:1045D0004E463CB1012006E043F20520CFE7000043
:1045E000F001002000200CF021FB10B90CF02AFB98
:1045F00010B143F20420C2E764B300270DF117089D
:1046000026E000BF54F827006946103000F0D3FCC4
:1046100000B1FFDF54F82700102250F8111FCDF829
:1046200001108088ADF8050054F827100DF107003F
:1046300009F0CDFE96B156F827101022404609F039
:10464000C6FE68460CF0B2FA00B1FFDF7F1CFFB275
:10465000AF42D7D3FEF712FF002090E7404601F0AB
:10466000EBFCEEE730B585B00446FDF7BBF830B99A
:1046700006200EF065FA10B1062005B030BD2046C8
:10468000FCF7E7FD18B96068FCF730FE08B11020B0
:10469000F3E760884AF2B811884206D82078F94DCD
:1046A00028B1012806D0022804D00720E5E7FEF74C
:1046B0001FFD18E06078022804D0032802D043F2DE
:1046C0000220DAE785F82F00C1B200200090ADF893
:1046D000040002292CD0032927D0FFDF68460CF004
:1046E0003DFB04F0BBFD0028C7D1606801F097FCDA
:1046F000207858B101208DF800000DF1010001F083
:104700009BFC68460DF0ABFA00B1FFDF207885F81E
:104710002E00FEF7B3FE608860B1A88580B20CF071
:104720007DFA00B1FFDF0020A7E78DF80500D5E78F
:104730004020FAE74FF46170EFE710B50446FCF74C
:10474000AEFD20B9606838B1FCF7C7FD08B1102094
:1047500010BD606801F070FCCA4830F82C1F618001
:10476000C178617080782070002010BD2DE9F84379
:10477000144689460646FCF792FDA0B94846FCF768
:10478000B5FD80B92046FCF7B1FD60B9BD4DA878F4
:10479000012800D13CB13178FF2906D049B143F25C
:1047A0000400BDE8F8831020FBE7012801D00420B5
:1047B000F7E7CCB3052811D004280FD0694620466E
:1047C000FEF775FE0028ECD1217D49B1012909D001
:1047D000022909D0032909D00720E2E70820E0E7F1
:1047E000024604E0012202E0022200E003228046A9
:1047F0002346174600200099FEF793FE0028D0D1EB
:10480000A0892880A07BE875BDF80000A882AF755C
:10481000BDF80010090701D5A18931B1A18929800E
:10482000C00704D0032003E006E08021F7E7022060
:10483000FEF7FCFB86F800804946BDE8F8430020FF
:10484000FEF71BBF7CB58F4C05460E46A0780228AC
:1048500003D0032801D008207CBD15B143F2040029
:104860007CBD07200EF074F910B9A078032806D09B
:10487000FEF70AFC28B1A078032804D009E0122032
:104880007CBD13207CBD304600F053FB0028F9D1DD
:10489000E670FEF770FD0AF009F901208DF80000BE
:1048A0008DF801008DF802502088ADF80400E07DFD
:1048B0008DF8060068460DF07BF804F0CFFC002868
:1048C000E0D1A078032805D05FF00400FEF7AEFB2E
:1048D00000207CBDE07800F03CFB0520F6E71CB52D
:1048E00010B143F204001CBD664CA078042803D02C
:1048F000052801D008201CBD00208DF800000121F2
:104900008DF801108DF8020068460DF051F804F0A2
:10491000A5FC0028EFD1A078052805D05FF00200A3
:10492000FEF784FB00201CBDE07800F01FFB032095
:10493000F6E72DE9FC4180460E4603250846FCF7C4
:10494000D5FC002866D14046FEF77DFD040004D06A
:104950002078222804D2082058E543F2020055E5C9
:10496000A07F00F003073EB1012F0CD0002031469C
:10497000FEF725FC0500EFD1012F06D0022F1AD03B
:10498000FFDF284642E50120F1E7A07D31460228FD
:1049900001D011B107E0112038E56846FCF756FE5A
:1049A0000028D9D16946404606F045FE0500E8D109
:1049B0000120A075E5E7A07D032804D1314890F8D7
:1049C0003000C00701D02EB30EE026B1A07F400713
:1049D0001ED4002100E00121404606F04CFE0500F7
:1049E000CFD1A075002ECCD03146404600F0EDFA74
:1049F00005461128C5D1A07F4107C2D4316844F8CB
:104A00000E1F7168616040F0040020740025B8E753
:104A10001125B6E71020F9E470B50C460546FEF7FF
:104A200012FD010005D022462846BDE87040FEF781
:104A30000DBD43F2020070BD10B5012807D1114B26
:104A40009B78012B00D011B143F2040010BD0CF093
:104A500017F9BDE8104004F001BC012300F090BA42
:104A600000231A46194600F08BBA70B506460C466C
:104A70000846FCF7EEFB18B92068FCF710FC18B1EB
:104A8000102070BDF0010020F84D2A7E112A04D0BC
:104A9000132A00D33EB10820F3E721463046FEF743
:104AA0007AFE60B1EDE70920132A0DD0142A0BD04D
:104AB000A188FF29E5D31520FEF7D0FA0020D4E91C
:104AC0000012C5E90712DCE7A1881F29D9D31320FA
:104AD000F2E71CB5E548007E132801D208201CBD72
:104AE00000208DF8000068460CF020FB04F0B6FBB7
:104AF0000028F4D11120FEF7B1FA00201CBD2DE9E9
:104B0000F04FDFF868A3814691B09AF818009B46F1
:104B100015460C46132803D3FFF7DBFF00281FD1EF
:104B20002046FCF796FB78BB2846FCF792FB58BB67
:104B300020784FF00107C0074FF0000102D08DF838
:104B40003A7001E08DF83A1020788846C0F3C10031
:104B50008DF8000060788DF80910C10803D0072097
:104B600011B0BDE8F08F80B1C10701D08DF8097098
:104B7000810705D59DF8091041F002018DF8091053
:104B8000400704D50620EBE720E08DF809709DF87A
:104B90000900810703D540F001008DF809000020CD
:104BA0006E4606EB400162884A81401CA288C0B272
:104BB0000A820328F5D32078C0F3C100012821D050
:104BC00003281FD04846FCF744FB08B11020C7E774
:104BD00099F80000400808D0012809D0022807D021
:104BE000032805D043F20220BAE78DF8028001E0E5
:104BF0008DF80270484650F8011FCDF803108088E8
:104C0000ADF80700FEF7B7FB8DF801000020424623
:104C100006EB40012B88CB826B888B83AB884B845F
:104C2000EB880B85401CCA85C0B28A860328EFD367
:104C3000E088ADF83C0068460CF025FB00288ED1DA
:104C40009AF818005546112801D0082088E7062058
:104C50000DF07EFF38B12078C0F3C100012804D0E8
:104C6000032802D006E012207AE795F824000028F5
:104C70003FF475AFFEF708FA022801D213206FE760
:104C8000584600F056F90028A1D185F819B06846B9
:104C90000CF022FC04F0E2FA040098D1687E00F0E7
:104CA00058F91220FEF7DAF9204659E770B56F4D32
:104CB000287E122801D00820E3E60CF010FC04F056
:104CC000CDFA040005D1687E00F050F91120FEF7FE
:104CD000C5F92046D5E670B5064615460C46084689
:104CE000FCF7DDFA18B92846FCF7D9FA08B110200C
:104CF000C7E62A46214630460CF0FBFE04F0AEFA29
:104D00000028F5D121787F29F2D10520B9E67CB5BC
:104D100005460C460846FCF79CFA08B110207CBDFD
:104D20002846FEF790FB20B10078222804D2082004
:104D30007CBD43F202007CBD4C4890F83000400737
:104D400001D511207CBD2178C80802D16078C20845
:104D500001D007207CBD890801D1800801D0062040
:104D60007CBDADF8005020788DF8020060788DF899
:104D700003000220ADF8040068460BF076FD04F055
:104D80006DFA7CBD70B586B014460D460646FEF73A
:104D90005AFB28B10078222805D2082006B070E618
:104DA00043F20200FAE72846FCF7A0FA20B944B122
:104DB0002046FCF792FA08B11020EFE700202060AF
:104DC000A0802A4890F83000800701D51120E5E73F
:104DD00003A930460BF086FD18B100BF04F03EFA7F
:104DE000DCE7ADF80060BDF81400ADF80200BDF8D6
:104DF0001600ADF80400BDF81000BDF81210ADF8B3
:104E00000600ADF808107DB1298809B1ADF806108B
:104E1000698809B1ADF80210A98809B1ADF8081088
:104E2000E98809B1ADF80410DCB1BDF80610814283
:104E300001D9081A2080BDF80210BDF81400814283
:104E400001D9081A6080BDF80800BDF80410BDF84B
:104E500016200144BDF812001044814201D9081AFD
:104E6000A08068460BF00CFEB8E70000F0010020BF
:104E70001CB572490968CDE9001068460CF005FAC6
:104E800004F0ECF91CBD1CB50020009001906846B0
:104E90000CF0FBF904F0E2F91CBD70B505460C46B8
:104EA0000846FCF7FCF908B11020EAE5214628463F
:104EB0000CF044F8BDE8704004F0D0B93EB50546AA
:104EC0000C460846FCF7EBF908B110203EBD002067
:104ED000009001900290ADF800502089ADF80800D4
:104EE00020788DF80200606801902089ADF80800F4
:104EF0006089ADF80A0068460CF032F804F0AEF9AB
:104F00003EBD0EB5ADF800000020019068460CF0E3
:104F100027F804F0A3F90EBD108008885080488857
:104F20009080C88810818888D0800020508190812E
:104F3000704710B5044604F0FDF830B1407830B148
:104F4000204604F010FC002010BD052010BD1220EA
:104F500010BD10B504F0EEF8040000D1FFDF60785A
:104F600000B9FFDF6078401E607010BD10B504F01E
:104F7000E1F8040000D1FFDF6078401C607010BDD4
:104F80001CB5ADF800008DF802308DF803108DF8D7
:104F9000042068460CF070FD04F060F91CBD0CB5EF
:104FA00027A2D2E90012CDE900120079694601EB8F
:104FB000501000780CBD0278520804D0012A02D0AB
:104FC00043F202207047FEF7ADB91FB56A46FFF7FE
:104FD000A3FF68460CF0B6FA04F040F904B010BD27
:104FE00070B50C0006460DD0FEF72DFA050000D175
:104FF000FFDFA68028892081288960816889A081B7
:10500000A889E0813DE510B500231A4603E0845CE1
:105010002343521CD2B28A42F9D30BB1002010BDF7
:10502000012010BD00B530B1012803D0022801D005
:10503000FFDF002000BDFF2000BD0000F45502008E
:10504000070605040302010010B50446FCF701F948
:1050500008B1102010BD2078C0F30210042807D832
:105060006078072804D3A178102901D8814201D2A1
:10507000072010BDE078410706D421794A0703D400
:10508000000701D4080701D5062010BD002010BD7F
:1050900010B513785C08837F64F3C71383771378A4
:1050A0009C08C37F64F30003C3771078C309487872
:1050B00063F34100487013781C090B7864F34713BD
:1050C0000B701378DB0863F3000048705078487168
:1050D00010BD10B5C4780B7864F300030B70C4786E
:1050E000640864F341030B70C478A40864F382037A
:1050F0000B70C478E40864F3C3030B700379117870
:1051000063F30001117003795B0863F341011170CF
:1051100003799B0863F3820111700079C00860F382
:10512000C301117010BD70B514460D46064604F05B
:1051300073FA80B10178182221F00F01891C21F047
:10514000F001A03100F8081B214609F040F9BDE844
:10515000704004F064BA29463046BDE8704013221E
:10516000FEF774B92DE9F047064608A8904690E886
:10517000300489461F4614220021284609F051F9BF
:105180000021CAF80010B8F1000F03D0B9F1000FE8
:1051900003D114E03878C00711D02068FCF77FF8FD
:1051A000C0BBB8F1000F07D120681230286020681A
:1051B000143068602068A8602168CAF80010387848
:1051C000800724D56068FCF788F818BBB9F1000F98
:1051D00021D0FFF7D2F80168C6F868118188A6F8D7
:1051E0006C11807986F86E0101F015FDF94FEF60C2
:1051F000626862B196F8680106F2691140081032DF
:10520000FEF7F1F810223946606809F0E0F8002056
:10521000BDE8F08706E0606820B1E8606068C6F825
:105220006401F4E71020F3E730B5054608780C4632
:1052300020F00F00401C20F0F00110312170002000
:10524000607095F8230030B104280FD0052811D0E4
:10525000062814D0FFDF20780121B1EB101F04D203
:1052600095F8200000F01F00607030BD21F0F000C4
:10527000203002E021F0F00030302070EBE721F028
:10528000F0004030F9E7F0B591B0022715460C4622
:1052900006463A46ADF80870092103AB05F04FF811
:1052A0000490002810D004208DF804008DF80170BF
:1052B000E034099605948DF818500AA968460FF055
:1052C00092F900B1FFDF012011B0F0BD10B588B038
:1052D0000C460A99ADF80000CBB11868CDF8020071
:1052E000D3F80400CDF80600ADF80A20102203A878
:1052F00009F06DF868460CF095F903F0AFFF00284F
:1053000003D1A17F41F01001A17708B010BD0020AA
:10531000CDF80200E6E72DE9F84F0646808A0D46F3
:1053200080B28246FEF78FF804463078DFF8A48218
:1053300000274FF00209A8F120080F2870D2DFE8FB
:1053400000F06FF23708387D8CC8F1F0EFF35FF3AF
:10535000F300A07F00F00300022809D05FF00000F6
:1053600080F0010150460DF043FC050003D101E03F
:105370000120F5E7FFDF98F85C10C90702D0D8F8E4
:1053800060000BE0032105F11D0010F0D2FED5F8FE
:105390001D009149B0FBF1F201FB1200C5F81D00A0
:1053A00070686867B068A8672078252800D0FFDF9C
:1053B000CAE0A07F00F00300022809D05FF00000DF
:1053C00080F0010150460DF013FC060003D101E00E
:1053D0000120F5E7FFDF3078810702D52178252904
:1053E00004D040F001003070BDE8F88F85F80090DF
:1053F000307F287106F11D002D36C5E90206F3E75E
:10540000A07F00F00300022808D0002080F00101F6
:1054100050460DF0EDFB040004D102E00120F5E759
:10542000A7E1FFDF2078C10604D5072028703D34AE
:105430006C60D9E740F008002070D5E7E07F0007F6
:1054400000D5FFDF307CB28800F0010301B0504688
:10545000BDE8F04F092106F050B804B9FFDF7168CC
:1054600021B1102204F1240008F0B1FF28212046C8
:10547000FDF750FEA07F00F0030002280ED104F1DA
:105480002400002300901A4621465046FFF71EFFD5
:10549000112807D029212046FDF73CFE307A84F8F8
:1054A0002000A1E7A07F000700D5FFDF14F81E0F42
:1054B00040F008002070E782A761E761C1096078C9
:1054C00061F34100014660F382016170307AE0705F
:1054D0008AE7A07F00F00300022809D05FF00000F7
:1054E00080F0010150460DF083FB040003D101E080
:1054F0000120F5E7FFDF022104F1850010F019FE1D
:105500000420287004F5B4706860B4F8850028821F
:10551000304810387C346C61C5E9028064E703E0F0
:1055200024E15BE02DE015E0A07F00F003000228FD
:1055300007D0002080F0010150460DF059FB18B94A
:1055400001E00120F6E7FFDF324621465046BDE884
:10555000F84FE8E504B9FFDF20782128A1D9307998
:10556000012803D1E07F40F00800E0773246214671
:105570005046FFF7D8FD2046BDE8F84F2321FDF740
:10558000C9BD3279AA8005F108030921504604F00B
:10559000D6FEE86010B10520287025E7A07F00F056
:1055A0000300022808D0002080F0010150460DF0D1
:1055B0001FFB040003D101E00120F5E7FFDF04F148
:1055C000620102231022081F0DF099F9077031794A
:1055D000417009E75002002040420F00A07F00F018
:1055E0000300022808D0002080F0010150460DF091
:1055F000FFFA050003D101E00120F5E7FFDF95F890
:10560000840000F0030001287AD1A07F00F0030796
:10561000E07F10F0010602D0022F04D133E095F8AC
:10562000A000C0072BD0D5F8601121B395F88320D6
:10563000087C62F387000874A17FCA09D5F860115D
:1056400062F341000874D5F8601166F30000087435
:10565000AEB1D5F86001102204F12401883508F0BC
:10566000B6FE287E40F001002876287820F0010060
:1056700005F8880900E016B1022F04D02DE095F856
:105680008800C00727D0D5F85C1121B395F8832096
:10569000087C62F387000874A17FCA09D5F85C1101
:1056A00062F341000874D5F85C1166F300000874D9
:1056B0008EB1D5F85C01102204F12401883508F080
:1056C00086FE287840F0010005F8180B287820F0B5
:1056D000010005F8A009022F44D0002000EB400093
:1056E00005EBC00090F88800800709D595F87C008C
:1056F000D5F86421400805F17D011032FDF773FEF5
:105700008DF8009095F884006A4600F003008DF84B
:10571000010095F888108DF8021095F8A0008DF81A
:1057200003002146504601F05FFA2078252805D075
:10573000212807D0FFDF2078222803D92221204604
:10574000FDF7E8FCA07F00F0030002280CD0002049
:1057500080F0010150460DF05DFA00283FF44FAE95
:10576000FFDF41E60120B9E70120F1E770684770EB
:105770003AE6FFDF38E670B5FE4C002584F85C5051
:1057800025660EF0FCFE04F11001204603F000FF38
:1057900084F8305070BD70B50D46FDF754FE04001E
:1057A00000D1FFDF4FF4B8720021284608F039FE1F
:1057B00004F124002861A07F00F00300022809D032
:1057C0005FF0010105F1E0000EF0DAFE002800D0E4
:1057D000FFDF70BD0221F5E70A46014602F1E00055
:1057E0000EF0EFBE70B50546406886B001780A2914
:1057F00006D00D2933D00E292FD0FFDF06B070BDA3
:1058000086883046FDF71FFE040000D1FFDF2078B8
:105810002128F3D028281BD1686802210E3001F01E
:10582000D8F9A8B168680821801D01F0D2F978B1D3
:1058300004F1240130460CF0BDF803F00FFD00B177
:10584000FFDF06B02046BDE870402921FDF762BCAD
:1058500006B0BDE8704003F0E2BE01210172686845
:10586000C6883046FDF7EFFD040000D1FFDFA07FC2
:1058700000F00301022902D120F01000A077207867
:1058800021280AD06868017A09B1007980B1A07F27
:1058900000F00300022862D0FFDFA07F00F00300C9
:1058A0000228ABD1FEF71AF80028A7D0FFDFA5E742
:1058B00003F0B5FEA17F08062BD5E07FC00705D019
:1058C00094F8200000F01F00102820D05FF00500A1
:1058D00084F82300207829281DD02428DDD13146E2
:1058E000042010F00DFF22212046FDF713FCA07FBD
:1058F00000F00300022830D05FF0000080F00101CA
:1059000030460DF087F90028C7D0FFDFC5E7062035
:10591000DEE70420DCE701F00300022808D00020C5
:1059200080F0010130460DF063F9050003D101E07C
:105930000120F5E7FFDF25212046FDF7EBFB0320E3
:105940008DF80000694605F1E0000EF031FE0228F6
:10595000A3D00028A1D0FFDF9FE70120CEE703F00E
:105960005EFE9AE72DE9F04387B0994616468846D1
:105970000746FDF768FD04004BD02078222848D365
:10598000232846D0E07F000743D4A07F00F0030027
:10599000022809D05FF0000080F0010138460DF0C8
:1059A00027F9050002D00CE00120F5E7A07F00F008
:1059B0000300022805D00121002238460DF00FF91E
:1059C00005466946284601F036F9009800B9FFDF20
:1059D00045B10098E03505612078222806D02428BA
:1059E00004D007E000990020086103E0252120464B
:1059F000FDF790FB0098012141704762868001A964
:105A0000C0E902890EF0EFFD022802D0002800D084
:105A1000FFDF07B0BDE8F08370B586B00546FDF73F
:105A200012FD017822291ED9807F00F00300022890
:105A300008D0002080F0010128460DF0D9F80400BC
:105A40002FD101E00120F5E7FFDF2AE0B4F85E0086
:105A500004F1620630440178427829B12146284693
:105A6000FFF711FCB0B9C9E6ADF8042009212846BA
:105A700002AB04F064FC03900028F4D005208DF8FC
:105A80000000694604F1E0000EF092FD022801D00A
:105A900000B1FFDF02231022314604F15E000CF05A
:105AA00064FFB4F860000028D0D1A7E610B586B036
:105AB0000446FDF7C8FC017822291BD9807F00F03D
:105AC0000300022808D0002080F0010120460DF0DC
:105AD0008FF8040003D101E00120F5E7FFDF062085
:105AE0008DF80000694604F1E0000EF061FD002829
:105AF00000D0FFDF06B010BD2DE9F05F05460C4673
:105B000000270078904601093E4604F1080BBA468A
:105B100002297DD0072902D00A2909D146E0686808
:105B200001780A2905D00D2930D00E292ED0FFDFAB
:105B3000BBE114271C26002C6BD08088A080FDF7C9
:105B400082FC5FEA000900D1FFDF99F817005A468E
:105B5000400809F11801FDF746FC6868C0892082F9
:105B6000696851F8060FC4F812004868C4F81600B6
:105B7000A07E01E03002002020F0060040F001008D
:105B8000A07699F81E0040F020014DE01A270A2661
:105B9000002CD1D0C088A080FDF755FC050000D1B5
:105BA000FFDF59462846FFF73FFB7EE10CB1A88B8B
:105BB000A080287A0B287DD006DC01287BD0022823
:105BC00008D0032804D135E00D2875D00E2874D0F4
:105BD000FFDF6AE11E270926002CADD0A088FDF763
:105BE00032FC5FEA000900D1FFDF287B00F00300F0
:105BF0000128207A1BD020F001002072297B89081F
:105C000061F341002072297BC90861F3820001E041
:105C100041E1F2E02072297B090961F3C30020729F
:105C200099F81E0040F0400189F81E103DE140F057
:105C30000100E2E713270D26002CAAD0A088FDF76B
:105C400002FC8146807F00F00300022808D000207B
:105C500080F00101A0880CF0CBFF050003D101E02A
:105C60000120F5E7FFDF99F81E0000F00302022A89
:105C700050D0686F817801F003010129217A4BD05F
:105C800021F00101217283789B0863F341012172A5
:105C90008378DB0863F38201217283781B0963F345
:105CA000C3012172037863F306112172437863F311
:105CB000C71103E061E0A9E090E0A1E0217284F85F
:105CC00009A0C178A172022A29D00279E17A62F38F
:105CD0000001E1720279520862F34101E172027936
:105CE000920862F38201E1720279D20862F3C30181
:105CF000E1724279217B62F30001217342795208FB
:105D000062F3410121734279920862F382012173A7
:105D1000407928E0A86FADE741F00101B2E7427990
:105D2000E17A62F30001E1724279520862F34101C3
:105D3000E1724279920862F38201E1724279D208FB
:105D400062F3C301E1720279217B62F300012173E6
:105D50000279520862F3410121730279920862F3D9
:105D6000820121730079C00860F3C301217399F89F
:105D70000000232831D9262140E018271026E4B35B
:105D8000A088FDF760FB8346807F00F003000228B7
:105D900009D0002080F00101A0880CF029FF5FEA03
:105DA000000903D101E00120F4E7FFDFE868A0600B
:105DB00099F8000040F0040189F8001099F80100FA
:105DC000800708D5012020739BF8000023286CD998
:105DD0002721584651E084F80CA066E015270F26CD
:105DE0005CB1A088FDF72FFB814606225946E86882
:105DF00008F076FB0120A073A0E041E048463CE0BB
:105E000016270926E4B3287B20724EE0287B192749
:105E10000E26ACB3C4F808A0A4F80CA0012807D043
:105E2000022805D0032805D0042803D0FFDF0DE0A9
:105E3000207207E0697B042801F00F0141F0800126
:105E400021721ED0607A20F003006072A088FDF7F6
:105E5000FAFA05460078212827D0232800D0FFDF52
:105E6000A87F00F00300022813D0002080F0010179
:105E7000A0880CF0CFFE22212846FDF74BF914E054
:105E800004E0607A20F00300401CDEE7A8F8006020
:105E900010E00120EAE70CB16888A080287A68B396
:105EA00001280AD002284FD0FFDFA8F800600CB10B
:105EB000278066800020BDE8F09F15270F26002C64
:105EC000E4D0A088FDF7BFFA807F00F0030002282D
:105ED00008D0002080F00101A0880CF089FE0500A8
:105EE00003D101E00120F5E7FFDFD5F81D00062210
:105EF000594608F0F5FA84F80EA0D6E717270926C8
:105F0000002CC3D0A088FDF79EFA8146807F00F068
:105F10000300022808D0002080F00101A0880CF0C6
:105F200067FE050003D101E00120F5E7FFDF687897
:105F3000800701D5022000E00120207299F80000BE
:105F40002328B2D9272159E719270E26002C9DD0E6
:105F5000A088FDF778FA5FEA000900D1FFDFC4F8F6
:105F600008A0A4F80CA084F808A0A07A40F00300D0
:105F7000A07299F81E10C90961F38200A07299F805
:105F80001F2099F81E1012EAD11F05D099F8201091
:105F900001F01F0110292BD020F00800A07299F801
:105FA0001F10607A61F3C3006072697A01F0030127
:105FB0000129A2D140F00400607299F81E0000F09F
:105FC00003000228E87A16D0217B60F300012173D8
:105FD000AA7A607B62F300006073EA7A520862F387
:105FE00041012173A97A490861F3410060735CE7BC
:105FF00040F00800D2E7617B60F300016173AA7A88
:10600000207B62F300002073EA7A520862F34101B8
:106010006173A97A490861F34100207345E710B51F
:10602000F74C30B10146102204F1200008F0CFF9FE
:10603000012084F8300010BD10B5044600F0EBFDDF
:10604000EF4920461022BDE81040203108F0BFB9CA
:1060500070B5EB4D06004FF0000413D0FBF7F9F8D4
:1060600008B110240CE00621304608F020FA411C4B
:1060700005D028665FF0010085F85C0000E0072489
:10608000204670BD0020F7E7007810F00F0204D022
:10609000012A05D0022A0CD110E0000909D10AE03A
:1060A0000009012807D0022805D0032803D00428BE
:1060B00001D0072070470870002070470620704705
:1060C00005282AD2DFE800F003070F171F00087821
:1060D00020F0FF001EE0087820F00F00401C20F0A8
:1060E000F000103016E0087820F00F00401C20F07F
:1060F000F00020300EE0087820F00F00401C20F067
:10610000F000303006E0087820F00F00401C20F04E
:10611000F0004030087000207047072070472DE9DC
:10612000F041804688B00D4600270846FBF7DEF8B0
:10613000A8B94046FDF787F9040003D0207822284B
:1061400015D104E043F2020008B0BDE8F08145B982
:10615000A07F410603D500F00300022801D01020E3
:10616000F2E7A07FC10601D4010702D50DB10820D6
:10617000EAE7E17F090701D50D20E5E700F003001C
:1061800002280DD165B12846FEF75EFF0700DBD17E
:10619000FBF728FB20B9E878800701D50620D3E774
:1061A000A07F00F00300022808D0002080F0010149
:1061B00040460CF01DFD060002D00FE00120F5E77F
:1061C000A07F00F0030002280ED0002080F0010123
:1061D000002240460CF003FD060007D0A07F00F02F
:1061E0000300022804D009E00120EFE70420ABE718
:1061F00025B12A4631462046FEF74AFF6946304619
:1062000000F019FD009800B9FFDF0099022006F1A7
:10621000E0024870C1F824804A6100220A81A27F0E
:1062200002F00302022A1CD001200871287800F035
:106230000102087E62F3010008762A78520862F3B0
:10624000820008762A78920862F3C30008762A78DA
:10625000D20862F30410087624212046FCF75AFF86
:1062600033E035B30871301D886130784009087714
:106270007078C0F340004877287800F00102887FEA
:1062800062F301008877A27FD20962F382008877E7
:10629000E27F62F3C3008877727862F30410887734
:1062A000A878C87701F1210228462031FEF711FFB6
:1062B00003E0032008710520087625212046FCF71D
:1062C00029FFA07F20F04000A07701A900980EF0E0
:1062D0008AF9022801D000B1FFDF384634E72DE902
:1062E000FF4F9346474A0D4699B09A4607CA0AABF4
:1062F000002783E807001998FDF7A5F8060006D0E7
:106300003078262806D008201DB0BDE8F08F43F273
:106310000200F9E7B07F00F00309B9F1020F11D0D4
:106320004DB95846FEF790FE0028EDD1B07F00F041
:106330000300022806D0BBF1000F11D0FBF752FA80
:1063400020B10DE0BBF1000F4FD109E006200CF0A9
:10635000F7FB28B19BF80300800701D50620D3E79F
:10636000B07F00F00300022808D0002080F0010177
:1063700019980CF03DFC040003D101E00120F5E781
:10638000FFDF852D27D007DCEDB1812D1DD0822DBB
:106390001DD0832D08D11CE0862D1ED0882D1ED047
:1063A000892D1ED08A2D1ED00F2020710F281CD0C1
:1063B00003F032F9D8B101208DF83C00201D109077
:1063C0002079B0B156E10020EFE70120EDE702208F
:1063D000EBE70320E9E70520E7E70620E5E70820EB
:1063E000E3E70920E1E70A20DFE707208CE7112037
:1063F0008AE7B9F1020F07D0A56F07D1A06F06E0B9
:1064000030020020FC550200656FF6E7606F8046A1
:106410002DD04FF0010001904FF0020000905A463D
:1064200021463046FEF734FE9BF8000000F00101E3
:10643000A87861F30100A870B17FC90961F38200F7
:10644000A870F17F61F3C300A870617861F3041054
:10645000A8702078400928706078C0F34000687008
:106460009BF80200E87000206871287103E00220A8
:10647000019001200090A87898F80210C0F3C000A5
:10648000C1F3C001084003902CD05046FAF7E1FE5A
:10649000C0BBDAF80C00FAF7DCFE98BBDAF81C0097
:1064A000FAF7D7FE70BBDAF80C00A060DAF81C002F
:1064B000E060607898F8012042EA500161F3410001
:1064C000607098F80210C0B200EA111161F3000088
:1064D000607000202077009906F11700022907D08C
:1064E000012106E0607898F8012002EA5001E5E712
:1064F000002104EB810148610199701C022902D03E
:10650000012101E028E0002104EB81014861A87825
:1065100000F00300012857D198F8020000F00300B2
:10652000012851D1B9F1020F04D02A1D691D584626
:10653000FEF7CFFD287998F8041008408DF8340054
:10654000697998F8052011408DF8381008433BD040
:106550005046FAF77EFE08B11020D5E60AF1100188
:106560008B46B9F1020F17D00846002104F18C03C5
:10657000CDE9000304F5AE7202920DAB2046039AFA
:10658000FEF7F0FD0028E8D1B9F1020F08D050461F
:1065900008D14FF0010107E050464FF00101E5E757
:1065A0005846F5E74FF0000104F1A403CDE90003DC
:1065B00004F5B072029281F001010EAB2046039AFD
:1065C000FEF7D0FD0028C8D16078800733D4A878C2
:1065D00098F80210C0F38000C1F3800108432AD06C
:1065E000297898F800000AAAB9F1020F06D032F80B
:1065F00011204300DA4002F003070AE032F81020CD
:106600004B00DA4012F0030705D0012F0AD0022F09
:106610000AD0032F06D0039A6AB1012906D00429B3
:1066200004D008E00227F6E70127F4E7012801D0AB
:10663000042800D10427B07F40F08000B077F17FBC
:10664000039860F30001F1776078800705D5032097
:10665000A071039870B9002029E00220022F18D001
:10666000012F18D0042F2AD00020A071B07F20F075
:106670008000B07725213046FCF74CFD0FA904F1CE
:10668000E0000DF095FF10B1022800D0FFDF0020E0
:106690003AE6A071DFE7A0710D22002104F120008D
:1066A00007F0BFFE207840F00200207001208DF836
:1066B0005C0017AA3146199800F096FADAE7012033
:1066C000A071D7E72DE9F04387B09046894604468C
:1066D0000025FCF7B8FE060006D03078272806D043
:1066E000082007B0BDE8F08343F20200F9E7B07F6D
:1066F00000F00300022809D05FF0000080F00101E3
:1067000020460CF075FA040003D101E00120F5E702
:10671000FFDFA7795FEA090005D0012821D0B9F190
:10672000020F26D110E0B8F1000F22D1012F05D0C1
:10673000022F05D0032F05D0FFDF2EE00C252CE023
:1067400001252AE0022528E04046FAF782FDB0B98B
:10675000032F0ED11022414604F11D0007F037FE31
:106760001BE0012F02D0022F03D104E0B8F1000F8B
:1067700013D00720B5E74046FAF76BFD08B11020AB
:10678000AFE71022002104F11D0007F04AFE0621A8
:10679000404607F08CFEC4F81D002078252140F00B
:1067A000020020703046FCF7B5FC2078C10713D0FA
:1067B00020F00100207002208DF8000004F11D007F
:1067C00002908DF804506946C3300DF0F1FE0228A6
:1067D00003D010B1FFDF00E02577002081E730B55E
:1067E00087B00D460446FCF72EFE98B1807F00F07E
:1067F0000300022811D0002080F0010120460CF097
:10680000F7F904000ED02846FAF723FD38B110201E
:1068100007B030BD43F20200FAE70120ECE7207830
:10682000400701D40820F3E7294604F13D00202267
:10683000054607F0CCFD207840F0100020700107DD
:106840000FD520F00800207007208DF80000694661
:1068500004F1E00001950DF0ABFE022801D000B17B
:10686000FFDF0020D4E770B50D460646FCF7EBFDD0
:1068700018B10178272921D102E043F2020070BD4E
:10688000807F00F00300022808D0002080F0010182
:1068900030460CF0ADF9040003D101E00120F5E72A
:1068A000FFDFA079022809D16078C00706D02A4608
:1068B00021463046FEF7E7FC10B10FE0082070BD1E
:1068C000B4F860000E280BD204F1620102231022FA
:1068D000081F0CF014F8012101704570002070BDF4
:1068E000112070BD70B5064614460D460846FAF7ED
:1068F000B0FC18B92046FAF7D2FC08B1102070BDE0
:10690000A6F57F40FF380ED03046FCF79CFD38B12D
:10691000417822464B08811C1846FCF764FD07E0CD
:1069200043F2020070BD2046FDF78FFD0028F9D12B
:106930001021E01D0FF0FDFBE21D294604F11700B8
:1069400000F089F9002070BD2DE9F04104468AB0BD
:106950001546884600270846FAF7C8FC18B92846A5
:10696000FAF7C4FC18B110200AB0BDE8F081204647
:10697000FCF769FD060003D0307827281BD102E020
:1069800043F20200F0E7B07F00F00300022809D0D4
:106990005FF0000080F0010120460CF029F90400AE
:1069A00003D101E00120F5E7FFDF2078400702D5A1
:1069B0006078800701D40820D6E7B07F00F003009C
:1069C000022803D0A06F03D1A16F02E0606FFAE745
:1069D000616F407800B19DB1487810B1B8F1000FF7
:1069E0000ED0ADB1EA1D06A8E16800F034F910221E
:1069F00006A905F1170007F0BDFC18B1042707E050
:106A00000720B1E71022E91D04F12D0007F0DFFC9B
:106A1000B8F1000F06D0102208F1070104F11D00A3
:106A200007F0D5FC2078252140F002002070304688
:106A3000FCF770FB2078C10715D020F00100207012
:106A400002208DF8000004F11D0002901030039028
:106A50008DF804706946B3300DF0AAFD022803D00A
:106A600010B1FFDF00E0277700207DE7F8B515467D
:106A70000E460746FCF7E7FC040004D020782228E5
:106A800004D00820F8BD43F20200F8BDA07F00F05A
:106A90000300022802D043F20500F8BD3046FAF7A1
:106AA000D8FB18B92846FAF7D4FB08B11020F8BD76
:106AB00000953288B31C21463846FEF707FC1128A2
:106AC00015D00028F3D1297C4A08A17F62F3C711B1
:106AD000A177297CE27F61F30002E277297C8908B3
:106AE00084F82010A17F21F04001A177F8BDA17F9B
:106AF0000907FBD4D6F80200C4F83600D6F8060021
:106B0000C4F83A003088A0861022294604F12400F7
:106B100007F05DFC287C4108E07F61F34100E077ED
:106B2000297C61F38200E077287C800884F82100CA
:106B3000A07F40F00800A0770020D3E770B50D4695
:106B400006460BB1072070BDFCF77DFC040007D0A2
:106B50002078222802D3A07F800604D4082070BDAC
:106B600043F2020070BDADB1294630460AF022FF63
:106B700002F074FB297C4A08A17F62F3C711A17758
:106B8000297CE27F61F30002E277297C890884F89E
:106B9000201004E030460AF030FF02F05FFBA17FD6
:106BA00021F02001A17770BD70B50D46FCF74BFCBC
:106BB000040005D02846FAF772FB20B1102070BD02
:106BC00043F2020070BD29462046FEF72DFB00204F
:106BD00070BD04E010F8012B0AB100207047491E77
:106BE00089B2F7D20120704770B51546064602F00B
:106BF00013FD040000D1FFDF207820F00F00801C7F
:106C000020F0F0002030207066802868A060BDE889
:106C1000704002F004BD10B5134C94F83000002809
:106C200008D104F12001A1F110000DF003FD0120B5
:106C300084F8300010BD10B190F8B9202AB10A488C
:106C400090F8350018B1002003E0B83001E00648A4
:106C500034300860704708B50023009313460A4695
:106C60000CF0C5F908BD00003002002018B1817891
:106C7000012938D101E010207047018842F6011245
:106C8000881A914231D018DC42F60102A1EB0200D1
:106C900091422AD00CDC41B3B1F5C05F25D06FF42E
:106CA000C050081821D0A0F57060FF381BD11CE03F
:106CB00001281AD002280AD117E0B0F5807F14D03D
:106CC00008DC012811D002280FD003280DD0FF289E
:106CD00009D10AE0B0F5817F07D0A0F580700338B4
:106CE00003D0012801D0002070470F2070470A28E8
:106CF0001FD008DC0A2818D2DFE800F0191B1F1F7C
:106D0000171F231D1F21102815D008DC0B2812D0B7
:106D10000C2810D00D2816D00F2806D10DE0112810
:106D20000BD084280BD087280FD003207047002079
:106D3000704705207047072070470F2070470420D8
:106D40007047062070470C20704743F202007047DE
:106D500038B50C46050041D06946FFF795F9002883
:106D600019D19DF80010607861F3020060706946E7
:106D7000681CFFF789F900280DD19DF80010607894
:106D800061F3C5006070A978C1F34101012903D006
:106D9000022905D0072038BD217821F0200102E02A
:106DA000217841F020012170410704D0A978C90859
:106DB00061F386106070607810F0380F07D0A97802
:106DC000090961F3C710607010F0380F02D16078C4
:106DD000400603D5207840F040002070002038BDE8
:106DE00070B504460020088015466068FFF7B0FFC4
:106DF000002816D12089A189884211D8606880783E
:106E0000C0070AD0B1F5007F0AD840F20120B1FBDB
:106E1000F0F200FB1210288007E0B1F5FF7F01D9E6
:106E20000C2070BD01F201212980002070BD10B539
:106E30000478137864F3000313700478640864F32F
:106E4000410313700478A40864F382031370047878
:106E5000E40864F3C30313700478240964F304138F
:106E600013700478640964F3451313700078800983
:106E700060F38613137031B10878C10701D1800720
:106E800001D5012000E0002060F3C713137010BD8E
:106E90004278530702D002F0070306E012F0380FE1
:106EA00002D0C2F3C20300E001234A7863F3020276
:106EB0004A70407810F0380F02D0C0F3C20005E0ED
:106EC000430702D000F0070000E0012060F3C50294
:106ED0004A7070472DE9F04F95B00D00824613D0EF
:106EE00012220021284607F09CFA4FF6FF7B05AAE4
:106EF0000121584607F05DF80024264637464FF436
:106F000020586FF4205972E0102015B0BDE8F08FC2
:106F10009DF81E0001280AD1BDF81C1041450BD078
:106F200011EB09000AD001280CD002280CD0042C47
:106F30000ED0052C0FD10DE0012400E00224BDF895
:106F40001A6008E0032406E00424BDF81A7002E089
:106F5000052400E00624BDF81A10514547D12C74D1
:106F6000BEB34FF0000810AA4FF0070ACDE9028225
:106F7000CDE900A80DF13C091023CDF81090424650
:106F80003146584607F0E5F808BBBDF83C002A46F4
:106F9000C0B210A90DF0D9FBC8B9AE81CFB1CDE90F
:106FA00000A80DF1080C0AAE40468CE841021323FC
:106FB00000223946584607F0CCF840B9BDF83C00ED
:106FC000F11CC01EC0B22A1D0DF0BFFB10B1032082
:106FD0009BE70AE0BDF82900E881062C05D19DF861
:106FE0001E00A872BDF81C00288100208DE705A8AE
:106FF00006F0EBFF00288BD0FFF779FE85E72DE93F
:10700000F0471C46DDE90978DDF8209015460E00B2
:10701000824600D1FFDF0CB1208818B1D5B1112014
:10702000BDE8F087022D01D0012100E0002106F12A
:10703000140005F087FEA8F8000002463B462946EA
:10704000504603F07CF9C9F8000008B9A41C3C6064
:107050000020E5E71320E3E7F0B41446DDE904522D
:107060008DB1002314B1022C09D101E0012306E007
:107070000D7CEE0703D025F0010501230D74214698
:10708000F0BC04F03ABA1A80F0BC70472DE9FE4F0C
:1070900091461A881C468A468046FAB102AB494698
:1070A00003F04DF9050019D04046A61C27880BF0C7
:1070B000E4FE3246072629463B4600960BF0F1FADD
:1070C00020882346CDE900504A4651464046FFF706
:1070D000C3FF002020800120BDE8FE8F0020FBE7D9
:1070E0002DE9F04786B082460EA8904690E8B000A1
:1070F000894604AA05A903A88DE807001E462A466A
:1071000021465046FFF77BFF039901B101213970F9
:10711000002818D1FA4904F1140204AB086003985E
:1071200005998DE8070042464946504606F0BDF9EC
:10713000A8B1092811D2DFE800F005080510100AEF
:107140000C0C0E00002006B06AE71120FBE70720B8
:10715000F9E70820F7E70D20F5E70320F3E7BDF88E
:1071600010100398CDE9000133462A4621465046C7
:10717000FFF772FFE6E72DE9F04389B01646DDE937
:1071800010870D4681461C461422002103A807F0F3
:1071900048F9012002218DF810108DF80C008DF8AF
:1071A0001170ADF8146064B1A278D20709D08DF8DF
:1071B0001600E088ADF81A00A088ADF81800A068A5
:1071C000079008A80095CDE90110424603A948465A
:1071D0006B68FFF785FF09B0BDE8F083F0B58BB0B1
:1071E00000240646069407940727089405A80994E6
:1071F000019400970294CDE903400D4610232246E6
:10720000304606F0A6FF78B90AA806A901940097AF
:107210000294CDE90310BDF814300022294630460F
:1072200006F035FD002801D0FFF761FD0BB0F0BD81
:1072300006F0C6BB2DE9FC410C468046002602F054
:10724000EBF9054620780D287ED2DFE800F0BC0778
:1072500013B325BD49496383AF959B00A8480068D7
:1072600020B1417841F010014170ADE0404602F09C
:1072700003FAA9E0042140460BF0BAFC070000D154
:10728000FFDF07F11401404605F0F1FCA5BB132117
:107290004046FDF7C1FB97E0042140460BF0A8FCF7
:1072A000070000D1FFDFE088ADF800000020B881C2
:1072B0009DF80000010704D5C00602D5A088B8815A
:1072C00005E09DF8010040067ED5A088F88105B94B
:1072D000FFDF22462946404601F0C0FC022673E04B
:1072E000E188ADF800109DF8011009060FD50728B8
:1072F00003D006280AD00AE024E0042140460BF01F
:1073000077FC060000D1FFDFA088F0810226CDB90E
:10731000FFDF17E0042140460BF06AFC070000D1B4
:10732000FFDF07F1140006F082FB90F0010F02D19D
:10733000E079000648D5387C022640F00200387417
:1073400005B9FFDF224600E03DE02946404601F056
:1073500085FC39E0042140460BF04AFC017C002DFD
:1073600001F00206C1F340016171017C21F00201CC
:107370000174E7D1FFDFE5E702260121404602F074
:10738000ADF921E0042140460BF032FC054660686F
:1073900000902089ADF8040001226946404602F0C1
:1073A000BEF9287C20F0020028740DE0002DC9D120
:1073B000FFDFC7E7022600214046FBF789F8002DD2
:1073C000C0D1FFDFBEE7FFDF3046BDE8FC813EB540
:1073D0000C0009D001466B4601AA002006F03EFFD2
:1073E00020B1FFF784FC3EBD10203EBD0020208070
:1073F000A0709DF8050002A900F00700FEF760FEEE
:1074000050B99DF8080020709DF8050002A9C0F34E
:10741000C200FEF755FE08B103203EBD9DF80800EE
:1074200060709DF80500C109A07861F30410A07098
:107430009DF80510890961F3C300A0709DF8041040
:10744000890601D5022100E0012161F342009DF887
:10745000001061F30000A07000203EBD70B514461E
:1074600006460D4651EA040005D075B10846F9F705
:1074700034FF78B901E0072070BD2946304606F098
:1074800054FF10B1BDE8704031E454B12046F9F723
:1074900024FF08B1102070BD21463046BDE8704081
:1074A00095E7002070BD2DE9FC5F0C46904605462F
:1074B000002701780822007A3E46B2EB111F7DD1E9
:1074C00004F10A0100910A31821E4FF0020A04F110
:1074D000080B0191092A72D2DFE802F0EDE005F510
:1074E00028287BAACE00688804210BF081FB0600C7
:1074F00000D1FFDFB08928B152270726C3E0000082
:107500009402002051271026002C7DD06888A0808E
:107510000120A071A88900220099FFF79FFF002891
:1075200073D1A8892081288AE081D1E0B5F8129032
:10753000072824D1E87B000621D5512709F1140042
:1075400086B2002CE1D0A88900220099FFF786FFBF
:1075500000285AD16888A08084F806A0A8892081D4
:107560000120A073288A2082A4F81290A88A009093
:1075700068884B46A969019A01F04CFBA8E05027A6
:1075800009F1120086B2002C3ED0A889002259468B
:10759000FFF764FF002838D16888A080A889E080C0
:1075A000287A072813D002202073288AE081E87BFC
:1075B000C0096073A4F81090A88A01E085E082E019
:1075C000009068884B4604F11202A969D4E70120B3
:1075D000EAE7B5F81290512709F1140086B2002CA1
:1075E00066D0688804210BF003FB83466888A0807E
:1075F000A88900220099FFF731FF00286ED184F896
:1076000006A0A889208101E052E067E00420A07371
:10761000288A2082A4F81290A88A009068884B4695
:10762000A969019A01F0F6FAA989ABF80E104FE0AA
:107630006888FBF708FF0746688804210BF0D8FA32
:10764000064607B9FFDF06B9FFDF687BC00702D037
:107650005127142601E0502712264CB36888A080D9
:10766000502F06D084F806A0287B594601F0E2FA94
:107670002EE0287BA11DF9E7FE49A88949898142AE
:1076800005D1542706269CB16888A08020E05327A6
:107690000BE06888A080A889E08019E06888042150
:1076A0000BF0A6FA00B9FFDF55270826002CF0D111
:1076B000A8F8006011E056270726002CF8D068884B
:1076C000A080002013E0FFDF02E0012808D0FFDFE8
:1076D000A8F800600CB1278066800020BDE8FC9F00
:1076E00057270726002CE3D06888A080687AA0710D
:1076F000EEE7401D20F0030009B14143091D01EBF5
:107700004000704713B5DB4A00201071009848B163
:10771000002468460BF089F8002C02D1D64A009963
:1077200011601CBD01240020F4E770B50D4614461D
:10773000064686B05C220021284606F072FE04B997
:10774000FFDFA0786874A2782188284601F09DFAAE
:107750000020A881E881228805F11401304605F057
:107760006AFA6A460121304606F023FC1AE000BF9F
:107770009DF80300000715D5BDF806103046FFF749
:107780002DFD9DF80300BDF8061040F010008DF8A7
:107790000300BDF80300ADF81400FF233046059A3E
:1077A00006F08BFD684606F010FC0028E0D006B01D
:1077B00070BD10B50C4601F1140005F074FA0146D5
:1077C000627C2046BDE8104001F094BA30B5044612
:1077D000A84891B04FF6FF75C18905AA284606F062
:1077E000E8FB30E09DF81E00A0422AD001282AD1F3
:1077F000BDF81C00B0F5205F03D042F601018842BD
:1078000021D1002002AB0AAA0CA9019083E807004D
:1078100007200090BDF81A1010230022284606F019
:1078200098FC38B9BDF828000BAAC0B20CA90CF01E
:107830008CFF10B1032011B030BD9DF82E00A04286
:1078400001D10020F7E705A806F0BFFB0028C9D04A
:107850000520F0E770B5054604210BF0C9F90400D6
:1078600000D1FFDF04F114010C46284605F0FFF9B2
:1078700021462846BDE8704005F000BA70B58AB0D0
:107880000C460646FBF7DFFD050014D028782228B9
:1078900027D30CB1A08890B101208DF80C000320F3
:1078A0008DF8100000208DF8110054B1A088ADF8BB
:1078B0001800206807E043F202000AB070BD0920FA
:1078C000FBE7ADF818000590042130460BF090F965
:1078D000040000D1FFDF04F1140005F0FAF90007FD
:1078E00001D40820E9E701F097FE60B108A8022161
:1078F0000094CDE9011095F8232003A93046636870
:10790000FFF7EEFBD9E71120D7E72DE9F04FB2F8EA
:1079100002A0834689B0154689465046FBF793FD81
:107920000746042150460BF063F9002604460596ED
:107930004FF002080696ADF81C6007B9FFDF04B9E6
:10794000FFDF4146504603F03FFF50B907AA06A9A2
:1079500005A88DE807004246214650466368FFF7B8
:107960004EFB444807AB0660DDE9051204F1140044
:10797000CDF80090CDE90320CDE9013197F823201F
:10798000594650466B6805F0EDF906000AD0022E04
:1079900004D0032E14D0042E00D0FFDF09B03046EF
:1079A000BDE8F08FBDF81C000028F7D00599CDE99F
:1079B00000104246214650466368FFF74DFBEDE755
:1079C000687840F008006870E8E72DE9F04F99B05A
:1079D00004464FF000082748ADF81C80ADF8208021
:1079E000ADF82480A0F80880ADF81480ADF81880B8
:1079F000ADF82C80ADF82880007916460D46474634
:107A0000012808D0022806D0032804D0042802D078
:107A1000082019B0C4E72046F9F71BFC70BB2846C4
:107A2000F9F717FC50BB6068F9F760FC30BB606881
:107A300048B160892189884202D8B1F5007F01D917
:107A40000C20E6E780460EAA06A92846FFF7C8F9EB
:107A50000028DED168688078C0F34100022808D190
:107A60009DF8190010F0380F03D02869F9F735FC9C
:107A700020B904E0940200201800002022E005A9AB
:107A80002069FFF765F90028C3D1206948B1607803
:107A900080079DF8150000F0380001D5F0B300E034
:107AA000E0BB9DF8140080060ED59DF8150010F07F
:107AB000380F03D06068F9F710FC18B96068F9F75F
:107AC00015FC08B11020A4E70AA96069FFF740F986
:107AD00000289ED1606940B19DF8290000F007019F
:107AE00001293CD110F0380F39D00BA9A069FFF75C
:107AF0002FF900288DD19DF8280080062FD49DF8FD
:107B00002C0080062BD4A06950B19DF82D0000F008
:107B10000701012923D110F0380F00E01FE01ED02B
:107B2000E06818B10078D0B11C2818D20FAA611CE7
:107B30002046FFF77CF90121384661F30F20824689
:107B40008DF85210B94642F603000F46ADF85000CA
:107B50000DF13F0218A928680CF0F9FD08B10720C3
:107B600057E79DF8600015A9CDF80090C01CCDE93D
:107B7000019100F0FF0B00230BF20122514614A8E3
:107B800006F042F9F0BBBDF854000C90FE482A897B
:107B900029690092CDE901106B89BDF83820286869
:107BA000069906F031F901007ED120784FF0020AE3
:107BB000C10601D480062BD5CDF80C90606950B970
:107BC0000AA906A8FFF764F99DF8290020F007002C
:107BD000401C8DF829009DF8280008A940F0C80035
:107BE0008DF828008DF8527042F60210ADF8500062
:107BF00003AACDF800A0CDE90121002340F2032221
:107C000014A800E01EE00A9906F0FEF801004BD12E
:107C1000DD484D4608385B460089ADF83D000FA8A9
:107C2000CDE90290CDF80490CDF810904FF00709FF
:107C30000022CDF80090BDF854104FF6FF7006F00A
:107C400026F810B1FFF753F8E3E69DF83C00000674
:107C500024D52946012060F30F218DF852704FF48E
:107C600024500395ADF8500062789DF80C00002375
:107C700062F300008DF80C006278CDF800A0520885
:107C800062F341008DF80C0003AACDE9012540F212
:107C9000032214A806F0B8F8010005D1606888B383
:107CA0002069A8B905A900E084E006A8FFF7F0F86C
:107CB0006078800706D49DF8150020F038008DF814
:107CC000150005E09DF8140040F040008DF8140008
:107CD0008DF8527042F60110ADF85000208940F244
:107CE0000121B0FBF1F201FB1202606809ABCDF893
:107CF0000080CDE90103002314A8059906F084F85B
:107D0000010057D12078C00728D00395A06950B949
:107D10000BA906A8FFF7BCF89DF82D0020F007007E
:107D2000401C8DF82D009DF82C008DF8527040F00D
:107D300040008DF82C0042F60310ADF8500007A962
:107D400003AACDF800A0CDE90121002340F20322CF
:107D500014A80B9906F058F801002BD1E06868B31D
:107D60002946012060F30F218DF8527042F604106D
:107D7000ADF85000E068002302788DF85820407874
:107D80008DF85900E06816AA4088ADF85A00E068FE
:107D900000798DF85C00E068C088ADF85D00CDF832
:107DA0000090CDE901254FF4027214A806F02CF8DA
:107DB000010003D00C9800F0C9FF2AE672480321A5
:107DC0000838017156B100893080BDF824007080F8
:107DD000BDF82000B080BDF81C00F080002018E63F
:107DE00070B501258AB016460B46012802D002283C
:107DF00016D104E08DF80E504FF4205003E08DF8BA
:107E00000E5042F60100ADF80C005BB10024601C7E
:107E100060F30F2404AA08A918460CF098FC18B1C6
:107E200007204AE5102048E504A99DF8202056487F
:107E3000CDE90021801E02900023214603A802F212
:107E4000012205F0E1FF10B1FEF751FF35E54E4884
:107E500008380EB1C1883180057100202DE5F0B5DC
:107E600093B0074601268DF83E6041F60100ADF85B
:107E70003C0012AA0FA93046FFF7B2FF002849D1F3
:107E8000414C0025083CEFB31C22002102A806F05B
:107E9000C8FA9DF808008DF83E6040F020008DF88B
:107EA000080042F60520ADF83C000E959DF83A001A
:107EB000119520F00600801C8DF83A009DF83800DE
:107EC0006A4620F0FF008DF838009DF8390009A9B6
:107ED00020F0FF008DF839000420ADF82C00ADF83B
:107EE00030000EA80A9011A80D900FA80990ADF8C7
:107EF0002E5002A8FFF769FD00280BD1BDF8000045
:107F0000608100E008E0BDF80400A081401CE08131
:107F10002571002013B0F0BD6581A581BDF8480032
:107F2000F4E72DE9F74F1849A0B000240839179459
:107F30000A79A146012A04D0022A02D0082023B0DF
:107F40002EE5CA88824201D00620F8E721988A46A9
:107F5000824201D10720F2E70120214660F30F2180
:107F6000ADF848004FF6FF780691ADF84A808DF8DD
:107F70006E0042F6020B8DF872401CA9ADF86CB091
:107F8000ADF87040139101E09C020020ADF85080E4
:107F900012A806F049F800252E462F460DAB072201
:107FA00012A9404606F043F878B10A285DD195B38E
:107FB0008EB3ADF86450ADF866609DF85E008DF844
:107FC000144019AC012864D06BE09DF83A001FB34F
:107FD000012859D1BDF8381059451FD118A809A951
:107FE00001940294CDE9031007200090BDF83610EB
:107FF00010230022404606F0ACF8B0BBBDF860008C
:10800000042801D006284AD1BDF8241021988142C5
:108010003AD10F2093E73AE0012835D1BDF8380076
:10802000B0F5205F03D042F6010188422CD1BAF8A6
:108030000600BDF83610884201D1012700E0002774
:1080400005B19EB1219881421ED118A809AA0194B8
:108050000294CDE90320072000900D461023002252
:10806000404606F076F800B902E02DE04E460BE0FF
:10807000BDF86000022801D0102810D1C0B217AAA4
:1080800009A90CF062FB50B9BDF8369086E70520CF
:1080900055E705A917A8221D0CF059FB08B10320CC
:1080A0004DE79DF814000023001DC2B28DF8142086
:1080B00022980092CDE901401BA8069905F0A4FE84
:1080C00010B902228AF80420FEF711FE37E710B536
:1080D0000B46401E88B084B205AA00211846FEF760
:1080E000A6FE00200DF1080C06AA05A901908CE857
:1080F0000700072000900123002221464FF6FF7061
:1081000005F0C5FD0446BDF81800012800D0FFDFCA
:108110002046FEF7ECFD08B010BDF0B5F74F044661
:1081200087B038790E46032804D0042802D00820EE
:1081300007B0F0BD04AA03A92046FEF751FE0500D2
:10814000F6D160688078C0F3410002280AD19DF81A
:108150000D0010F0380F05D02069F9F7BEF808B10E
:108160001020E5E7208905AA21698DE807006389C9
:10817000BDF810202068039905F046FE10B1FEF707
:10818000B6FDD5E716B1BDF8140030800420387173
:108190002846CDE7F8B50C0006460CD001464FF650
:1081A000FF7500236A46284606F058F828B100BF3C
:1081B000FEF79DFDF8BD1020F8BD69462046FEF78C
:1081C000C7FD0028F8D1A078314600F00103284609
:1081D000009A06F072F8EBE730B587B0144600223B
:1081E0000DF1080C05AD01928CE82C0007220092DD
:1081F0000A46014623884FF6FF7005F048FDBDF89A
:1082000014102180FEF773FD07B030BD70B50D4628
:1082100004210AF0EDFC040000D1FFDF294604F13F
:108220001400BDE8704004F04DBD70B50D4604214A
:108230000AF0DEFC040000D1FFDF294604F114003F
:10824000BDE8704004F061BD70B50D4604210AF030
:10825000CFFC040000D1FFDF294604F11400BDE883
:10826000704004F079BD70B5054604210AF0C0FCE9
:10827000040000D1FFDF214628462368BDE8704096
:108280000122FEF703BF70B5064604210AF0B0FCD8
:10829000040000D1FFDF04F1140004F004FD401DD0
:1082A00020F0030511E0011D00880022431821463B
:1082B0003046FEF7EBFE00280BD0607CABB2684383
:1082C00082B2A068011D0AF050FBA0684188002915
:1082D000E9D170BD70B5054604210AF089FC04009F
:1082E00000D1FFDF214628466368BDE870400222C6
:1082F000FEF7CCBE70B50E46054601F08DF90400C0
:1083000000D1FFDF0120207266726580207820F0A6
:108310000F00001D20F0F00040302070BDE87040DC
:1083200001F07DB910B50446012900D0FFDF2046D9
:10833000BDE810400121FAF7CBB82DE9F04F97B016
:108340004FF0000A0C008346ADF814A0D04619D0B7
:10835000E06830B1A068A8B10188ADF81410A0F8A9
:1083600000A05846FBF76FF8070043F2020961D0FE
:10837000387822285CD3042158460AF039FC0500DD
:1083800005D103E0102017B0BDE8F08FFFDF05F145
:10839000140004F088FC401D20F00306A07801289A
:1083A00003D0022801D00720EDE7218807AA58460C
:1083B00005F0FFFD30BB07A805F007FE10BB07A8BE
:1083C00005F003FE48B99DF82600012805D1BDF847
:1083D0002400A0F52451023902D04FF45050D2E7C6
:1083E000E068B0B1CDE902A00720009005AACDF861
:1083F00004A00492A2882188BDF81430584605F0E4
:1084000046FC10B1FEF773FCBDE7A168BDF814008F
:1084100008809DF81F00C00602D543F20140B2E774
:108420000B9838B1A1780078012905D080071AD4BB
:108430000820A8E74846A6E7C007F9D002208DF833
:108440003C00A8684FF00009A0B1697C42887143E4
:1084500091420FD98AB2B3B2011D0AF03CFA8046AC
:10846000A0F800A006E003208DF83C00D5F80080BD
:108470004FF001099DF8200010F0380F00D1FFDF08
:108480009DF820001E49C0F3C200084497F823104D
:1084900010F8010C884201D90F2074E72088ADF84C
:1084A000400014A90095CDE90191434607220FA988
:1084B0005846FEF715FE002891D19DF8500050B99E
:1084C000A078012807D1687CB3B2704382B2A86853
:1084D000011D0AF014FA002055E770B5064615464E
:1084E0000C460846FEF7C2FB002805D12A46214665
:1084F0003046BDE8704073E470BD12E59402002080
:108500000656020070B51E4614460D0009D044B14F
:10851000616831B138B1FC49C988814203D0072074
:1085200070BD102070BD2068FEF7A0FB0028F9D1B7
:10853000324621462846BDE87040FFF746BA70B57E
:1085400015460C0006D038B1EF490989814203D0A5
:10855000072070BD102070BD2068FEF787FB002843
:10856000F9D129462046BDE87040D6E570B50646EB
:1085700086B00D4614461046F8F791FED0BB6068F1
:10858000F8F7B4FEB0BBA6F57F40FF3803D0304605
:10859000FAF759FF80B128466946FEF79BFC002890
:1085A0000CD19DF810100F2008293DD2DFE801F012
:1085B00008060606060A0A0843F2020006B070BD65
:1085C0000320FBE79DF80210012908D1BDF8001037
:1085D000B1F5C05FF2D06FF4C052D142EED09DF839
:1085E000061001290DD1BDF80410A1F52851062966
:1085F00007D200E029E0DFE801F0030304030303EE
:10860000DCE79DF80A1001290FD1BDF80810B1F57B
:10861000245FD3D0A1F60211B1F50051CED00129CB
:10862000CCD0022901D1C9E7FFDF606878B9002307
:1086300005AA2946304605F011FE10B1FEF757FB9A
:10864000BCE79DF81400800601D41020B6E76188CD
:10865000224628466368FFF7BFFDAFE72DE9F043E8
:10866000814687B0884614461046F8F718FE18B1C0
:10867000102007B0BDE8F083002306AA4146484613
:1086800005F0ECFD18B100BFFEF731FBF1E79DF8F6
:108690001800C00602D543F20140EAE7002507278B
:1086A00005A8019500970295CDE9035062884FF621
:1086B000FF734146484605F04CFD060013D1606843
:1086C000F8F7EDFD60B960680195CDE902500097BB
:1086D0000495238862884146484605F03AFD0646DF
:1086E000BDF8140020803046CEE739B1864B0A88A9
:1086F0009B899A4202D843F2030070471DE610B5E9
:1087000086B0814C0423ADF81430638943B1A48949
:108710008C4201D2914205D943F2030006B010BD4C
:108720000620FBE7ADF81010002100910191ADF893
:10873000003002218DF8021005A9029104A90391CD
:10874000ADF812206946FFF7F8FDE7E72DE9FC4791
:1087500081460D460846F8F77CFD88BB4846FAF787
:1087600072FE5FEA00080AD098F80000222829D398
:10877000042148460AF03CFA070005D103E043F221
:108780000200BDE8FC87FFDF07F1140004F0A1FA46
:1087900006462878012803D0022804D00720F0E7F5
:1087A000B0070FD502E016F01C0F0BD0A8792C1DD6
:1087B000C00709D0E08838B1A068F8F74AFD18B1C1
:1087C0001020DEE70820DCE721882A780720B1F5B1
:1087D000847F35D01EDC40F20315A1F20313A942B9
:1087E00026D00EDCB1F5807FCBD003DCF9B10129B6
:1087F00026D1C6E7A1F58073013BC2D0012B1FD162
:1088000013E0012BBDD0022B1AD0032BB9D0042BBF
:1088100016D112E0A1F20912082A11D2DFE802F003
:108820000B04041010101004ABE7022AA9D007E0D3
:10883000012AA6D004E0320700E0F206002AA0DAFE
:10884000CDB200F0E9FE50B198F82300CDE9000563
:10885000FA89234639464846FEF78DFC91E71120F8
:108860008FE72DE9F04F8BB01F4615460C46834627
:108870000026FAF7E8FD28B10078222805D2082062
:108880000BB081E543F20200FAE7B80801D00720F7
:10889000F6E7032F00D100274FF6FF79CCB1022D68
:1088A00073D32046F8F722FD30B904EB0508A8F190
:1088B0000100F8F71BFD08B11020E1E7AD1E38F804
:1088C000028CAAB22146484605F01CFE40455CD108
:1088D000ADB20D49B80702D58889401C00E00120DF
:1088E0001FFA80F8F80701D08F8900E04F4605AAEB
:1088F0004146584605F05DFB4FF0070A4FF000096E
:10890000DCB320460BE000009402002040881028D1
:108910003BD8361D304486B2AE4236D2A01902880A
:108920004245F3D351E000BF9DF8170002074CD534
:1089300094B304EB0608361DB8F80230B6B2102B1B
:1089400023D89A19AA4220D8B8F8002091421CD105
:10895000C0061CD5CDE900A90DF1080C0AAAA11981
:1089600048468CE80700B8F800100022584605F089
:108970008EF920B1FEF7BBF982E726E005E0B8F8F2
:108980000200BDF82810884201D00B2078E7B8F823
:108990000200304486B207E0FFE7C00604D558461F
:1089A000FEF71CFC002888D19DF81700BDF81A10AE
:1089B00020F010008DF81700BDF81700ADF800008A
:1089C000FF235846009A05F078FC05A805F0FDFA4B
:1089D00018B9BDF81A10B942A6D9042158460AF0B0
:1089E00007F9040000D1FFDFA2895AB1CDE900A93F
:1089F0004D46002321465846FEF7BDFB0028BBD15B
:108A0000A5813DE700203BE72DE9FF4F8BB01E46D7
:108A100017000D464FF0000412D0B00802D0072016
:108A20000FB0B1E4032E00D100265DB10846F8F77F
:108A300054FC28B93888691E0844F8F74EFC08B180
:108A40001020EDE7C74AB00701D5D18900E0012128
:108A5000F0074FF6FF7802D0D089401E00E0404674
:108A600086B206AA0B9805F0A4FA4FF000094FF061
:108A7000070B0DF1140A38E09DF81B00000734D5F0
:108A8000CDF80490CDF800B0CDF80890CDE9039A68
:108A9000434600220B9805F05CFB60BB05B3BDF8B4
:108AA00014103A8821442819091D8A4230D3BDF890
:108AB0001E2020F8022BBDF8142020F8022BCDE94F
:108AC00000B9CDE90290CDF810A0BDF81E10BDF898
:108AD000143000220B9805F03CFB08B103209FE7FF
:108AE000BDF814002044001D84B206A805F06DFAFC
:108AF00020B10A2806D0FEF7FAF891E7BDF81E105B
:108B0000B142B9D934B17DB13888A11C884203D2B1
:108B10000C2085E7052083E722462946404605F0DC
:108B2000F1FC014628190180A41C3C80002077E755
:108B300010B50446F8F7B3FB08B1102010BD894802
:108B4000C0892080002010BDF0B58BB00D460646D0
:108B50001422002103A805F064FC01208DF80C000C
:108B60008DF8100000208DF81100ADF8145030463B
:108B7000FAF769FC48B10078222812D30421304664
:108B80000AF036F8040005D103E043F202000BB00E
:108B9000F0BDFFDF04F11400074604F09AF88006E8
:108BA00001D40820F3E7207C022140F0010020746A
:108BB00009A80094CDE90110072203A93046636893
:108BC000FEF78EFA20B1217C21F001012174DEE74D
:108BD00029463046F9F76DFC08A9384604F068F8D4
:108BE00000B1FFDFBDF82040172C01D2172000E0B4
:108BF0002046A84201D92C4602E0172C00D21724A7
:108C000021463046FFF711FB21463046F9F775F94A
:108C10000020BCE7F8B51C4615460E46069F0AF034
:108C20001AF92346FF1DBCB231462A46009409F0CA
:108C300004FDF8BD70B50C4605460E220021204605
:108C400005F0EFFB002020802DB1012D01D0FFDFCA
:108C500070BD062000E00520A07170BD10B54880F1
:108C60000878134620F00F00001D20F0F00080303F
:108C70000C4608701422194604F1080005F0A7FB01
:108C800000F0CDFC3748046010BD2DE9F047DFF857
:108C9000D890491D064621F0030117460C46D9F825
:108CA000000009F0E0FD050000D1FFDF4FF00008F3
:108CB0003560A5F800802146D9F8000009F0D3FD01
:108CC000050000D1FFDF7560A5F800807FB104FBCF
:108CD00007F1091D0BD0D9F8000009F0C4FD04000C
:108CE00000D1FFDFB460C4F80080BDE8F087C6F8AB
:108CF0000880FAE72DE9F0411746491D21F00302EB
:108D0000194D064601681446286809F0D7FD224629
:108D10007168286809F0D2FD3FB104FB07F2121D0B
:108D200003D0B168286809F0C9FD042009F008FFE4
:108D30000446042009F00CFF201A012804D12868F9
:108D4000BDE8F04109F084BDBDE8F08110B50C46E6
:108D500005F0FEF800B1FFDF2046BDE81040FDF74A
:108D6000C6BF0000940200201800002038B50C4651
:108D70008288817B19B14189914200D90A462280BB
:108D8000C188121D90B26A4608F03EFFBDF800008F
:108D9000032800D30320C1B2208801F02AF838BD8F
:108DA00038B50C468288817B19B10189914200D97E
:108DB0000A462280C188121D90B26A4608F024FF3C
:108DC000BDF80000022800D30220C1B2208801F0C3
:108DD00010F8401CC0B238BD2DE9FF5F82468B46BB
:108DE000FB4814460BF10302D0E90110CDE9021053
:108DF00022F0030201A84FF49071019209F015FDD1
:108E0000F44E002C02D1F449019A8A600199014480
:108E10000191B57F05F1010504D1E8B20BF018FC12
:108E200000B1FFDF019800EB0510C01C20F003012A
:108E300001915CB9707AB27A1044C2B20020087015
:108E4000308C80B204F0E3FE00B1FFDF0198316A9C
:108E500008440190214601A800F08EFF8046019849
:108E6000C01C20F003000190B37AF27A717A04B149
:108E7000002009F0D0FD019908440190214601A885
:108E800000F0C2FFD34800273D4690F801900CE067
:108E9000284600F054FF064681788088F9F7C4F828
:108EA00071786D1C00FB0177EDB24D45F0D1019852
:108EB000C01C20F00300019004B100203946F9F7EE
:108EC000BEF80199002708440190C2483D4690F839
:108ED00001900CE0284600F032FF0646C1788088F9
:108EE000FEF707FC71786D1C00FB0177EDB24D4574
:108EF000F0D10198C01C20F00300019004B10020C3
:108F00003946FEF7FFFB01994FF000090844019034
:108F1000B0484D4647780EE0284600F010FF064660
:108F2000807B30B106F1080002F072F9727800FB24
:108F300002996D1CEDB2BD42EED10198C01C20F02B
:108F40000300019004B10020A3494A78494602F089
:108F500063F9019908440190214601A800F0BFFE81
:108F60000198C01D20F007000190DAF8001081423E
:108F700004D3A0EB0B01B1F5803F04DB4FF00408F4
:108F8000CAF8000004E0CAF80000B8F1000F03D0EE
:108F9000404604B0BDE8F09F74BB90490020019AA0
:108FA0000DF042FCFBF7ECF98A4C207F0090607FCB
:108FB000012823D0002318B3002286480021103056
:108FC000F8F716FA00B1FFDFE07FFEF748FF00B1C7
:108FD000FFDF80484FF4F6720021403005F021FA9F
:108FE0007C480421403080F8E91180F8EA1106211C
:108FF00080F8EB11032101710020CAE70123DAE7B1
:1090000002AADAE770B5734C06464034207804EBC8
:109010004015E078083598B9A01990F8E8010028C3
:109020000FD0A0780F2800D3FFDF20220021284690
:1090300005F0F7F9687866F3020068700120E070C7
:10904000284670BD2DE9F04105460C460027007802
:10905000052190463E46B1EB101F00D0FFDF287A75
:1090600050B101280ED0FFDFA8F800600CB12780B6
:1090700066800020BDE8F0810127092674B1688868
:10908000A08008E00227142644B16888A0802869DF
:10909000E060A88A2082287B2072E5E7A8F80060BB
:1090A000E7E730B54B4C0120002120706170207241
:1090B00060720322A272E0726177217721732174BA
:1090C000052121831F216183607445A161610A210B
:1090D000A177E077404D4FF4B06020626868C11C12
:1090E00021F00301814200D0FFDF6868606030BD7D
:1090F00030B5394C1568636810339D4202D20420A4
:10910000136030BD334B5D785A6802EB0512107066
:1091100051700320D080172090800120D070907073
:10912000002090735878401C587060681030606060
:10913000002030BD70B5064626480024457807E07B
:10914000204600F0FCFD0178B14204D0641CE4B27A
:10915000AC42F5D1002070BDF7B5074608780C4643
:1091600010B3FFF7E7FF0546A7F12006202F06D032
:10917000052E19D2DFE806F00F3838151A0000F076
:10918000E9FD0DB1697800E00021401AA17880B2B4
:109190000844FF2808D8A07830B1A088022831D22E
:1091A00002E0608817282DD20720FEBD207A48B340
:1091B00061881729F8D3A1881729F5D3A179002947
:1091C000F2D0E1790029EFD0402811D9ECE7000076
:1091D0000C560200B00300201C00002000000020FC
:1091E0006E52463578000000242F0BD1207A48B10A
:1091F00061884FF6FB70814202D8A188814201D973
:109200000420FEBD65B9207802AA0121FFF770FF96
:109210000028F6D12078FFF78DFF050000D1FFDF91
:10922000052E18D2DFE806F0030B0E081100A07817
:109230006870A088E8800FE06088A8800CE0A078C3
:10924000A87009E0A078E87006E054F8020FA86062
:109250006068E86000E0FFDF0020FEBD1A2835D01E
:109260000DDC132832D2DFE800F01B31203131272A
:109270002723252D313129313131312F0F0030286D
:1092800002D003DC1E2821D1072070473A38092874
:109290001CD2DFE800F0151B0F1B1B1B1B1B07005C
:1092A0000020704743F20400704743F20200704709
:1092B000042070470D2070470F207047082070472A
:1092C0001120704713207047062070470320704715
:1092D00010B5007800F0010008F088FCBDE81040EF
:1092E000BCE710B5007800F0010008F088FCBDE88C
:1092F0001040B3E70EB5017801F001018DF80010C0
:10930000417801F001018DF801100178C1F34001AD
:109310008DF802104178C1F340018DF803100178F7
:1093200089088DF80410417889088DF80510817836
:109330008DF80610C1788DF8071000798DF80800B7
:10934000684607F018FDFFF789FF0EBD2DE9F84FBD
:10935000DFF8F883FE4C00264FF490771FE00120E1
:1093600000F095FD0120FFF74DFE05463946D8F87F
:10937000080009F078FA686000B9FFDF686807F054
:10938000C8FBB0B12846FAF73EFB284600F085FD41
:1093900028B93A466968D8F8080009F08FFA94F9B4
:1093A000E9010428DBDA022009F0CAFB07460025A0
:1093B000A5E03A466968D8F8080009F07FFAF2E7B4
:1093C000B8F802104046491C89B2A8F80210B94208
:1093D00001D3002141800221B8F8020009F008FC05
:1093E000002864D0B8F80200694608F06FFBFFF768
:1093F00035FF00B1FFDF9DF8000078B1B8F802003A
:1094000009F03BFD5FEA000900D1FFDF484608F0A4
:10941000A8FF18B1B8F8020002F0C4F9B8F80200C9
:1094200009F019FD5FEA000900D1FFDF484608F0A6
:1094300090FFE0BB0321B8F8020009F0D9FB5FEA16
:10944000000B47D1FFDF45E0DBF8100010B10078DA
:10945000FF2849D0022000F01AFD0220FFF7D2FDBC
:109460008246484609F081F8CAF8040000B9FFDFD7
:10947000DAF8040009F049F9002100900170B8F809
:1094800002105046AAF8021002F092F8484609F07D
:109490003EF900B9FFDF504600F0FFFC18B99AF81A
:1094A0000100000704D50098CBF8100012E024E07A
:1094B000DBF8100038B10178491C11F0FF01017090
:1094C00008D1FFDF06E000221146484600F005FC07
:1094D00000B9FFDF94F9EA01022805DBB8F80200C1
:1094E00002F02DF80028AFD194F9E901042804DB3B
:1094F000484609F070F900B101266D1CEDB2BD427D
:1095000004D294F9EA010228BFF65AAF002E7FF484
:1095100022AFBDE8F84F032000F0B9BC10B58B4C6A
:10952000E06008682061AFF2DB10F9F7CEFC6070F4
:1095300010BD87480021403801708448017085497A
:109540004160704770B505464FF080500C46D0F82A
:10955000A410491C05D1D0F8A810C9430904090C6E
:109560000BD050F8A01F01F0010129704168216063
:109570008068A080287830B970BD062120460CF0A4
:10958000D8FD01202870607940F0C000607170BD86
:1095900070B54FF080540D46D4F88010491C0BD1A3
:1095A000D4F88410491C07D1D4F88810491C03D181
:1095B000D4F88C10491C0CD0D4F880100160D4F879
:1095C00084104160D4F888108160D4F88C10C16098
:1095D00002E010210CF0ADFDD4F89000401C0BD13E
:1095E000D4F89400401C07D1D4F89800401C03D153
:1095F000D4F89C00401C09D054F8900F2860606893
:109600006860A068A860E068E86070BD2846BDE8B2
:10961000704010210CF08DBD4D480079F2E470B51A
:109620004B4CE07830B3207804EB4010407A00F0E7
:109630000700204490F9E801002800DCFFDF2078D3
:10964000002504EB4010407A00F00700011991F862
:10965000E801401E81F8E8012078401CC0B220706B
:109660000F2800D12570A078401CA0700CF058FC89
:10967000E57070BDFFDF70BD3EB50546032109F002
:10968000B7FA0446284609F0E6FB054604B9FFDFB1
:10969000206918B10078FF2800D1FFDF01AA6946D0
:1096A000284600F01AFB60B9FFDF0AE0002202A999
:1096B000284600F012FB00B9FFDF9DF8080000B15A
:1096C000FFDF9DF80000411E8DF80010EED22069EA
:1096D0000199884201D1002020613EBD70B5054648
:1096E000A0F57F400C46FF3800D1FFDF012C01D0F0
:1096F000FFDF70BDFFF790FF040000D1FFDF20788F
:1097000020F00F00401D20F0F000503020706580E8
:109710000020207201202073BDE870407FE72DE912
:10972000F04116460D460746FFF776FF040000D1CC
:10973000FFDF207820F00F00401D20F0F0005030B7
:109740002070678001202072286805E01C0000203E
:10975000F0030020381400202061A888A08226731E
:10976000BDE8F0415BE77FB5FFF7E4FC040000D102
:10977000FFDF02A92046FFF7F9FA054603A92046B4
:10978000FFF70EFB8DF800508DF80100BDF80800C2
:10979000001DADF80200BDF80C00001DADF804007E
:1097A000E088ADF80600684608F00AFA002800D004
:1097B000FFDF7FBD2DE9F05FF64E8146307810B1B6
:1097C0000820BDE8F09F4846F7F769FD08B1102072
:1097D000F7E7F14C207808B9FFF763FCA17A607ACB
:1097E0004D460844C4B200F0B5FAA04207D2201A90
:1097F000C1B22A460020FFF77BFC0028E1D1716846
:10980000E548C91C002721F003017160B3463E46BC
:109810003D46BA463C4690F801800AE0204600F0FA
:109820008EFA4178807B0E4410FB0155641CE4B233
:109830007F1C4445F2D10AEB870000EBC600D64EF0
:1098400000EB85005C46F17A012200EB8100DBF839
:109850000410451829464846FFF7BEFA070012D003
:109860000020FFF767FC05000BD005F113006168CD
:1098700020F00300884200D0FFDF7078401E707037
:10988000656038469DE7002229464846FFF7A4FA5E
:1098900000B1FFDFD9F8000060604FF6FF70608014
:1098A0000120207000208CE72DE9F0410446B948E2
:1098B00017460E46007810B10820BDE8F081084632
:1098C000F7F7C7FC08B11020F7E7B34D287808B9BF
:1098D000FFF7E7FB601E1E2807D8012C22D1307845
:1098E000FE281FD8A8770020E7E7A4F120001F2852
:1098F00005D8E0B23A463146BDE8F0412CE4A4F187
:1099000040001F2805D831462046BDE8F04100F050
:10991000ECBAA4F1A0001F2804D80020A02C03D08A
:10992000A12C06D00720C8E7317801F00101E977C2
:10993000C3E731680922F82901D38B0701D010460B
:10994000BBE76B7C03F00303012B04D16B8BD73394
:109950009CB28C42F3D82962AFE72DE9F0478146EB
:109960000E460846F7F79BFC48B94846F7F7B5FCA2
:1099700028B909F1030020F00301494502D0102065
:10998000BDE8F08784484FF0000A4030817869B123
:109990004178804600EB4114083437883246002174
:1099A000204600F088FA050004D027E0A6F800A0C1
:1099B0000520E5E7B9F1000F24D03088B84201D97D
:1099C0000C251FE0607800F00705284600F05FFADC
:1099D00008EB0507324697F8E8014946401C87F82E
:1099E000E801204607F5F47700F065FA0546387877
:1099F000401E3870032000F04AFA2DB10C2D01D022
:109A0000A6F800A02846BBE76078624E00F0070188
:109A1000012923D002290CD0032934D0FFDF98F884
:109A200001104046491CC9B288F801100F2935D0F1
:109A300036E0616821B1000702D46088FFF71CFEA0
:109A400098F8EA014746012802D17078F9F75CFAE4
:109A500097F9EA010428E2DBFFDFE0E7616821B162
:109A60004FF49072B06808F029FF98F8E901474672
:109A7000032802D17078F9F747FA97F9E901042829
:109A8000CDDBFFDFCBE7C00602D56088FFF7F4FD32
:109A900098F9EB010628C2DBFFDFC0E780F801A0E0
:109AA0008178491E8170617801F0070101EB08009F
:109AB00090F8E811491C80F8E811A3E770B50C464E
:109AC0000546F7F7C6FB18B92046F7F7E8FB08B1DB
:109AD000102070BD28460AF0F2FD207008B1002069
:109AE00070BD042070BD70B505460AF001FEC4B219
:109AF0002846F7F7F2FB08B1102070BD35B1287881
:109B00002C7018B1A04201D0072070BD2046FDF78F
:109B10005DFE052805D10AF0EEFD012801D00020E8
:109B200070BD0F2070BD70B5044615460E46084640
:109B3000F7F78FFB18B92846F7F7B1FB08B11020EB
:109B400070BD022C03D0102C01D0092070BD2A4614
:109B5000314620460AF0F9FD0028F7D0052070BDF7
:109B600070B514460D460646F7F773FB38B928461C
:109B7000F7F795FB18B92046F7F7AFFB08B11020AF
:109B800070BD2246294630460AF0E1FD0028F7D094
:109B9000072070BD1C000020B00300203EB5044625
:109BA000F7F77DFB08B110203EBD684607F057F877
:109BB000FFF754FB0028F7D19DF806002070BDF890
:109BC00008006080BDF80A00A08000203EBD70B58E
:109BD00005460C460846F7F780FB20B93CB12068E3
:109BE000F7F75DFB08B1102070BDA08828B12146B1
:109BF0002846BDE87040FDF741BE092070BD70B534
:109C000004460D460846F7F724FB90BB601E1E284D
:109C10000ED8032C01D9072070BD04B9FFDFFD4821
:109C200000EB840050F8041C2846BDE8704008474B
:109C3000A4F120001F2805D829462046BDE8704021
:109C4000FAF70BBBA4F160001F2805D8294620466F
:109C5000BDE87040F8F7A9BCF02C0BD0BF2CDAD1CE
:109C6000A878298800F0010001F058FB78B10020A5
:109C700070BD03E0A868F7F7ECFA08B11020F7E729
:109C8000284608F002F8BDE87040FFF7E7BA082060
:109C9000EEE770B504460D460846F7F700FB30B90D
:109CA000601E1E280FD82846F7F7D3FA08B11020F7
:109CB000DEE7012C03D0022C01D0032C01D10620B9
:109CC000D6E70720D4E7A4F120001F28F9D82946B9
:109CD0002046BDE87040FAF733BB08F009BB7CB5FD
:109CE0000446CD48007B00F0010511BB04F0BBFB2E
:109CF0000DB1226800E00022C8484178C06806F033
:109D0000E3FCC6481030C0788DF8000010B101287F
:109D100002D004E0012000E000208DF80000684639
:109D200007F00AF8BB4824380068019001A807F042
:109D300043FD002D02D02068283020607CBD30B566
:109D4000B54D04466878A04200D8FFDF686800EB94
:109D5000041030BD70B5B04800252C46467807E0A9
:109D60002046FFF7ECFF4078641C2844C5B2E4B2FB
:109D7000B442F5D128467BE72DE9F0410C46074671
:109D80004FF0000800F0EDF80646FF2801D94FF02B
:109D900013083868C01C20F003023A6054EA080433
:109DA00021D19D48F3B2072124300CF0CFFB09E00C
:109DB000072C10D2DFE804F0060408080A040600A5
:109DC000974804E0974802E0974800E097480CF075
:109DD000DDFB054600E0FFDFA54200D0FFDF641C8D
:109DE000E4B2072CE4D3386800EB06103860404634
:109DF00063E5021D5143452900D245210844C01C9A
:109E0000B0FBF2F0C0B270472DE9FC5F0646824815
:109E10004FF000088B464746444690F8019022E0F8
:109E20002046FFF78CFF050000D1FFDF6878694608
:109E30003844C7B22846FEF799FF824601A9284652
:109E4000FEF7AEFF0346BDF804005246001D81B286
:109E5000BDF80000001D80B208F048FF6A78641C5D
:109E600000FB0288E4B24C45DAD13068C01C20F017
:109E700003003060BBF1000F00D00020424639469D
:109E800008F042FF316808443060BDE8FC9F624939
:109E9000403108710020C87070475F494031CA786E
:109EA0002AB10A7801EB42110831814201D0012028
:109EB0007047002070472DE9F041064600781546AE
:109EC00000F00F0400201080601E0F46052800D30C
:109ED000FFDF50482A46183800EB8400394650F816
:109EE000043C3046BDE8F04118472DE9F0414A4EA8
:109EF0000C46402806D0412823D042282BD04328A6
:109F000006D123E0A07861780D18E178814201D96B
:109F10000720D2E42078012801D91320CDE4FF2DB9
:109F200008D80AF07FFD07460BF0B2FF381A801EF2
:109F3000A84201DA1220C0E42068B06020793073B2
:109F40000DE0BDE8F041084600F036B80878022878
:109F5000DED8307703E008780228D9D8707700205F
:109F6000ABE42DE9F047DFF8B0900026344699F8CD
:109F7000090099F80A2099F801700244D5B299F8BD
:109F80000B20104400F0FF0808E02046FFF7D7FE42
:109F9000817B407811FB0066641CE4B2BC42F4D1C2
:109FA00099F8091099F80A0029442944414400B15C
:109FB000012008443044E3E438B50446407800F01A
:109FC0000300012803D002280BD0072038BD6068A9
:109FD00058B1F7F78BF9D0B96068F7F77EF920B977
:109FE00015E06068F7F735F988B969462046FCF74F
:109FF0004BF80028EAD1607800F00300022817D15E
:10A000009DF80000A0B16068F7F767F980B11020F3
:10A0100038BD000030560200B00300201C000020B4
:10A020005B41000039B30000DD2F00004344010014
:10A030006189F8290DD8208988420AD8607800F013
:10A0400003020A48012A06D1D731026A89B28A423C
:10A0500001D20920DCE794E80E0000F1100585E844
:10A060000E000AB9002101830020D1E7B0030020CF
:10A070002DE9F041074614468846084601F08AFD5E
:10A08000064608EB88001C22796802EBC0000D1818
:10A09000688C58B14146384601F08BFD014678681E
:10A0A0000078C200082305F120000CE0E88CA8B17C
:10A0B0004146384601F084FD01467868082340781F
:10A0C000C20005F1240008F050FC38B106212172CD
:10A0D0006681D0E90010C4E9031009E02878092856
:10A0E0000BD00520207266816868E060002028702F
:10A0F0002046BDE8F04101F02EBD072020726681A8
:10A10000F4E72DE9F04116460D460746406801EB9D
:10A1100085011C2202EBC1014418204601F072FDAA
:10A1200040B10021708865F30F2160F31F410620C4
:10A130000CF0E6FA09202070324629463846BDE880
:10A14000F04195E72DE9F0410E46074600241C2119
:10A15000F07816E004EB8403726801EBC303D25C71
:10A160006AB1FFF759FA050000D1FFDF6F802A4678
:10A1700021463046FFF7C5FF0120BDE8F081641C91
:10A18000E4B2A042E6D80020F7E770B50646002406
:10A190001C21C0780AE000BF04EB8403726801EB65
:10A1A000C303D5182A782AB1641CE4B2A042F3D8BC
:10A1B000402070BD28220021284604F032F9706842
:10A1C00080892881204670BD70B5034600201C257B
:10A1D000DC780CE000EB80065A6805EBC6063244DA
:10A1E000167816B1128A8A4204D0401CC0B284424A
:10A1F000F0D8402070BDF0B5044600201C26E5785C
:10A200000EE000BF00EB8007636806EBC7073B4426
:10A210001F788F4202D15B78934204D0401CC0B2B9
:10A220008542EFD84020F0BD0078032801D00020FF
:10A230007047012070470078022801D00020704745
:10A24000012070470078072801D0002070470120C6
:10A2500070472DE9F041064688461078F17815469A
:10A26000884200D3FFDF2C781C27641CF078E4B20E
:10A27000A04201D8201AC4B204EB8401706807EB35
:10A28000C1010844017821B14146884708B12C70CA
:10A2900073E72878A042E8D1402028706DE770B5B8
:10A2A00014460B880122A240134207D113430B80AE
:10A2B00001230A22011D08F022FB047070BD2DE964
:10A2C000FF4F81B00878DDE90E7B9A4691460E4635
:10A2D00040072CD4019808F0D0FD040000D1FFDF26
:10A2E00007F1040820461FFA88F107F00DFF05006A
:10A2F00000D1FFDF204629466A4608F058F9009849
:10A30000A0F80370A0F805A0284608F0FEF901782F
:10A3100069F306016BF3C711017020461FFA88F13B
:10A3200007F035FF00B9FFDF019806F03CF906EBB6
:10A330000900017F491C017705B0BDE8F08F2DE9C8
:10A34000F84F0E469A4691460746032108F050FC06
:10A350000446008DDFF8B885002518B198F8000094
:10A36000B0421ED1384608F088FD070000D1FFDF5B
:10A3700009F10401384689B207F0C6FE050010D085
:10A38000384629466A4608F012F9009800210A4624
:10A390000180817006F0C3F90098C01DCAF8000062
:10A3A00021E098F80000B04216D104F1260734F8F5
:10A3B000341F012000FA06F911EA090F00D0FFDF6F
:10A3C0002088012340EA090020800A22391D3846EE
:10A3D00008F0B0FA067006E0324604F1340104F1E8
:10A3E0002600FFF75CFF0A2188F800102846BDE828
:10A3F000F88FFEB515460C46064602AB0C22062128
:10A40000FFF79DFF002827D00299607812220A707A
:10A41000801C487008224A80A07002982988052371
:10A4200081806988C180A9880181E98841810025EE
:10A430000C20CDE90005062221463046FFF73FFFFC
:10A440002946002266F31F41F02310460CF0AEF8B7
:10A450006078801C60700120FEBDFEB514460D467C
:10A460000622064602AB1146FFF769FF002812D00C
:10A47000029B132000211870A87858700220588081
:10A480009C800620CDE9000102460523294630467E
:10A49000FFF715FF0120FEBD2DE9FE430C46804667
:10A4A00044E002AB0E2207214046FFF748FF002898
:10A4B00041D060681C2267788678BF1C06EB860155
:10A4C00002EBC101451802981421017047700A215E
:10A4D0004180698A0181E98A4181A9888180A989AD
:10A4E0008181304601F056FB029905230722C8807E
:10A4F0006F700420287000250E20CDE9000521464C
:10A500004046FFF7DCFE294666F30F2168F31F4142
:10A51000F023002206200CF049F86078FD49801CE9
:10A52000607062682046921CFFF793FE6068807836
:10A530004028B6D10120BDE8FE83FEB50D46064693
:10A5400038E002AB0E2207213046FFF7F8FE002864
:10A5500035D068681C23C17801EB810203EBC2028D
:10A560008418029815220270627842700A22428092
:10A57000A2894281A2888281084601F00BFB014634
:10A5800002988180618AC180E18A0181A088B8B186
:10A590000020207000210E20CDE9000105230722B4
:10A5A00029463046FFF78BFE6A68DB492846D21CF5
:10A5B000FFF74FFE6868C0784028C2D10120FEBD79
:10A5C0000620E6E72DE9FE430C46814644E020469E
:10A5D00001F002FBD0B302AB082207214846FFF787
:10A5E000AEFE0028A7D060681C2265780679AD1CF5
:10A5F00006EB860102EBC10147180298B7F81080FC
:10A6000006210170457004214180304601F0C2FAF4
:10A610000146029805230722C180A0F804807D70BE
:10A62000082038700025CDE9000521464846FFF78F
:10A6300046FE294666F30F2169F31F41F0230022ED
:10A6400006200BF0B3FF6078801C60706268B3492D
:10A650002046121DFFF7FDFD606801794029B6D143
:10A66000012068E72DE9F34F83B00D4691E02846BD
:10A6700001F0B2FA00287DD068681C2290F806A08C
:10A680000AEB8A0102EBC10144185146284601F049
:10A6900097FAA178CB0069684978CA00014604F1AD
:10A6A000240008F07EF907468188E08B4FF000090E
:10A6B000091A8EB208B1C84607E04FF001085046AB
:10A6C00001F053FA08B9B61CB6B2208BB04200D8DC
:10A6D0000646B34602AB324607210398FFF72FFE2A
:10A6E000060007D0B8F1000F0BD0504601F03DFA3C
:10A6F00010B106E000201FE60299B8884FF0020969
:10A7000008800196E28B3968ABEB09001FFA80F8EC
:10A710000A4403984E46009208F0AFFBDDE90021A1
:10A72000F61D4346009607F0BCFFE08B404480B224
:10A73000E083B988884201D1012600E00026CDE9F6
:10A7400000B6238A072229460398FFF7B8FD504632
:10A7500001F00BFA10B9E089401EE08156B1A078F3
:10A76000401CA0706868E978427811FB02F1CAB217
:10A77000012300E007E081690E3008F0C0F880F89E
:10A7800000A00020E0836A6865492846921DFFF713
:10A7900060FD6868817940297FF469AF0120CBE5CD
:10A7A00070B5064648680D4614468179402910D197
:10A7B00004EB84011C2202EBC101084401F043FABE
:10A7C000002806D06868294684713046BDE870408C
:10A7D00048E770BDFEB50C460746002645E020461A
:10A7E00001F0FAF9D8B360681C22417901EB8101CC
:10A7F00002EBC1014518688900B9FFDF02AB0822EE
:10A8000007213846FFF79BFD002833D00299607876
:10A8100016220A70801C48700420488060684079C5
:10A8200001F0B8F901460298052307228180698961
:10A83000C1800820CDE9000621463846FFF73FFDDC
:10A840006078801C6070A88969890844B0F5803FF1
:10A8500000D3FFDFA88969890844A8816E816268F6
:10A8600030492046521DFFF7F4FC606841794029C9
:10A87000B5D10120FEBD30B5438C458BC3F3C70471
:10A88000002345B1838B641EED1AC38A6D1E1D44DF
:10A8900095FBF3F3E4B22CB1008918B1A04200D8C3
:10A8A000204603444FF6FF70834200D303461380D3
:10A8B0000C7030BD2DE9FC41074616460D46486830
:10A8C00002EB86011C2202EBC10144186A4601A971
:10A8D0002046FFF7D0FFA089618901448AB2BDF804
:10A8E0000010914212D0081A00D5002060816868DB
:10A8F000407940280AD1204601F09BF9002805D074
:10A900006868294646713846FFF764FFBDE8FC8158
:10A910003000002029A2000037A2000045A200005C
:10A9200047BC000033BC00002DE9FE4F0F468146B6
:10A9300015465088032108F05BF90190B9F8020030
:10A9400001F01BF982460146019801F045F9002803
:10A9500024D001981C2241680AEB8A0002EBC00057
:10A960000C18204601F04EF9002817D1B9F8000064
:10A97000E18A88420ED8A18961B1B8420ED1002681
:10A980005146019801F015F9218C01EB0008608B0C
:10A9900030B114E0504601F0E8F8A0B3BDE8FE8FF6
:10A9A000504601F0E2F808B1678308E0022FF5D3C2
:10A9B000B9F804006083618A884224D80226B81B53
:10A9C00087B2B8F80400A28B801A002814DD8742F1
:10A9D00000DA38461FFA80FB688869680291D8F867
:10A9E00000100A44009208F036FAF61D009A5B4601
:10A9F0000299009607F021FEA08B384480B2A08314
:10AA0000618B884207D96888019903B05246BDE836
:10AA1000F04F01F035B91FD14FF009002872B9F895
:10AA200002006881D8E90010C5E90410608BA88194
:10AA3000284601F090F85146019801F0BAF8014615
:10AA40000198082340680078C20004F1200007F054
:10AA50008CFF0020A0836083504601F086F810B977
:10AA6000A089401EA0816888019903B00AF0FF0206
:10AA7000BDE8F04F1EE72DE9F041064615460F46AA
:10AA80001C461846F6F7E5FB18B92068F6F707FCF0
:10AA900010B11020BDE8F0817168688C0978B0EBC6
:10AAA000C10F01D31320F5E73946304601F081F894
:10AAB0000146706808230078C20005F1200007F005
:10AAC0001EFFD4E90012C0E900120020E2E710B531
:10AAD0000446032108F08CF80146007800F00300DA
:10AAE000022805D02046BDE8104001F1140280E4A0
:10AAF0008A8A2046BDE81040AFE470B504460321C1
:10AB000008F076F8054601462046FFF75BFD002871
:10AB100016D029462046FFF75DFE002810D02946B2
:10AB20002046FFF70AFD00280AD029462046FFF7F5
:10AB3000B3FC002804D029462046BDE8704091E5CA
:10AB400070BD2DE9F0410C4680461EE0E178427868
:10AB500011FB02F1CAB2816901230E3007F005FF33
:10AB6000077860681C22C179491EC17107EB870113
:10AB7000606802EBC10146183946204601F02CF806
:10AB800018B1304601F037F820B16068C17900296A
:10AB9000DCD17FE7FEF740FD050000D1FFDF0A2092
:10ABA0002872384600F0F6FF68813946204601F0E9
:10ABB00007F80146606808234078C20006F12400C7
:10ABC00007F0D3FED0E90010C5E90310A5F8028014
:10ABD000284600F0C0FFB07800B9FFDFB078401E13
:10ABE000B07057E770B50C460546032108F000F831
:10ABF00001464068C2792244C2712846BDE87040CF
:10AC00009FE72DE9FE4F8246507814460F464FF0DD
:10AC1000000800284FD0012807D0022822D0FFDFEB
:10AC20002068B8606068F860B8E602AB0E220821C0
:10AC30005046FFF784FB0028F2D002981521052327
:10AC40000170217841700A214180C0F80480C0F869
:10AC50000880A0F80C80628882810E20CDE900086F
:10AC6000082221E0A678304600F094FF054606EB66
:10AC700086012C22786802EBC1010822465A02ABF9
:10AC800011465046FFF75BFB0028C9D00298072108
:10AC90000170217841700421418008218580C6809F
:10ACA000CDE9001805230A4639465046FFF707FB51
:10ACB00087F8088072E6A678022516B1022E13D016
:10ACC000FFDF2A1D914602AB08215046FFF737FBF4
:10ACD0000028A5D002980121022E01702178417030
:10ACE0004580868002D005E00625EAE7A188C1807C
:10ACF000E1880181CDE900980523082239465046B4
:10AD0000D4E710B50446032107F072FF014600F1B5
:10AD100008022046BDE8104073E72DE9F04F0F46CA
:10AD200005468DB014465088032107F061FF4FF0AF
:10AD300000088DF814800646ADF81680042F7BD3EA
:10AD40006A78002A78D028784FF6FF794FF01C0AED
:10AD5000132834D008DC012871D006284AD00728EF
:10AD60006ED012280ED106E014286AD0152869D0BA
:10AD7000162807D1AAE10C2F04D1307800F0030186
:10AD8000022907D0CDF80880CDF80C8068788DF8BE
:10AD900008004CE040F0080030706878B070012086
:10ADA0008DF81400A888ADF81800E888ADF81A00EE
:10ADB0002889ADF81C006889ADF81E0011E1B07853
:10ADC000904239D13078010736D5062F34D120F0A2
:10ADD000080030706088414660F31F4100200BF08E
:10ADE0008FFC02208DF81400ADF81890A888ADF8FB
:10ADF0001A00F6E0082F1FD1A888EF88814600F0DE
:10AE0000BCFE80460146304600F0E6FE18B14046E2
:10AE100000F0ABFEB8B1FC48D0E90010CDE902105B
:10AE20006878ADF80C908DF80800ADF80E70608869
:10AE300002AA3146FFF7E5FE0DB0BDE8F08FB6E09F
:10AE40001EE041E0ECE0716808EB88002C2202EB88
:10AE5000C000085AB842EFD1EB4802AAD0E902106C
:10AE6000CDE9021068788DF8080008F0FF058DF82C
:10AE70000A5060883146FFF7C4FE224629461FE08B
:10AE8000082FD9D1B5F80480E88800F076FE07468F
:10AE90000146304600F0A0FE0028CDD007EB870227
:10AEA00071680AEBC2000844028A4245C4D10178A5
:10AEB0000829C1D1407869788842BDD1F9B22246CB
:10AEC0003046FFF71EF9B7E70E2F7FF45BAFE98836
:10AED0006F898B46B5F808903046FFF775F9ABF1EE
:10AEE0004001402901D309204AE0B9F1170F01D3ED
:10AEF000172F01D20B2043E040280ED000EB800238
:10AF000071680AEBC20008440178012903D1407836
:10AF10006978884290D00A2032E03046FFF735F950
:10AF2000014640282BD001EB810372680AEBC30075
:10AF300002EB0008012288F800206A7888F80120D6
:10AF40007068AA884089B84200D93846AD89032381
:10AF50002372A282E7812082A4F80C9065820846C1
:10AF600000F018FE6081A8F81490A8F81870A8F8EE
:10AF70000E50A8F810B0204600F0EDFD5CE704206C
:10AF800005212172A4F80A80E081012121739E49E4
:10AF9000D1E90421CDE9022169788DF80810ADF8D6
:10AFA0000A00608802AA3146FFF72BFEE3E7062F6E
:10AFB00089D3B07890421AD13078010717D520F0A4
:10AFC000080030706088414660F31F4100200BF09C
:10AFD00097FB02208DF81400A888ADF81800ADF892
:10AFE0001A906088224605A9F9F7E3F824E70421BE
:10AFF0003046FFF700F905464028BFD00220830302
:10B00000009022462946304600F003FE4146608803
:10B0100065F30F2160F31F4106200BF071FB0BE776
:10B020000E2FABD104213046FFF7E5F881464028CA
:10B03000A4D04146608869F30F2160F31F410620C8
:10B040000BF05EFBA8890B906889099070682F89C6
:10B050004089B84200D938468346B5F80680A888AA
:10B060000A90484600F096FD60810B9818B10220C6
:10B0700000900B9B24E0B8F1170F1ED3172F1CD3A1
:10B080000420207209986082E781A4F810B0A4F827
:10B090000C8009EB890271680AEBC2000D18DDE92A
:10B0A0000913A5F81480A5F818B0E9812B82204671
:10B0B00000F051FD06202870BEE601200B23009011
:10B0C00022464946304600F0A4FDB5E6082F8DD152
:10B0D000A9883046FFF778F80746402886D000F068
:10B0E00044FD00289BD107EB870271680AEBC20080
:10B0F0000844804600F086FD002890D1ED88B8F81D
:10B100000E002844B0F5803F05D360883A463146AA
:10B1100000F0B6FD90E6002DCED0A8F80E006088B5
:10B120003A463146FFF73CFB08202072384600F0D3
:10B1300031FD6081A5811EE72DE9F05F0C460128F5
:10B140001FD0957992F8048092F8056005EB85018F
:10B150001F2202EBC10121F0030B08EB060111FBDA
:10B1600005F14FF6FF7202EAC10909F1030115FB6F
:10B170000611264F21F0031ABB6840B101283ED1C9
:10B1800025E06168E57891F800804E78DEE7594661
:10B19000184607F068FB606000B9FFDF5A460021DF
:10B1A000606803F03EF9E5705146B86807F05BFB54
:10B1B0006168486100B9FFDF6068426902EB09011C
:10B1C0008161606880F800806068467017E06068A0
:10B1D00052464169184607F071FB5A466168B868E3
:10B1E00007F06CFB032007F0ABFC0446032007F0DC
:10B1F000AFFC201A012802D1B86807F029FB0BEB3D
:10B200000A00BDE8F09F00003C560200300000201C
:10B210000246002102208FE7F7B5FF4C0A201646B0
:10B220002070009860B100254FEA0D0007F0FDFA8C
:10B230000021A1706670002D01D10099A160FEBDB2
:10B2400001250020F2E770B50C4615463822002192
:10B25000204603F0E6F8012666700A22002104F178
:10B260001C0003F0DEF805B9FFDF297A207861F3CE
:10B2700001002070A87900282DD02A462146002000
:10B28000FFF75AFF61684020E34A88706168C87020
:10B2900061680871616848716168887161682888AF
:10B2A0000881616868884881606886819078002894
:10B2B00011D061680620087761682888C8856168B0
:10B2C0002888488660680685606869889288018653
:10B2D00081864685828570BDC878002802D000220C
:10B2E000012029E7704770B50546002165F31F412D
:10B2F00000200BF005FA0321284607F079FC040032
:10B3000000D1FFDF21462846FEF71CFF002804D0AD
:10B31000207840F010002070012070BD70B5054607
:10B320000C46032007F0FEFB08B1002070BDBA48B0
:10B3300085708480012070BD2DE9FF4180460E4656
:10B340000F0CFEF769F9050007D06F80032138461E
:10B3500007F04EFC040008D106E004B03846BDE812
:10B36000F0411321F9F758BBFFDF5FEA080005D071
:10B37000B8F1060F18D0FFDFBDE8FF8120782A461C
:10B3800020F0080020700020ADF8020002208DF8A7
:10B3900000004FF6FF70ADF80400ADF806006946F6
:10B3A0003846F8F706FFE7E7C6F3072101EB81020D
:10B3B0001C23606803EBC202805C042803D00828C9
:10B3C0000AD0FFDFD8E7012000904FF440432A461F
:10B3D000204600F01EFCCFE704B02A462046BDE818
:10B3E000F041FEF78EBE2DE9F05F0546408900274B
:10B3F00090460C463E46824600F0BFFB8146287AC6
:10B40000C01E08286BD2DFE800F00D041920583662
:10B410003C4772271026002C6CD0D5E90301C4E903
:10B4200002015CE070271226002C63D00A2205F18D
:10B430000C0104F1080002F0CAFF50E071270C264D
:10B44000002C57D0E868A06049E0742710269CB310
:10B45000D5E90301C4E902016888032107F0C8FBAC
:10B460008346FEF7D9F80246688850804946584618
:10B47000FEF7FEFD33E075270A26ECB1A88920818E
:10B480002DE076271426BCB105F10C0004F1080369
:10B4900007C883E8070022E07727102664B1D5E9C2
:10B4A0000301C4E902016888032107F0A1FB0146FA
:10B4B0006888FFF746FB12E01CE073270826CCB132
:10B4C0006888032107F094FB01460078C00606D582
:10B4D0006888FEF737FE10B96888F8F778FAA8F898
:10B4E00000602CB12780A4F806A066806888A08040
:10B4F000002086E6A8F80060FAE72DE9FC410C463A
:10B500001E4617468046032107F072FB05460A2CAB
:10B510000AD2DFE804F00505050505050909090754
:10B52000042303E0062301E0FFDF0023CDE90076DA
:10B53000224629464046FEF7C2FEBDE8FC81F8B52A
:10B540000546A0F57F40FF382BD0284607F083FC46
:10B55000040000D1FFDF204607F007F8002821D0C3
:10B5600001466A46204607F022F800980321B0F809
:10B570000560284607F03CFB0446052E13D03046F4
:10B5800000F0FBFA05460146204600F025FB40B1DD
:10B59000606805EB85013E2202EBC101405A00289C
:10B5A00000D00120F8BD007A0028FAD00020F8BDB4
:10B5B000F8B50446408807F04EFC050000D1FFDFD7
:10B5C0006A462846616800F0C4FA01460098091FDF
:10B5D0008BB230F8032F0280428842800188994262
:10B5E00005D1042A08D0052A20D0062A16D02246E2
:10B5F0001946FFF799F9F8BD001D0E4605460146AC
:10B6000022463046F6F73FFF0828F4D12246294665
:10B610003046FCF77AF9F8BD300000206368648892
:10B620000A46011D2046FAF79DF9F4E72246001D5F
:10B63000FFF773FBEFE770B50D460646032107F0F1
:10B64000D7FA040004D02078000704D5112070BD7B
:10B6500043F2020070BD2A4621463046FEF7C9FE7D
:10B6600018B9286860616868A061207840F0080017
:10B670002070002070BD70B50D460646032107F00E
:10B68000B7FA040004D02078000704D4082070BD65
:10B6900043F2020070BD2A4621463046FEF7DDFE29
:10B6A00000B9A582207820F008002070002070BD2D
:10B6B0002DE9F04F0E4691B08046032107F098FA2D
:10B6C0000446404607F0D9FB074600200790089043
:10B6D0000990ADF830000A9002900390049004B9EC
:10B6E000FFDF0DF10809FFB9FFDF1DE038460BA9A8
:10B6F000002206F0FDFD9DF82C0000F07F050A2DCC
:10B7000000D3FFDF6019017F491E01779DF82C00EF
:10B71000000609D52A460CA907A8FEF7C0FD19F8AE
:10B720000510491C09F80510761EF6B2DED204F1A8
:10B730003400F84D04F1260BDFF8DCA304F12A07EE
:10B74000069010E05846069900F08CFA06462870DC
:10B750000A2800D3FFDF5AF8261040468847E08CBD
:10B76000C05DB04202D0208D0028EBD10A202870A5
:10B77000E94D4E4628350EE00CA907A800F072FAF4
:10B780000446375D55F8240000B9FFDF55F8242042
:10B79000394640469047BDF81E000028ECD111B054
:10B7A000BDE8F08F10B5032107F022FA040000D1A4
:10B7B000FFDF0A22002104F11C0002F032FE207893
:10B7C00040F00400207010BD10B50C46032107F0B6
:10B7D0000FFA2044007F002800D0012010BD2DE981
:10B7E000F84F894615468246032107F001FA070003
:10B7F00004D02846F5F72DFD40B903E043F20200DE
:10B80000BDE8F88F4846F5F74AFD08B11020F7E784
:10B81000786828B169880089814201D90920EFE759
:10B82000B9F800001C2488B100F0A7F98046014651
:10B83000384600F0D1F988B108EB8800796804EB4C
:10B84000C000085C01280BD00820D9E73846FEF775
:10B850009CFC8046402807D11320D1E70520CFE784
:10B86000FDF7DAFE06000BD008EB8800796804EBE0
:10B87000C0000C18B9F8000020B1E88910B113E03D
:10B880001120BDE72888172802D36888172801D21D
:10B890000720B5E7686838B12B1D22464146384677
:10B8A000FFF7E9F80028ABD104F10C026946204605
:10B8B000FEF7E1FF288860826888E082B9F800001E
:10B8C00030B102202070E889A080E889A0B12BE087
:10B8D00003202070A889A08078688178402905D14C
:10B8E00080F8028039465046FEF7D6FD404600F00B
:10B8F00051F9A9F8000021E07868218B408988423D
:10B9000000D908462083A6F802A004203072B9F8B6
:10B9100000007081E0897082F181208B3082A08AE2
:10B92000B081304600F017F97868C178402905D118
:10B9300080F8038039465046FEF7FFFD00205FE7A0
:10B9400070B50D460646032107F052F904000ED0EB
:10B95000284600F012F905460146204600F03CF961
:10B9600018B1284600F001F920B1052070BD43F25E
:10B97000020070BD05EB85011C22606802EBC1016D
:10B98000084400F03FF908B1082070BD2A4621465E
:10B99000304600F075F9002070BD2DE9F0410C46ED
:10B9A00017468046032107F023F90546204600F09C
:10B9B000E4F8044695B10146284600F00DF980B13F
:10B9C00004EB84011C22686802EBC1014618304672
:10B9D00000F018F938B10820BDE8F08143F2020008
:10B9E000FAE70520F8E73B46324621462846FFF7AE
:10B9F00042F80028F0D1E2B229464046FEF75AFF4D
:10BA0000708C0838082803D242484078F7F77CFA4F
:10BA10000020E1E72DE9F0410D461746804603215D
:10BA200007F0E6F80446284600F0A7F8064624B1D9
:10BA30003846F5F70EFC38B902E043F20200CBE7D6
:10BA40003868F5F706FC08B11020C5E731462046F6
:10BA500000F0C2F860B106EB86011C22606802EBC0
:10BA6000C1014518284600F0CDF818B10820B3E709
:10BA70000520B1E7B888A98A884201D90C20ABE734
:10BA80006168E88C4978B0EBC10F01D31320A3E7BC
:10BA90003146204600F094F801466068082340785B
:10BAA000C20005F1240006F02AFFD7E90012C0E920
:10BAB0000012F2B221464046FEF772FE00208BE7EC
:10BAC0002DE9F0470D461F4690468146032107F0B9
:10BAD0008FF80446284600F050F806463CB14DB1B8
:10BAE0003846F5F7FAFB50B11020BDE8F08743F275
:10BAF0000200FAE7606858B1A0F80C8027E03146F0
:10BB0000204600F069F818B1304600F02EF828B150
:10BB10000520EAE7300000205456020006EB8601BB
:10BB20001C22606802EBC1014518284600F06AF843
:10BB300008B10820D9E7A5F80880F2B221464846A6
:10BB4000FEF7B8FE1FB1A889698908443880002033
:10BB5000CBE706F02CBD017821F00F01491C21F044
:10BB6000F00110310170FDF75ABD20B94E488078C0
:10BB700008B101207047002070474B4989888842EE
:10BB800001D100207047402801D2402000E0403819
:10BB900080B2704710B50446402800D9FFDF204628
:10BBA000FFF7E3FF10B14048808810BD4034A0B2D9
:10BBB00010BD406842690078484302EBC0007047FE
:10BBC000C2784068037812FB03F24378406901FBB6
:10BBD000032100EBC1007047C2788A4209D940684E
:10BBE00001EB81011C2202EBC101405C08B1012084
:10BBF0007047002070470078062801D9012070475F
:10BC0000002070470078062801D0012070470020EE
:10BC10007047F0B401EB81061C27446807EBC606A9
:10BC20003444049D05262670E3802571F0BCFEF7A0
:10BC30001FBA10B5418911B1FFF7DDFF08B100202F
:10BC400010BD012010BD10B5C18C8278B1EBC20FC0
:10BC500004D9C18911B1FFF7CEFF08B1002010BD92
:10BC6000012010BD10B50C4601230A22011D06F06B
:10BC70007CFE00782188012282409143218010BD02
:10BC8000F0B402EB82051C264C6806EBC5050723C1
:10BC900063554B681C79402C03D11A71F0BCFEF738
:10BCA00091BCF0BC704700003000002010B5EFF3ED
:10BCB000108000F0010472B6F8484178491C4170C8
:10BCC0004078012801D10AF053F9002C00D162B666
:10BCD00010BD70B5F14CA07848B90125A570FFF7EB
:10BCE000E5FF0AF056F920B100200AF020F9002003
:10BCF00070BD4FF08040E570C0F80453F7E770B5B1
:10BD0000EFF3108000F0010572B6E44C607800B9E2
:10BD1000FFDF6078401E6070607808B90AF02CF987
:10BD2000002D00D162B670BDDC4810B5817821B11C
:10BD30000021C1708170FFF7E2FF002010BD10B537
:10BD400004460AF026F9D5498978084000D0012038
:10BD50002060002010BD10B5FFF7A8FF0AF019F908
:10BD600002220123CD49540728B1CD480260236146
:10BD70000320087202E00A72C4F8043300208871BC
:10BD800010BD2DE9F84FDFF814934278817889F8D7
:10BD90000420002689F80510074689F80660007817
:10BDA000DFF800B3354620B1012811D0022811D0A8
:10BDB000FFDF0AF000F94FF0804498B10AF002F971
:10BDC000B0420FD130460AF001F90028FAD042E023
:10BDD0000126EEE7FFF76AFF58460168C907FCD065
:10BDE0000226E6E70120E060C4F80451AE490E6087
:10BDF0000107D1F84412AC4AC1F342312432116038
:10BE0000A949343108604FF0020AC4F804A3A060C5
:10BE1000A6480168C94341F3001101F10108016816
:10BE200041F01001016001E019F01EFAD4F804019C
:10BE30000028F9D030460AF0C9F80028FAD0B8F145
:10BE4000000F04D19948016821F010010160C4F885
:10BE500008A3C4F8045199F805004E4680B138781B
:10BE600070B90AF096F880460AF02EFA6FF0004298
:10BE7000B8F1000F02D0C6E9032001E0C6E90302D1
:10BE8000DBF80000C00701D00AF07FF8387810B165
:10BE90003572BDE8F88F4FF01808C4F80883012701
:10BEA000A7614FF42070ADF8000000BFBDF800009E
:10BEB000411EADF80010F9D2C4F80C51C4F810516D
:10BEC0007648C01D0AF094F83570FFF744FF6761AB
:10BED0007549307920310860C4F80483D9E770B51A
:10BEE000050000D1FFDF4FF080424FF0FF30C2F875
:10BEF00008030021C2F80011C2F80411C2F80C11A5
:10BF0000C2F81011654C61700AF04FF810B10120B1
:10BF1000A070607063480068C00701D00AF035F86F
:10BF20002846BDE870402CE75C48007A002800D025
:10BF3000012070472DE9FC5F5D48D0F800905C4A15
:10BF40005C49083211608406D4F8080100B1012070
:10BF5000D4F8001111B14FF0010801E04FF00008D2
:10BF6000D4F8041101B101210191D4F80C1101B1EF
:10BF700001210091D4F8101101B10121474D8A46E9
:10BF800095F800B0002620B1C4F80861012009F03E
:10BF9000CEFF4248C01D0AF033F800B1FFDF012791
:10BFA000B8F1000F10D0C4F80873E87818B1EE703B
:10BFB000002009F0BCFF287A022805D1032028724E
:10BFC0003748022101602761019808B1C4F8046173
:10BFD000009850B1C4F80C61287A032800D0FFDF24
:10BFE0002F4806602F72FFF78AFEBAF1000F07D0C4
:10BFF000C4F81061287A012801D100F05DF867616A
:10C00000BBF1000F07D02E70287A012801D1FFF76D
:10C01000A2FEFFF774FE2148C01D0AF007F824496C
:10C02000091DC1F80090BDE8FC9F1C4810B5C01D5B
:10C0300009F0E6FF194940B1012008704FF0E021F6
:10C04000C1F80002BDE8104030E6087A012801D1AD
:10C05000FFF781FE1148BDE81040C01D09F0E6BFA2
:10C0600070B50E4CA07808B909F086FF012085074D
:10C07000A861207A002603280AD100BFD5F80C0158
:10C0800020B9002009F0A2FF0028F7D1C5F80C6103
:10C0900026724FF0FF30C5F8080370BD4400002041
:10C0A000340C00400C0400401805004010ED00E086
:10C0B000100502400100000170B5134C6079F0B129
:10C0C000012803D0A179401E814218DA09F061FFEE
:10C0D00005460AF0F9F86179012902D9A179491CCC
:10C0E000A1710DB1216900E0E168411A022902DA6B
:10C0F00011F1020FD1DC0DB1206100E0E060BDE87C
:10C10000704028E6C9E70000440000200F4A12688A
:10C110000D498A420CD118470C4A12680A4B9A42C0
:10C1200006D101B50AF0A2F80AF075FBBDE801409E
:10C13000074909680958084706480749054A064B50
:10C140007047000000000000BEBAFECA5C0000207C
:10C1500004000020B8130020B8130020F8B51D46D5
:10C16000DDE906470E000AD006F087FE2346FF1DD4
:10C17000BCB231462A46009406F093FAF8BDD019B5
:10C180002246194602F023F92046F8BD70B50D4647
:10C1900004461022002102F044F925811720608115
:10C1A000A07B40F00A00A07370BD4FF6FF720A80BA
:10C1B000014602200AF0A4BA704700897047827BCA
:10C1C000D30701D1920703D48089088000207047EB
:10C1D00005207047827B920700D581817047014618
:10C1E0000020098841F6FE52114200D0012070471C
:10C1F00000B50346807BC00701D0052000BD5981F2
:10C200001846FFF7ECFFC00703D0987B40F004000E
:10C210009873987B40F001009873002000BD827BEA
:10C22000520700D509B14089704717207047827BBB
:10C2300061F3C302827370472DE9FC5F0E4604462A
:10C2400001789646012000FA01F14DF6FF5201EA0D
:10C25000020962684FF6FF7B1188594502D1092017
:10C26000BDE8FC9FB9F1000F05D041F6FE5529420B
:10C2700001D00120F4E741EA090111801D0014D02A
:10C2800000232B7094F800C0052103221F464FF0B5
:10C29000020ABCF10E0F76D2DFE80CF0F909252F67
:10C2A00047646B77479193B4D1D80420D8E761688D
:10C2B00020898B7B9B0767D517284AD30B8983423C
:10C2C00047D38989172901D3814242D185F800A03B
:10C2D000A5F801003280616888816068817B21F067
:10C2E00002018173C6E0042028702089A5F80100AE
:10C2F0006089A5F803003180BCE0208A3188C01D28
:10C300001FFA80F8414524D3062028702089A5F81B
:10C3100001006089A5F80300A089A5F805000721A0
:10C32000208ACDE90001636941E00CF0FF00082894
:10C3300010D0082028702089A5F801006089A5F890
:10C34000030031806A1D694604F10C0008F0FFF912
:10C3500010B15EE01020EDE730889DF80010084431
:10C36000308087E00A2028702089A5F801003280FB
:10C3700044E00C2028702089A5F801006089A5F808
:10C38000030031803AE082E064E02189338800EBE9
:10C3900041021FFA82F843453BD3B8F1050F38D369
:10C3A0000E222A700BEA4101CDE90010E368608893
:10C3B0002A467146FFF7D2FEA6F800805AE04020D8
:10C3C000287060893188C01C1FFA80F8414520D34D
:10C3D0002878714620F03F00123028702089A5F897
:10C3E00001006089CDE9000260882A46E368FFF712
:10C3F000B5FEA6F80080287840063BD46168208905
:10C40000888037E0A0893288401D1FFA80F84245B5
:10C4100001D204273DE0162028702089A5F80100EC
:10C420006089A5F80300A089CDE9000160882A464B
:10C4300071462369FFF792FEA6F80080DEE7182018
:10C440002870207A6870A6F800A013E061680A8856
:10C45000920401D405271CE0C9882289914201D0A9
:10C46000062716E01E21297030806068018821F4BB
:10C4700000510180B9F1000F0BD0618878230022B0
:10C4800002200AF093F861682078887006E0338013
:10C4900003276068018821EA090101803846DFE648
:10C4A0002DE9FF4F85B01746129C0D001E461CD08B
:10C4B0003078C10703D000F03F00192801D90121CD
:10C4C00000E000212046FFF7AAFEA8420DD32088F5
:10C4D000A0F57F41FF3908D03078410601D400062D
:10C4E00005D5082009B0BDE8F08F0720FAE7002045
:10C4F0008DF800008DF8010030786B1E00F03F0CC5
:10C500000121A81E4FF0050A4FF002094FF0030B5E
:10C510009AB2BCF1200F75D2DFE80CF08B10745E7C
:10C520007468748C749C74B574BA74C874D474E1EF
:10C53000747474F174EF74EE74ED748B052D78D10E
:10C540008DF80090A0788DF804007088ADF8060092
:10C5500030798DF80100707800F03F000C2829D068
:10C560000ADCA0F10200092863D2DFE800F01262C1
:10C5700015621A621D622000122824D004DC0E28E5
:10C580001BD01028DBD11BE016281FD01828D6D1CD
:10C590001FE02078800701E020784007002848DA73
:10C5A000EEE020780007F9E72078C006F6E720786B
:10C5B0008006F3E720784006F0E720780006EDE7F4
:10C5C0002088C005EAE720884005E7E720880005C5
:10C5D000E4E72088C004E1E72078800729D5032D0F
:10C5E00027D18DF800B0B6F8010081E02178490725
:10C5F0001FD5062D1DD381B27078012803D00228E3
:10C6000017D102E0C9E0022000E0102004228DF8DA
:10C61000002072788DF80420801CB1FBF0F2ADF898
:10C62000062092B242438A4203D10397ADF80890A4
:10C63000A6E079E02078000776D598B282088DF8D8
:10C6400000A0ADF80420B0EB820F6DD10297ADF8D9
:10C65000061095E02178C90666D5022D64D381B213
:10C6600006208DF80000707802285DD3B1FBF0F24F
:10C670008DF80400ADF8062092B242438A4253D1AD
:10C68000ADF808907BE0207880064DD5072003E0C8
:10C69000207840067FD508208DF80000A088ADF8EE
:10C6A0000400ADF80620ADF8081068E02078000618
:10C6B00071D50920ADF804208DF80000ADF8061002
:10C6C00002975DE02188C90565D5022D63D381B24B
:10C6D0000A208DF80000707804285CD3C6E7208813
:10C6E000400558D5012D56D10B208DF80000A088AB
:10C6F000ADF8040044E021E026E016E0FFE72088E2
:10C70000000548D5052D46D30C208DF80000A088E3
:10C71000ADF80400B6F803006D1FADF80850ADF891
:10C720000600ADF80AA02AE035E02088C00432D522
:10C73000012D30D10D208DF8000021E020888004EB
:10C7400029D4B6F80100E080A07B000723D5032D93
:10C7500021D3307800F03F001B2818D00F208DF82F
:10C760000000208840F40050A4F80000B6F8010052
:10C77000ADF80400ED1EADF80650ADF808B0039713
:10C7800069460598F5F7C8FB050008D016E00E20AD
:10C790008DF80000EAE7072510E008250EE0307864
:10C7A00000F03F001B2809D01D2807D00220059962
:10C7B00009F0A6FF208800F400502080A07B4007ED
:10C7C00008D52046FFF70BFDC00703D1A07B20F062
:10C7D0000400A073284685E61FB5022806D1012073
:10C7E0008DF8000088B26946F5F796FB1FBD000082
:10C7F000F8B51D46DDE906470E000AD006F03DFB00
:10C800002346FF1DBCB231462A46009405F049FF7D
:10C81000F8BDD0192246194601F0D9FD2046F8BDD1
:10C820002DE9FF4F8DB09B46DDE91B57DDF87CA05D
:10C830000C46082B05D0E06901F0FEF850B110203D
:10C84000D2E02888092140F0100028808AF80010E2
:10C85000022617E0E16901208871E2694FF4205156
:10C860009180E1698872E06942F601010181E06925
:10C87000002181732888112140F0200028808AF847
:10C880000010042638780A900A2038704FF0020908
:10C8900004F118004D460C9001F0C6FBB04681E053
:10C8A000BBF1100F0ED1022D0CD0A9EB0800801C9B
:10C8B00080B20221CDE9001005AB52461E990D98B9
:10C8C000FFF796FFBDF816101A98814203D9F74872
:10C8D00000790F9004E003D10A9808B138702FE076
:10C8E0004FF00201CDE900190DF1160352461E99D1
:10C8F0000D98FFF77DFF1D980088401B801B83B2B9
:10C90000C6F1FF00984200D203461E990BA8D9B188
:10C910005FF00002DDF878C0CDE9032009EB0601E5
:10C9200089B2CDE901C10F980090BDF81610002220
:10C930000D9801F00EFC387070B1C0B2832807D09A
:10C94000BDF8160020833AE00AEB09018A19E1E7F5
:10C95000022011B0BDE8F08FBDF82C00811901F064
:10C96000FF08022D0DD09AF80120424506D1BDF8EE
:10C970002010814207D0B8F1FF0F04D09AF801804F
:10C980001FE08AF80180C94800680178052902D1B2
:10C99000BDF81610818009EB08001FFA80F905EB3D
:10C9A000080085B2DDE90C1005AB0F9A01F03FFBE2
:10C9B00028B91D980088411B4145BFF671AF022D73
:10C9C00013D0BBF1100F0CD1A9EB0800801C81B271
:10C9D0000220CDE9000105AB52461E990D98FFF7E4
:10C9E00007FF1D980580002038700020B1E72DE971
:10C9F000F8439C46089E13460027B26B9AB3491F22
:10CA00008CB2F18FA1F57F45FF3D05D05518AD885B
:10CA10002944891D8DB200E000252919B6F83C8013
:10CA20000831414520D82A44BCF8011022F8021BE5
:10CA3000BCF8031022F8021B984622F8024B9146DC
:10CA400006F009FA4FF00C0C41464A462346CDF851
:10CA500000C005F0F2FDF587B16B00202944A41D4C
:10CA60002144088003E001E0092700E083273846DD
:10CA7000BDE8F88310B50B88848F9C420CD9846B79
:10CA8000E018048844B1848824F40044A41D23449D
:10CA90000B801060002010BD0A2010BD2DE9F0476A
:10CAA0008AB00025904689468246ADF8185007277F
:10CAB0004BE0059806888088000446D4A8F80060FA
:10CAC00007A8019500970295CDE903504FF4007334
:10CAD00000223146504601F03CFB04003CD1BDF839
:10CAE0001800ADF82000059804888188B44216D15A
:10CAF0000A0414D401950295039521F4004100978E
:10CB0000049541F4804342882146504601F0BFF825
:10CB100004000BD10598818841F40041818005AA69
:10CB200008A94846FFF7A6FF0400DCD00097059847
:10CB300002950195039504950188BDF81C300022EB
:10CB4000504601F0A4F80A2C06D105AA06A94846C9
:10CB5000FFF790FF0400ACD0ADF8185004E0059842
:10CB6000818821F40041818005AA06A94846FFF783
:10CB700081FF0028F3D00A2C03D020460AB0BDE87C
:10CB8000F0870020FAE710B50C46896B86B051B1EA
:10CB90000C218DF80010A18FADF80810A16B019148
:10CBA0006946FAF747FB00204FF6FF71A063E18763
:10CBB000A08706B010BD2DE9F0410D460746896BF0
:10CBC0000020069E1446002911D0012B0FD13246B9
:10CBD00029463846FFF762FF002808D1002C06D00E
:10CBE000324629463846BDE8F04100F034BFBDE882
:10CBF000F0812DE9FC411446DDE9087C0E46DDE9B3
:10CC00000A15521DBCF800E092B2964502D20720E8
:10CC1000BDE8FC81ACF8002017222A70A5F801605D
:10CC2000A5F803300522CDE900423B462A46FFF72E
:10CC3000DFFD0020ECE770B50C46154648220021C8
:10CC4000204601F0EEFB04F1080044F81C0F002020
:10CC50004FF6FF71E06161842084A5841720E08491
:10CC600094F82A0040F00A0084F82A0070BD4FF6BC
:10CC7000FF720A800146032009F042BD30B585B03D
:10CC80000C460546FFF77FFFA18E284629B10121FA
:10CC90008DF800106946FAF7CDFA0020E0622063B3
:10CCA000606305B030BDB0F8400070476000002000
:10CCB00090F84620920703D4408808800020F4E7CB
:10CCC0000620F2E790F846209207EED5A0F844102F
:10CCD000EBE70146002009880A0700D5012011F082
:10CCE000F00F01D040F00200CA0501D540F0040069
:10CCF0008A0501D540F008004A0501D540F0100032
:10CD00000905D2D540F02000CFE700B5034690F8E2
:10CD10004600C00701D0062000BDA3F84210184607
:10CD2000FFF7D7FF10F03E0F05D093F8460040F014
:10CD3000040083F8460013F8460F40F00100187015
:10CD4000002000BD90F84620520700D511B1B0F880
:10CD50004200AAE71720A8E710F8462F61F3C302A4
:10CD60000270A2E72DE9FF4F9BB00E00DDE92B34E6
:10CD7000DDE92978289D24D02878C10703D000F068
:10CD80003F00192801D9012100E000212046FFF7CA
:10CD9000D9FFB04215D32878410600F03F010CD4EA
:10CDA0001E290CD0218811F47F6F0AD13A8842B134
:10CDB000A1F57F42FF3A04D001E0122901D100061B
:10CDC00002D504201FB0C5E5FA491D984FF0000AAE
:10CDD00008718DF818A08DF83CA00FAA0A60ADF874
:10CDE0001CA0ADF850A02978994601F03F02701FB1
:10CDF0005B1C04F1180C4FF0060E4FF0040BCDF83D
:10CE000058C01F2A7ED2DFE802F07D7D107D267D8E
:10CE1000AC7DF47DF37DF27DF17DF47DF07D7D7D53
:10CE2000EF7DEE7D7D7D7D7DED0094F84610B5F8BB
:10CE30000100890701D5032E02D08DF818B01EE33A
:10CE40004FF40061ADF85010608003218DF83C1064
:10CE5000ADF84000D4E2052EEFD1B5F801002083F3
:10CE6000ADF81C00B5F80310618308B1884201D900
:10CE7000012079E10020A07220814FF6FF7020840C
:10CE8000169801F0D1F8052089F8000002200290E0
:10CE900083460AAB1D9A16991B9801F0C8F890BBFF
:10CEA0009DF82E00012804D0022089F801001020EE
:10CEB00003E0012089F8010002200590002203A967
:10CEC0000BA807F044FCE8BB9DF80C0005998142D3
:10CED0003DD13988801CA1EB0B01814237DB0299DF
:10CEE0000220CDE900010DF12A034A4641461B9874
:10CEF000FFF77EFC02980BF1020B801C81B217AA8F
:10CF0000029101E09CE228E003A90BA807F01FFCB6
:10CF100002999DF80C00CDE9000117AB4A46414645
:10CF20001B98FFF765FC9DF80C000AAB0BEB0001AA
:10CF30001FFA81FB02991D9A084480B2029016994B
:10CF40001B9800E003E001F072F80028B6D0BBF1B6
:10CF5000020F02D0A7F800B04FE20A208DF81800A7
:10CF60004BE200210391072EFFF467AFB5F80100F3
:10CF70002083ADF81C00B5F80320628300283FF43D
:10CF800077AF90423FF674AF0120A072B5F805006C
:10CF900020810020A073E06900F04EFD78B9E169BE
:10CFA00001208871E2694FF420519180E169887213
:10CFB000E16942F601000881E06900218173F01FF8
:10CFC00020841E98606207206084169801F02CF877
:10CFD000072089F800000120049002900020ADF89D
:10CFE0002A0028E019E29FE135E1E5E012E2A8E03D
:10CFF00080E043E00298012814D0E069807901289C
:10D0000003D1BDF82800ADF80E00049803ABCDE9BC
:10D0100000B04A4641461B98FFF7EAFB0498001D02
:10D0200080B20490BDF82A00ADF80C00ADF80E00F7
:10D03000059880B202900AAB1D9A16991B9800F0D1
:10D04000F6FF28B902983988001D05908142D1D297
:10D050000298012881D0E0698079012803D1BDF8C8
:10D060002800ADF80E00049803ABCDE900B04A46A5
:10D0700041461B98FFF7BCFB0298BDE1072E02D08A
:10D08000152E7FF4DAAEB5F801102183ADF81C102F
:10D09000B5F80320628300293FF4EAAE91423FF6DF
:10D0A000E7AE0121A1724FF0000BA4F808B084F89C
:10D0B0000EB0052E07D0C0B2691DE26907F045FB2E
:10D0C00000287FF44AAF4FF6FF70208401A906AA1A
:10D0D00014A8CDF800B081E885032878214600F037
:10D0E0003F031D9A1B98FFF79BFB8246208BADF8F0
:10D0F0001C0082E10120032EC3D14021ADF8501065
:10D10000B5F801102183ADF81C100AAAB8F1000F80
:10D1100000D00023CDE9020304921D98CDF80480CD
:10D12000009038880022401E83B21B9801F011F84D
:10D130008DF8180090BB0B2089F80000BDF828007E
:10D1400035E04FF0010C052E9BD18020ADF850004A
:10D15000B5F801102183B5F803002084ADF81C1048
:10D16000B0F5007F03D907208DF8180087E140F45F
:10D170007C4222840CA8B8F1000F00D00023CDE936
:10D180000330CDE9018C1D9800903888401E83B291
:10D190001B9800F0DEFF8DF8180018B18328A8D185
:10D1A0000220BFE00D2189F80010BDF83000401CBE
:10D1B00022E1000060000020032E04D248067FF523
:10D1C0003CAE002018E1B5F80110ADF81C1028782D
:10D1D000400602D58DF83CE002E007208DF83C00C7
:10D1E0004FF000080320CDE902081E9BCDF8108007
:10D1F0001D980193A6F1030B00901FFA8BF3424692
:10D200001B9800F044FD8DF818008DF83C802978BB
:10D2100049060DD52088C00506D5208BBDF81C1009
:10D22000884201D1C4F8248040468DF81880E3E09C
:10D23000832801D14FF0020A4FF48070ADF85000FE
:10D24000BDF81C002083A4F820B01E986062032063
:10D2500060841321CDE0052EFFF4EFADB5F8011089
:10D26000ADF81C10A28F6AB3A2F57F43FE3B29D014
:10D2700008228DF83C2000BF4FF0000B0523CDE9BC
:10D28000023BDDF878C0CDF810B01D9A80B2CDF821
:10D2900004C040F400430092B5F803201B9800F04E
:10D2A000F6FC8DF83CB04FF400718DF81800ADF825
:10D2B0005010832810D0F8B1A18FA1F57F40FE381F
:10D2C00007D0DCE00B228DF83C204FF6FE72A287DF
:10D2D000D2E7A4F83CB0D2E000942B4631461E9A27
:10D2E0001B98FFF784FB8DF8180008B183284BD1F9
:10D2F000BDF81C00208353E700942B4631461E9A4C
:10D300001B98FFF774FB8DF81800E8BBE18FA06B4A
:10D310000844831D8DE888034388828801881B9810
:10D32000FFF767FC824668E095F80180022E70D115
:10D330005FEA080002D0B8F1010F6AD109208DF828
:10D340003C0007A800908DF840804346002221460B
:10D350001B98FFF730FC8DF842004FF0000B8DF862
:10D3600043B050B9B8F1010F12D0B8F1000F04D199
:10D37000A18FA1F57F40FF380AD0A08F40B18DF872
:10D380003CB04FF4806000E037E0ADF850000DE0B5
:10D390000FA91B98F9F74EFF82468DF83CB04FF469
:10D3A0008060ADF85000BAF1020F06D0FC4800686A
:10D3B000C07928B18DF8180027E0A4F8188044E05F
:10D3C000BAF1000F03D081208DF818003DE007A8C6
:10D3D00000904346012221461B98FFF7ECFB8DF895
:10D3E000180021461B98FFF7CEFB9DF8180020B9C6
:10D3F000192189F80010012038809DF83C0020B1E7
:10D400000FA91B98F9F716FF8246BAF1000F33D027
:10D410001BE018E08DF818E031E02078000712D505
:10D42000012E10D10A208DF83C00E088ADF84000B4
:10D4300003201B9909F064F90820ADF85000C0E6FC
:10D4400048067FF5FAAC4FF0040A2088BDF850106A
:10D4500008432080BDF8500080050BD5A18FA1F5B1
:10D460007F40FE3806D11E98E06228982063A68689
:10D470004FF0030A5046A5E49DF8180078B101204A
:10D4800089F80000297889F80110BDF81C10A9F866
:10D4900002109DF8181089F80410052038802088A3
:10D4A000BDF8501088432080E4E72DE9FF4F8846FF
:10D4B000087895B0012181404FF20900249C014079
:10D4C000ADF820102088DDF88890A0F57F424FF05D
:10D4D000000AFF3A06D039B1000705D5012019B07E
:10D4E000BDE8F08F0820FAE7239E4FF0000B0EA84E
:10D4F00086F800B018995D460988ADF83410A8493F
:10D500008DF81CB0179A0A718DF838B0086098F839
:10D51000000001283BD0022809D003286FD13078C1
:10D5200020F03F001D303070B8F80400E08098F81B
:10D5300000100320022904D1317821F03F011B3172
:10D54000317094F84610090759D505ABB9F1000FB1
:10D5500013D0002102AA82E80B000720CDE90009C0
:10D56000BDF83400B8F80410C01E83B2002215982C
:10D5700000F0EFFD0028D1D101E0F11CEAE7B8F896
:10D580000400A6F80100BDF81400C01C04E198F8DE
:10D5900005108DF81C1098F80400012806D04FF4EF
:10D5A000007A02282CD00328B8D16CE12188B8F881
:10D5B000080011F40061ADF8201020D017281CD30A
:10D5C000B4F84010814218D3B4F84410172901D39D
:10D5D000814212D1317821F03F01C91C3170A6F887
:10D5E00001000321ADF83410A4F8440094F846007B
:10D5F00020F0020084F8460065E105257EE177E130
:10D60000208808F1080700F4FE60ADF8200010F053
:10D61000F00F1BD010F0C00F03D03888228B90423F
:10D62000EBD199B9B878C00710D0B9680720CDE917
:10D6300002B1CDF804B00090CDF810B0FB88BA88E4
:10D640003988159800F023FB0028D6D12398BDF81F
:10D650002010401C80294ED006DC10290DD0202936
:10D660000BD0402987D124E0B1F5807F6ED05145A1
:10D670007ED0B1F5806F97D1DEE0C80601D50820D5
:10D6800000E0102082460DA907AA0520CDE902215D
:10D690008DF83800ADF83CB0CDE9049608A938887B
:10D6A000CDE900015346072221461598FFF7B8F847
:10D6B000A8E09DF81C2001214FF00A0A002A9BD106
:10D6C00005ABB9F1000F00D00020CDE90210072012
:10D6D000CDE90009BDF834000493401E83B2218BCC
:10D6E0000022159800F035FD8DF81C000B203070DD
:10D6F000BDF8140020E09DF81C2001214FF00C0A19
:10D70000002A22D113ABB9F1000F00D00020CDE9DF
:10D7100002100720CDE900090493BDF83400228CE3
:10D72000401E83B2218B159800F013FD8DF81C006C
:10D730000D203070BDF84C00401CADF834000520C1
:10D740008DF83800208BADF83C00BCE03888218B88
:10D7500088427FF452AF9DF81C004FF0120A002857
:10D760001CD1606AA8B1B878C0073FF446AF00E0AA
:10D7700018E0BA680720CDE902B2CDF804B00090F5
:10D78000CDF810B0FB88BA88159800F080FA8DF8B3
:10D790001C00132030700120ADF8340093E000002D
:10D7A000600000203988208B8142D2D19DF81C0076
:10D7B0004FF0160A0028A06B08D0E0B34FF6FF70B8
:10D7C00000215F46ADF808B0019027E068B1B97854
:10D7D000C907BED1E18F0DAB0844821D03968DE8C9
:10D7E0000C0243888288018809E0B878C007BCD061
:10D7F000BA680DAB03968DE80C02BB88FA881598C1
:10D80000FFF7F7F905005ED0072D72D076E00190A2
:10D8100005AA02A92046FFF72DF90146E28FBDF8BF
:10D820000800824201D00029F1D0E08FA16B0844AA
:10D8300007800198E08746E09DF81C004FF0180A29
:10D8400040B1208BC8B13888208321461598FFF756
:10D850009AF938E004F118000090237E0122214655
:10D860001598FFF7A8F98DF81C000028EDD11920B4
:10D8700030700120ADF83400E7E705252146159802
:10D88000FFF781F93AE0208800F40070ADF820003D
:10D8900050452DD1A08FA0F57F41FE3901D006253E
:10D8A0002CE0D8F808004FF0160A48B1A063B8F889
:10D8B0000C10A1874FF6FF71E187A0F800B002E0DD
:10D8C0004FF6FF70A087BDF8200030F47F611AD0BA
:10D8D000782300220320159908F068FE98F80000CC
:10D8E00020712088BDF82010084320800EE000E061
:10D8F00007252088BDF8201088432080208810F458
:10D900007F6F1CD03AE02188814321809DF8380048
:10D9100020B10EA91598F9F78DFC05469DF81C005D
:10D920000028EBD086F801A001203070208B708099
:10D930009DF81C0030710520ADF83400DEE7A18EA3
:10D94000E1B118980DAB0088ADF834002398CDE90B
:10D950000304CDE90139206B0090E36A179A15980A
:10D96000FFF700FA054601208DF838000EA915983A
:10D97000F9F760FC00B10546A4F834B094F846000D
:10D9800040070AD52046FFF7A4F910F03E0F04D156
:10D9900014F8460F20F0040020701898BDF83410D9
:10D9A000018028469BE500B585B0032806D10220FA
:10D9B0008DF8000088B26946F9F73CFC05B000BD5F
:10D9C00010B5384C0B782268012B02D0022B2AD1DB
:10D9D00011E013780BB1052B01D1042313702368D8
:10D9E0008A889A802268CB88D38022680B89138129
:10D9F000498951810DE08B8893802268CB88D38040
:10DA000022680B8913814B8953818B899381096922
:10DA100011612168F9F70EFC2268002102281170BB
:10DA200003D0002800D0812010BD832010BD806B62
:10DA3000002800D0012070478178012909D1008891
:10DA4000B0F5205F03D042F60101884201D10020E9
:10DA5000704707207047F0B587B0002415460E4682
:10DA60000746ADF8184011E0059800882880059811
:10DA70000194811DCDE9024107210494009183881E
:10DA800042880188384600F002F930B905AA06A993
:10DA90003046FEF7EFFF0028E6D00A2800D100202C
:10DAA00007B0F0BD6000002010B58B7883B102781C
:10DAB0009A4205D10B885BB102E08B79091D4BB10D
:10DAC0008B789A42F9D1B0F801300C88A342F4D196
:10DAD000002010BD812010BD072826D012B1012AD8
:10DAE00027D103E0497801F0070102E04978C1F34A
:10DAF000C20105291DD2DFE801F00318080C12004D
:10DB00000AB1032070470220704704280DD250B19B
:10DB10000DE0052809D2801E022808D303E006285C
:10DB200003D0032803D005207047002070470F2042
:10DB3000704781207047C0B282060BD4000607D51B
:10DB4000FA48807A4143C01D01EBD00080B2704793
:10DB5000084670470020704770B513880B800B781B
:10DB60001C0625D5F14CA47A844204D843F0100059
:10DB70000870002070BD956800F0070605EBD00521
:10DB80002D78F54065F304130B701378D17803F00A
:10DB9000030341EA032140F20123B1FBF3F503FB48
:10DBA00015119268E41D00FB012000EBD40070BD4C
:10DBB000906870BD37B51446BDF804101180117817
:10DBC00041F0040111709DF804100A061ED5D74AD1
:10DBD000A368C1F30011927A824208D8FE2811D1BD
:10DBE000D21DD2084942184600F01BFC0AE003EBA4
:10DBF000D00200F00703012510789D40A84399400A
:10DC000008431070207820F0100020703EBD2DE9F0
:10DC1000F0410746C81C0E4620F00300B04202D077
:10DC20008620BDE8F081C14D002034462E60AF80D3
:10DC30002881AA72E8801AE0E988491CE9808106F7
:10DC400014D4E17800F0030041EA002040F2012101
:10DC5000B0FBF1F201FB12012068FFF76CFF29898C
:10DC6000084480B22881381A3044A0600C342078EF
:10DC70004107E1D40020D4E7AC4801220189C088E3
:10DC800000EB400002EB8000084480B270472DE9B1
:10DC9000FF4F89B01646DDE9168A0F46994623F4F0
:10DCA0004045084600F054FB040002D020784007AD
:10DCB00003D401200DB0BDE8F08F099804F05EFF99
:10DCC00002902078000606D59848817A0298814211
:10DCD00001D88720EEE7224601A90298FFF73CFF12
:10DCE000834600208DF80C004046B8F1070F1AD08B
:10DCF00001222146FFF7F0FE0028DBD12078400604
:10DD000011D502208DF80C00ADF81070BDF804009C
:10DD1000ADF81200ADF814601898ADF81650CDF8B3
:10DD20001CA0ADF818005FEA094004D500252E4676
:10DD3000A84601270CE02178E07801F0030140EAD1
:10DD4000012040F20121B0FBF1F2804601FB128775
:10DD50005FEA494009D5B84507D1A178207901F09B
:10DD6000030140EA0120B04201D3BE4201D907209D
:10DD7000A0E7A8191FFA80F9B94501D90D2099E744
:10DD80009DF80C0028B103A90998F9F751FA002869
:10DD900090D1B84507D1A0784FEA192161F301006D
:10DDA000A07084F804901A9800B10580199850EA80
:10DDB0000A0027D0199830B10BEB06002A461999B2
:10DDC00000F005FB0EE00BEB06085746189E09987D
:10DDD00005F041F82B46F61DB5B23946424600958E
:10DDE00004F02BFC224601A90298FFF7B5FE9DF82E
:10DDF0000400224620F010008DF80400DDE9011037
:10DE0000FFF7D8FE002055E72DE9FF4FDFF81C9102
:10DE1000824685B0B9F80610D9F8000001EB41013F
:10DE200000EB810440F20120B2FBF0F1174600FB49
:10DE30001175DDE9138B4E4629460698FFF77BFEE8
:10DE40000346FFF719FF1844B1880C30884202D905
:10DE5000842009B02FE70698C6B2300603D5B00675
:10DE600001D50620F5E7B9F80620521C92B2A9F8B0
:10DE70000620BBF1000F01D0ABF80020B00602D5A0
:10DE8000C4F808800AE0B9F808201A4492B2A9F848
:10DE90000820D9F80000891A0844A0602246FE2014
:10DEA0000699FFF787FEE77025712078390A61F33C
:10DEB00001002A0AA17840F0040062F30101A17078
:10DEC00020709AF802006071BAF80000E080002526
:10DED0002573300602D599F80A7000E00127B006D4
:10DEE00001D54FF000084E4600244FF007090FE01F
:10DEF000CDE902580195CDF800900495F1882046AF
:10DF0000129B089AFFF7C3FE0028A2D1641CE4B25A
:10DF1000BC42EDD300209CE700B5FFF7ADFE0349FE
:10DF20000C308A88904203D9842000BDFC05002073
:10DF3000CA88086802EB420300EB8300521C037896
:10DF400023F004030370CA80002101730846ECE744
:10DF50002DE9F047804600F0FBF9070005D00026C8
:10DF60004446F74D40F2012916E00120BDE8F08754
:10DF7000204600F0EDF90278C17802F0030241EA90
:10DF80000222B2FBF9F309FB13210068FFF7D3FD6E
:10DF90003044641C86B2A4B2E988601E8142E7DC8A
:10DFA000A8F10100E8802889801B288100203870B2
:10DFB000DCE710B5144631B1491E218004F0DEFDC6
:10DFC000A070002010BD012010BD70B50446DC48D3
:10DFD000C188036801E0401C20802088884207D265
:10DFE00000EB400213EB820202D015786D07F2D5E8
:10DFF00080B2884216D2AAB15079A072D08820810E
:10E000009178107901F0030140EA0120A081A07805
:10E01000E11CFFF7A1FD20612088401C2080E080EA
:10E02000002070BD0A2070BD0121018270472DE9DA
:10E03000FF4F85B04FF6FF798246A3F800904868FD
:10E040001E460D4680788DF8060048680088ADF8B9
:10E05000040000208DF80A00088A0C88A04200D332
:10E0600004462C8251E03878400708D4641C288A82
:10E07000A4B2401C288208F10100C0B246E0288A00
:10E08000401C2882781D6968FFF70EFDD8BB3188D7
:10E09000494501D1601E30803188A1EB08003080F5
:10E0A0006888A04238D3B878397900F0030041EA93
:10E0B000002801A9781DFFF7F7FC20BB29894945F5
:10E0C0002ED0002239460798FFF706FDD8B92989D6
:10E0D000414518D1E9680391B5F80AC0D7F808B0EE
:10E0E0005046CDF800C004F0B6FEDDF800C05A4638
:10E0F0000CF1070C1FFA8CFC43460399CDF800C0C5
:10E1000004F065FA60B1641CA4B200208046204689
:10E1100000F01EF90700A6D1641E2C820A2098E6A2
:10E1200074807879B071F888B0803978F87801F027
:10E13000030140EA01207081A6F80C80504604F0EB
:10E140001DFD3A4606F10801FFF706FD306100208B
:10E150007FE62DE9FF4F87B081461C469246DDF8E9
:10E1600060B0DDF85480089800F0F2F8050002D0A5
:10E170002878400702D401200BB09CE5484604F003
:10E18000FDFC2978090605D56D49897A814201D8B7
:10E190008720F1E7CAF309062A4601A9FFF7DCFC4C
:10E1A0000746149807281CD000222946FFF794FC44
:10E1B0000028E1D12878400613D501208DF8080009
:10E1C0000898ADF80C00BDF80400ADF80E00ADF8ED
:10E1D0001060ADF8124002A94846F9F729F8002866
:10E1E000CAD12978E87801F0030140EA0121AA7830
:10E1F000287902F0030240EA0220564507D0B1F523
:10E20000007F04D9611E814201DD0B20B4E7864204
:10E2100001D90720B0E7801B85B2A54200D9254669
:10E22000BBF1000F01D0ABF80050179818B1B91925
:10E230002A4600F0CCF8B8F1000F0DD03E44484615
:10E240004446169F04F019FE2146FF1DBCB232461B
:10E250002B46009404F025FA00208DE72DE9F041CB
:10E2600007461D461646084600F072F8040002D024
:10E270002078400701D40120D3E4384604F07EFC26
:10E280002178090605D52E49897A814201D887204F
:10E29000C7E422463146FFF75FFC65B12178E0789C
:10E2A00001F0030140EA0120B0F5007F01D8012010
:10E2B00000E0002028700020B3E42DE9F04107467B
:10E2C0001D461646084600F043F8040002D02078A8
:10E2D000400701D40120A4E4384604F04FFC217823
:10E2E000090605D51649897A814201D8872098E424
:10E2F00022463146FFF75EFCFF2D14D02178E078EE
:10E3000001F0030240EA022040F20122B0FBF2F3E6
:10E3100002FB130015B900F2012080B2E070000A80
:10E3200060F30101217000207BE410B50C4600F081
:10E330000FF810B10178490704D4012010BD000086
:10E34000FC050020C18821804079A0700020F5E7FD
:10E350000749CA88824209D340B1096800EB4000EE
:10E360006FF00B0202EB80000844704700207047FA
:10E37000FC05002070B504460D4621462B460AB91F
:10E38000002070BD01E0491C5B1C501E021E03D022
:10E3900008781E78B042F6D008781E78801BF0E727
:10E3A00030B50C4601462346051B954206D202E0D5
:10E3B000521E9D5C8D54002AFAD107E004E01D78BE
:10E3C0000D70491C5B1C521E002AF8D130BDF0B5FF
:10E3D0000E460146334680EA030404F00304B4B950
:10E3E00006E002B9F0BD13F8017B01F8017B521E73
:10E3F00001F00307002FF4D10C461D4602E080CD4A
:10E4000080C4121F042AFAD221462B4600BF04E022
:10E4100013F8014B01F8014B521E002AF8D100BF3E
:10E42000E0E7F0B50C460146E6B204E002B9F0BD03
:10E4300001F8016B521E01F00307002FF6D10B46C5
:10E44000E5B245EA052545EA054501E020C3121F6E
:10E45000042AFBD2194602E001F8016B521E002A81
:10E46000FAD100BFE3E710B508F0C9FBF4F730FAC2
:10E4700008F040FABDE8104008F008BB202834BF7F
:10E48000012000207047012303FA00F04FF0A04262
:10E49000002914BFC2F80C05C2F8080570474FF0F8
:10E4A000A041012202FA00F0C1F81805704770B5CA
:10E4B0000346002002466FF02F050EE09C5CA4F19D
:10E4C00030060A2E02D34FF0FF3070BD00EB800003
:10E4D00005EB4000521C2044D2B28A42EED370BDFC
:10E4E00030B50A230BE0B0FBF3F403FB1404B0FBDC
:10E4F000F3F08D183034521E05F8014CD2B2002AC8
:10E50000F1D130BD30B500234FF6FF7510E0040A9D
:10E5100044EA002084B2C85C6040C0F30314604049
:10E5200005EA00344440E0B25B1C84EA40109BB230
:10E530009342ECD330BD00002DE9F041FE4B0026A4
:10E54000012793F864501C7893F868C0B8B183F839
:10E550009140A3F8921083F8902083F88E70BCF15C
:10E56000000F0CBF83F8946083F89450F3488068E0
:10E57000008804F070FCBDE8F04104F005B94FF6E6
:10E58000FF7083F89140A3F8920083F8902083F8FD
:10E590008E70BCF1000F14BF83F8945083F8946020
:10E5A000BDE8F0812DE9F041E44D296891F89C2007
:10E5B0000024012A23D091F89620012A30D091F826
:10E5C0006C301422DC4E0127012B32D091F88E30B2
:10E5D000012B4FD091F8A620012A1CBF0020BDE8D6
:10E5E000F08144701F2200F8042B2222A731FFF78C
:10E5F000EEFE286880F8A6400120BDE8F081447056
:10E600001B220270D1F89D204260D1F8A1208260C7
:10E6100091F8A520027381F89C400120BDE8F081AB
:10E62000447007220270D1F89820426081F8964029
:10E63000E2E78046447000F8042B20226E31FFF799
:10E64000C6FE88F80870286880F86C4090F86E0064
:10E650000028D1D1B6F87000A6F89800A868417BD0
:10E6600086F89A1086F89670008804F0F4FB04F09F
:10E670009AF8C1E791F86C30012B0BD04470172247
:10E680000270D1F890204260B1F89420028181F8A4
:10E690008E40B1E78046447000F8042B20226E3192
:10E6A000FFF795FE88F80870286880F86C4090F8AD
:10E6B0006E000028A0D1CDE7A048006890F86C104B
:10E6C000002914BFB0F870004FF6FF70704770B5A6
:10E6D0009A4C06462068002808BFFFDF0025206806
:10E6E00045706660002808BFFFDF20684178002978
:10E6F0001CBFFFDF70BDCC220021FFF792FE206817
:10E70000FF2101707F2180F83710132141842821D7
:10E7100080F86910012180F85C1080F8615008F0E1
:10E72000CBFFBDE8704008F012B984490968097848
:10E7300081420CBF0120002070478048006890F89B
:10E740002200C0F3400070477C48006890F8220027
:10E7500000F0010070477948006890F82200C0F38B
:10E76000001070472DE9F0437448D0F800C09CF8C1
:10E770002400BCF82240C0F38001C0F340021144E1
:10E7800000F001000144C4F30010F0B1132C17D0C5
:10E7900009DC102C02BF6A4830F81100BDE8F08394
:10E7A000122C0DD008E0152C08BF664809D01D2C8E
:10E7B00004BF6548BDE8F083FFDF0020BDE8F083BB
:10E7C000624830F81100BDE8F0839CF85E209CF8A8
:10E7D0005F002E2600234FF47A774FF014084FF095
:10E7E0004009022A04BF4AF2D745B5FBF7F510D01D
:10E7F000012A04BF4AF22F75B5FBF7F510D04AF68F
:10E800002315B5FBF7F5082A08BF4E4613D0042A96
:10E8100018D01E46082A0ED0042A13D0022A49D046
:10E8200003F12806042A0FD0082A1CBF4FF019084C
:10E83000082204D00AE04FF0140806F5A8764FF03D
:10E84000400203E006F5A8764FF0100218FB0262C2
:10E8500012FB0152C1EB01113D4D01EB810105EBB2
:10E860008101114414F0010F4FF4C8724FF4BF75C9
:10E8700004BFC4F34006002E5DD0C4F3400601F58A
:10E88000A571EEB1082804BF174640260CD0042815
:10E8900004BF2F46102607D0022807BF03F1180730
:10E8A000042603F12807082606EB860808EB8616DF
:10E8B0003E441BE003F118064FF019080422C5E797
:10E8C000082804BF164640270CD0042804BF2E4653
:10E8D000102707D0022807BF03F11806042703F109
:10E8E0002806082707EB871706EB870631449C317B
:10E8F000082804BF164640270CD0042804BF2E4623
:10E90000102707D0022807BF03F11806042703F1D8
:10E9100028060827C7EBC70707EB470706EB47069C
:10E920003144983114F0010F27D0082808BF402047
:10E930001CD004280EE063E00806002068000020D8
:10E94000B8560200C056020090891300B05602006B
:10E95000D4FEFFFF04BF2A46102007D0022807BFBD
:10E9600003F11802042003F12802082000EB400301
:10E9700003EB0010104401443EE0082804BF144695
:10E9800040260CD0042804BF2C46102607D00228AD
:10E9900007BF03F11804042603F12804082606EB38
:10E9A0008616BCF840C004EB86042144BCF1EB0F92
:10E9B00022D944F255240CF10B0C0CFB04FC4FEA59
:10E9C0009C5C082807D0042802D0022805D008E063
:10E9D0002A46102008E0402006E003F11802042037
:10E9E00002E003F12802082000EB801002EB800017
:10E9F00000F5A5700CFB001101F26710BDE8F08373
:10EA000001F5A574082804BF164640210CD004283F
:10EA100004BF2E46102107D0022807BF03F11806B5
:10EA2000042103F12806082101EB8111BCF848C03C
:10EA300006EB81012144BCF1EB0FDDD944F25524F2
:10EA40000CF10B0C0CFB04FC4FEA9C5C0828C2D0B8
:10EA50000428BDD00228C4D1BFE7FE4840F271218E
:10EA60000068806A48437047FA48006890F83600AA
:10EA7000002818BF0120704710B5F74C207B0228F2
:10EA800018BF032808D1207D04F115010DF0EFFB1C
:10EA900008281CBF012010BD207B002816BF0228BB
:10EAA00000200120BDE8104009F006BAEA490873C9
:10EAB0007047E849096881F8300070472DE9F04750
:10EAC000E44C2168087B002816BF022800200120A2
:10EAD000487301F10E0109F0D9F92168087B022879
:10EAE00016BF03280122002281F82F204FF00800D2
:10EAF00081F82D00487B01F10E034FF001064FF025
:10EB00000007012804BF5B7913F0C00F0AD001F1A0
:10EB10000E03012804D1587900F0C000402801D02C
:10EB2000002000E0012081F82E00002A04BF91F8A7
:10EB3000220010F0040F07D0087D01F115010DF03F
:10EB400096FB216881F82D002068476006F0B0F937
:10EB50002168C14D4FF00009886095F82D000DF037
:10EB6000A2FB804695F82F00002818BFB8F1000FCF
:10EB700004D095F82D000DF05BF968B195F83000E0
:10EB800000281CBF95F82E0000281DD0697B05F1D8
:10EB90000E0001290ED012E06E734A4605F10E01F7
:10EBA000404609F0C9F995F82D1005F10E000DF059
:10EBB00071FC09E0407900F0C000402831D03946AE
:10EBC00005F10E0009F0F0F92068C77690F82200F0
:10EBD00010F0040F08BFBDE8F087002795F82D005E
:10EBE0000DF0DCF9050008BFBDE8F08710210EF03C
:10EBF000D8F9002818BFBDE8F08720683A4600F130
:10EC00001C01C676284609F097F9206800F11C011E
:10EC100060680EF0A7FC6068BDE8F04701210EF0C7
:10EC2000BCBC0DF074FC4A4605F10E0109F084F9F4
:10EC3000CAE7884A1268137B0370D2F80E00086096
:10EC4000508A8880704778B583490446814D407B5F
:10EC500008732A68207810706088ADF8000080B2D0
:10EC600000F00101C0F3400341EA4301C0F3800317
:10EC700041EA8301C0F3C00341EAC301C0F30013BA
:10EC800041EA0311C0F3401341EA4311C0F380107D
:10EC900041EA80105084E07D012808BF012603D09E
:10ECA000022814BFFFDF0226286880F85E60607EBD
:10ECB000012808BF012603D0022814BFFFDF022667
:10ECC000286880F85F60217B80F82410418C1D2922
:10ECD0000CBF002161688162617D80F83610A17BE4
:10ECE000002916BF0229002101210175D4F80F1057
:10ECF000C0F81510B4F81310A0F81910A17E90F800
:10ED00006B2061F3071280F86B20E17E012918BFA8
:10ED1000002180F83410002078BD4E480068408CF7
:10ED2000C0F3001131B1C0F38000002804BF1F20E0
:10ED3000704702E0C0F3400109B10020704710F0B5
:10ED4000010F14BFEE20FF20704742480068408C3E
:10ED5000C0F3001119B1C0F3800028B102E0C0F384
:10ED6000400008B100207047012070473949002257
:10ED700009684A664B8C1D2B0CBF81F8682081F80E
:10ED8000680070470023334A126882F85D30D1640E
:10ED9000A2F85000012082F85D0070472D4A002340
:10EDA000126882F85C30A2F858000120516582F8A0
:10EDB0005C0070472749096881F83500704725498C
:10EDC000096881F8610070472248006890F9610085
:10EDD00070472048006890F82200C0F34010704748
:10EDE0001C48006890F82200C0F3C0007047012062
:10EDF00070471848006890F85F00704770B508F0D9
:10EE00003CFC08F01BFC08F0DCFA08F089FB114C14
:10EE10002068416E491C416690F83300002530B1EE
:10EE200008F04AFC07F093FD206880F83350206812
:10EE3000457090F8381021B1BDE87040042009F009
:10EE4000C0BC90F8681009B3406E81421ED80420FF
:10EE500004E00000680000200806002009F0B1FC72
:10EE6000206890F8220010F0010F07D0A06843221C
:10EE70000188BDE870400120FFF75EBBBDE870402F
:10EE800043224FF6FF710020FFF756BBBDE87040EC
:10EE9000002009F096BC2DE9F04782B00F4682466B
:10EEA000FE4E4FF000093068458C15F0030F10D06E
:10EEB00015F0010F05F0020005D0002808BF4FF043
:10EEC000010906D004E0002818BF4FF0020900D164
:10EED000FFDF4FF00008444615F0010F05F0020077
:10EEE0000DD080B915F0040F0DD048F00800002FA8
:10EEF0001CBF40F0010040F0020438D06EE010B1B9
:10EF000015F0040F0DD015F0070F10D015F0010FFC
:10EF100005F002002ED0002808BF15F0040F1FD006
:10EF200035E0002F18BF48F0090457D12CE02FB16D
:10EF300048F0080415F0200F4CD04FE0306805F081
:10EF40002001B0F84800084308BF48F0010445D04C
:10EF500048F0180415F0200F08BF44F001043DE00C
:10EF600048F00800002F18BF40F0010436D140F0EF
:10EF7000100433E0002818BF15F0040F07D0002F4D
:10EF800018BF48F00B0429D148F0180426E015F00A
:10EF9000030F22D115F0040F1FD03FB128F002005B
:10EFA00040F0080415F0200F14D017E0306805F089
:10EFB0002001B0F84800084308BF48F003040DD012
:10EFC00048F0180015F0200F08BF40F0010040F095
:10EFD000020403E024F0010400E0FFDF15F0400F1D
:10EFE00012D07FB93068B0F84810002904BF408CB7
:10EFF00010F0010F06D110F0020F04BF10F0200F27
:10F0000015F0010F44F040047068A0F8008001780A
:10F0100021F0200101704FF007010EF06FFA494610
:10F0200070680EF062FC214670680EF06AFC14F005
:10F03000010F0CD04FF006034FF0000298497068A2
:10F040000EF039FC3068417B70680EF099FA14F0CC
:10F05000020F18D0D6E90010BAF1000F4FF00603E6
:10F060004FF0010207D01C310EF025FC0121706821
:10F070000EF093FA07E015310EF01DFC3068017DAB
:10F0800070680EF08AFA14F0040F18BFFFDF14F056
:10F09000080F19D0CDF800803068BDF80020022399
:10F0A000B0F86A1061F30B02ADF8002090F86B0025
:10F0B000032201099DF8010061F307108DF801009A
:10F0C000694670680EF0F7FB012F62D13068B0F826
:10F0D0004810E1B390F82200C0F34000B8BB70685C
:10F0E0000EF0FFFB401CC7B23068C7F1FF05B0F857
:10F0F0004820B0F85A10511AA942B8BF0D46AA428A
:10F100003BD990F8220010F0010F36D144F01004E2
:10F11000214670680EF0F5FBF81CC0B2ED1E2844C5
:10F1200082B23068B0F86A10436EC1F30B0151FA35
:10F1300083F190F860305B4F1944BC460023E1FB3B
:10F1400007C31B096FF0240C03FB0C1100E020E047
:10F1500080F8601090F85F00012101F007F900903D
:10F16000BDF800009DF80210032340EA0140019021
:10F17000042201A970680EF09EFB3068AAB2416CAF
:10F1800070680EF0ECFB3068B0F85A102944A0F813
:10F190005A1014F0400F06D0D6E9001001230622C1
:10F1A00061310EF088FB14F0200F18BFFFDF002044
:10F1B000002818BFFFDF02B0BDE8F0872DE9F0435B
:10F1C000364C89B02068002808BFFFDF20684178EE
:10F1D000002936D10178FF2933D0002680F831602C
:10F1E000A0F85A60867080F83860304608F0B8F9A8
:10F1F0002D4802AD00F1240191E80E1085E80E10B3
:10F20000D0E90D10CDE9061002A808F097F907F033
:10F21000F4FD206890F9610007F0C4FE234807F070
:10F22000C7FE234808F076F9606808F09CF920686A
:10F2300090F8240010F0010F07D0252007F0C0FE41
:10F240000AE009B00C20BDE8F08310F0020F18BFEF
:10F25000262077D007F0B4FE206890F85E102520B5
:10F2600007F097FD206880F82C6008F073F920689B
:10F2700090F85E10002007F09FFF0F21052007F097
:10F2800065FE206890F82E10002901BF90F82F101D
:10F29000002990F8220010F0040F0BE06800002015
:10F2A0001606002053E4B36EA4560200AC560200CA
:10F2B000A956020075D005F0FBFD054620682946D9
:10F2C000806806F0E4FADFF82C84074690FBF8F03B
:10F2D00008FB10704142284605F0D1FA2168886089
:10F2E00097FBF8F04A68104448600CF0BDFF0146F7
:10F2F0002068426891426FD8C0E90165FE4D4FF029
:10F30000010895F82D000CF0CEFF814695F82F00EE
:10F310000127002818BFB9F1000F04D095F82D007F
:10F320000CF086FDA8B195F8300000281CBF95F8B8
:10F330002E00002825D0687B05F10E01012816D08B
:10F340001AE0FFE710F0040F14BF2720FFDF81D180
:10F3500082E73A466F7305F10E01484608F0ECFD6E
:10F3600095F82D1005F10E000DF094F809E048799C
:10F3700000F0C000402815D0414605F10E0008F00D
:10F3800013FE206890F8220010F0040F24D095F8A6
:10F390002D000CF003FE05001ED010210DF001FE23
:10F3A00040B119E00DF0B3F83A4605F10E0108F04E
:10F3B000C3FDE6E720683A4600F11C01C7762846FF
:10F3C00008F0BAFD206800F11C0160680EF0CAF870
:10F3D000012160680EF0E1F82068417B0E3007F0F3
:10F3E00097FD206890F85C1061B3B0F85810A0F851
:10F3F0004810416D416490F82210C1F30011F1B939
:10F40000B0F86A000221C0F30B05ADF80050684661
:10F4100006F070FE28B1BDF80000C0F30B00A84252
:10F4200004D1BDF80000401CADF800002168BDF813
:10F430000000B1F86A2060F30B02A1F86A2020688E
:10F4400080F85C60206890F85D1039B1B0F8501019
:10F45000A0F84010C16CC16380F85D60B0F86A101C
:10F46000426EC1F30B0151FA82F190F86020DFF88F
:10F470008CC2114463460022E1FB0C3212096FF08A
:10F48000240302FB031180F860100CF070FF0321CD
:10F4900060680CF0EFFF216881F8330009B00020AC
:10F4A000BDE8F0839649886070472DE9F043944C9D
:10F4B00083B0226892F831303BB1508C1D2808BFD0
:10F4C000FFDF03B0BDE8F04398E401260027F1B167
:10F4D000054692F8600007F073FD206890F85F1011
:10F4E000FF2007F056FC20684FF4A57190F85F20CC
:10F4F000002007F029FF206890F8221011F0030F78
:10F5000000F02C81002D00F0238100F027B992F843
:10F5100022108046D07EC1F30011002956D0054646
:10F5200060680780017821F020010170518C132957
:10F5300037D01FDC102908BF022144D0122908BF90
:10F54000062140D0FFDF6C4D606805F10E010DF023
:10F55000FBFF697B60680EF013F82068418C1D2961
:10F5600018BF152963D0B0F84820416C60680EF0D0
:10F5700020F85CE0152918BF1D29E3D14FF00101E7
:10F580000DF0BCFF6068017841F020010170216836
:10F5900085B11C310DF0E6FF012160680DF0FDFF23
:10F5A000D1E700210DF0AAFF6068017841F0200149
:10F5B0000170C8E715310DF0D5FF2068017D606846
:10F5C0000DF0EBFFBFE70DF099FFBCE70021FFF75F
:10F5D00062FC6068C17811F03F0F28D0017911F00A
:10F5E000100F24D00DF088FF2368024693F82410F2
:10F5F000C1F38000C1F3400C604401F001010844F4
:10F6000093F82C10C1F3800CC1F34005AC4401F019
:10F6100001016144401AC1B293F85E0000F0A6FEF9
:10F62000009003230422694660680EF044F92068C4
:10F63000002590F8241090F82C0021EA000212F026
:10F64000010F18BF01250ED111F0020F04D010F0E8
:10F65000020F08BF022506D011F0040F03D010F0EE
:10F66000040F08BF0425B8F1000F2BD0012D1BD0CB
:10F67000022D08BF26201BD0042D14BFFFDF27203A
:10F6800016D0206890F85E10252007F082FB2068D5
:10F6900090F82210C1F3001169B101224FF4967164
:10F6A000002007F051FE0DE0252007F089FCE8E777
:10F6B00007F086FCE5E790F85E204FF49671002095
:10F6C00007F042FE206890F82C10294380F82C1097
:10F6D00090F8242032EA01011CD04670418C132995
:10F6E0002BD026DC102904BF03B0BDE8F08312291B
:10F6F00023D007E040420F000806002053E4B36E19
:10F7000068000020C1F30010002818BFFFDF03B01D
:10F71000BDE8F083418C1D2908BF80F82C70DCD037
:10F72000C1F30011002914BF80F8316080F83170F6
:10F73000D3E7152918BF1D29DBD190F85E2003B04F
:10F740004FF00101BDE8F043084607F0F2BF00BFEB
:10F7500090F85F200121084607F0EBFF2168002D9B
:10F76000C87E7CD04A8C3D46C2F34000002808BFCA
:10F7700047F0080512F0400F18BF45F0400500287B
:10F7800019BFD1F83C90B1F84080D1F84490B1F85D
:10F7900048806068072107800DF0B0FE0021606896
:10F7A0000EF0A3F8294660680EF0ABF815F0080FCC
:10F7B00017D02068BDF800100223B0F86A2062F369
:10F7C0000B01ADF8001090F86B00032201099DF8C1
:10F7D000010061F307108DF80100694660680EF0C2
:10F7E0006AF860680DF046FF2168C0F1FE00B1F8CC
:10F7F0005A20A8EB02018142A8BF0146CFB2D0191E
:10F80000404544D245F0100160680EF07AF8606817
:10F810000DF030FF2168C0F1FE00B1F85A10A8EBDE
:10F8200001018142A8BF0146CFB260680EF059F8CD
:10F830003844421C2068B0F86A10436EC1F30B01D3
:10F8400051FA83F190F86030F94D1944AC46002329
:10F85000E1FB05C34FEA131C6FF0240300E03CE01A
:10F860000CFB031180F8601090F85F00012100F09C
:10F870007DFD0090BDF800009DF80210032340EAD2
:10F8800001400190042201A960680EF014F821687B
:10F8900091F8220010F0400F05D0012306226131BB
:10F8A00060680EF008F820683A46B0F85A0000EB9D
:10F8B000090160680EF053F82068B0F85A10394416
:10F8C000A0F85A1008F013FA002818BFFFDF2068CC
:10F8D0004670867003B0BDE8F0830121FFF7DBFAC4
:10F8E000F0E7D44810B50068417841B90078FF28A6
:10F8F00005D000210846FFF7D8FD002010BD07F015
:10F90000BCFE07F09BFE07F05CFD07F009FE0C2033
:10F9100010BD2DE9F041C74D0446174628680E4634
:10F9200090F86C00002818BFFFDF2868002F80F8CF
:10F930006E7018BFBDE8F0812188A0F87010618852
:10F94000A0F88610A188A0F88810E188A0F88A1095
:10F9500094F88C1180F88C1090F82F10002749B182
:10F96000427B00F10E01012A04D1497901F0C00166
:10F97000402935D090F8301041B1427B00F10E01A2
:10F98000012A04BF497911F0C00F29D000F17A0093
:10F99000F3F732FB6868FF2E0178C1F380116176BE
:10F9A000D0F80310C4F81A10B0F80700E0832868F4
:10F9B0001ED0C0F88010E18BA0F8841000F1740212
:10F9C000511E30460CF078FC002808BFFFDF286885
:10F9D00090F8731041F0020180F87310BDE8F081D7
:10F9E000D0F80E10C0F87A10418AA0F87E10D1E746
:10F9F000C0F88070A0F88470617E80F87310D4F82D
:10FA00001A104167E18BA0F87810BDE8F08170B55D
:10FA1000884C0125206890F82200C0F3C00038B15E
:10FA20003C22FF21A068FFF774FF206880F86C502B
:10FA3000206890F8220010F0010F1CBFA068018818
:10FA40004FF03C0212BF01204FF6FF710020FEF77D
:10FA500073FD206880F8385070BD7649096881F8D8
:10FA6000320070472DE9F041002608F076FE0028AC
:10FA700000F0F7806F4C20684178002701250129AC
:10FA800006D0022901D003297BD0FFDFBDE8F08139
:10FA9000817802270029418C37D0C1F34002002A27
:10FAA00008BF11F0010F6DD090F85F204FF00101F9
:10FAB0004FF0000007F03DFE216891F82200C0F3EE
:10FAC0004000002814BF0C20222091F85F1007F09E
:10FAD00060F92068477090F8330020B106F023FFEA
:10FAE000402007F0D6FD206890F83400002818BFA9
:10FAF00007F0FCFD0021962007F064FD08F0EEF809
:10FB0000002818BFFFDFBDE8F081C1F3001282B109
:10FB100010293ED090F8330020B106F004FF4020B9
:10FB200007F0B7FD206890F8221011F0040F35D0CF
:10FB300042E090F8242090F82C309A4229D1B0F875
:10FB40004800002808BF11F0010F05D111F0020F85
:10FB500008BF11F0200F6FD04FF001014FF00000EF
:10FB6000FFF7A3FC2068418C11F0010F04BFC1F323
:10FB7000400100290AD1B0F85A10B0F8482091424B
:10FB800001E032E026E018BFBDE8F08180F8315096
:10FB9000B9E7BDE8F0410021012086E490F8361075
:10FBA000012914BF0329102646F00E0190F85E20AB
:10FBB0004FF0000007F0BDFD206890F834000028E9
:10FBC00018BF07F093FD0021962007F0FBFC20688A
:10FBD000477098E7B0F85A10B0F84800814240D01A
:10FBE000BDE8F041012108465FE48178D9B1418C3C
:10FBF00011F0010F21D080F86C5090F86E20B0F811
:10FC000070100120FEF798FC2068477007F035FD62
:10FC100007F014FD07F0D5FB07F082FCBDE8F041CA
:10FC2000032008F0CEBD8178BDE8F04101203CE41E
:10FC300053E4B36E6800002013E011F0020F08BF18
:10FC4000FFDF3FF460AFB0F85A10B0F840008142D7
:10FC500007D001210846FFF728FC216803204870DF
:10FC600051E7BDE8F041FFF7C9B8FFF7C7B810B5D5
:10FC7000FE4C206890F8341049B1373007F041FD50
:10FC800018B921687F2081F8370007F025FD20682A
:10FC900090F8330018B107F00FFD06F058FE08F099
:10FCA0005CFDA8B1206890F82210C1F3001179B171
:10FCB0004078022818BFFFDF00210120FFF7F5FB85
:10FCC0002068417800291EBF40780128FFDF10BD61
:10FCD000BDE81040FFF792B82DE9F047E34C0F461E
:10FCE00080462168B8F1030F488C08BFC0F3400577
:10FCF00008D000F0010591F83200002818BF4FF03D
:10FD0000010901D14FF0000907F04EF90646B8F19C
:10FD1000030F0CBF4FF002084FF0010835EA09004D
:10FD200008BFBDE8F087206890F8330068B10CF098
:10FD300001FB38700146FF2807D06068C01C0CF03A
:10FD4000D2FA38780CF003FB064360680178C1F3FF
:10FD5000801221680B7D9A4208D10622C01C153101
:10FD6000FEF708FB002808BF012000D000203978EA
:10FD7000FF2906D0C8B9206890F82D00884216D116
:10FD800013E0A0B1616811F8030BC0F380100CF010
:10FD90006EFA05460CF0CEFB38B128460CF0FEF8A2
:10FDA00018B110210DF0FDF808B1012000E000208D
:10FDB000216891F8221011F0040F01D0F0B11AE07F
:10FDC000CEB9AB4890F83600002818BF404515D191
:10FDD000616811F8030BC0F380100CF048FA044678
:10FDE0000CF0A8FB38B120460CF0D8F818B110215F
:10FDF0000DF0D7F810B10120BDE8F0870020BDE874
:10FE0000F0872DE9F04F994D044683B0286800260D
:10FE10004078022818BFFFDF28684FF07F0A90F86B
:10FE2000341049B1373007F06CFC002804BF286853
:10FE300080F837A007F050FC68680DF081FB804621
:10FE4000002C00F0418207F07DF8002800F03C8291
:10FE5000012400274FF0FF09B8F1050F1ED1686893
:10FE600090F8240000F01F00102817D9286890F897
:10FE7000350098B18DF8009069460520FFF72CFFFA
:10FE8000002800F02182286880F8A64069682222B4
:10FE9000A730C91CFEF79BFA00F016BA68680DF08F
:10FEA000DAFC002800F010824046DFF8C4814FF0F1
:10FEB000030B062880F01A82DFE800F0FCFCFC034C
:10FEC000FCFB8DF8009069460320FFF705FF002832
:10FED00000F0F180296891F8340010B191F89C008D
:10FEE000D8B12868817801294DD06868042107803D
:10FEF0000DF004FB08F10E0168680DF025FB98F881
:10FF00000D1068680DF03CFB2868B0F84020C16B0C
:10FF100068680DF072FB00F05FB99DF8000081F891
:10FF20009C400A7881F89D20FF280FD001F19F02A4
:10FF30009E310CF0C1F9002808BFFFDF286890F857
:10FF40009E1041F0020180F89E100DE06868027872
:10FF5000C2F3801281F89E20D0F80320C1F89F20C0
:10FF6000B0F80700A1F8A300286800F1A50490F8F4
:10FF700037007F2808BFFFDF286890F8371021700E
:10FF800080F837A0ADE790F822000721C0F3801970
:10FF900038480479686869F3861407800DF0AEFA72
:10FFA000002168680DF0A1FC214668680DF0A9FCED
:10FFB0000623002208F10E0168680DF07CFC286819
:10FFC000417B68680DF0DCFA68680DF053FB296826
:10FFD000B1F84020C0F1FE018A42B8BF1146CFB24D
:10FFE000BA423CD9F81EC7B244F0100A51466868BC
:10FFF0000DF087FC68680DF074FC384400F10108CE
:020000040001F9
:100000002868B0F86A10426EC1F30B0151FA82F110
:1000100090F86020184C0A44A4460023E2FB04C375
:1000200019096FF0240301FB032180F8601090F898
:100030005F004246012100F099F90190BDF80400EB
:100040009DF80610032340EA01400290042202A911
:1000500068680DF030FC514668680DF052FCB9F14B
:10006000000F0FD0D5E90010012307E06800002041
:1000700008060020A456020053E4B36E0622613144
:100080000DF019FC28683A46C16B68680DF067FCF2
:100090002868A0F85A70B0F840108F420CBF0121B8
:1000A000002180F8311007F022FE002818BFFFDF82
:1000B00092E007E01AE128688078002840F0068185
:1000C00000F002B98DF8009068680178C1F38019DA
:1000D000D0F803100191B0F80700ADF808006946A8
:1000E0000520FFF7F9FD0028286879D081780029DC
:1000F00078D090F85FA0D5E90104D0F80F10C4F8CB
:100100000E10B0F813106182417D2175817D6175FB
:10011000B0F81710E182B0F819106180B0F81B1028
:10012000A180B0F81D10E18000F11F0104F108006A
:1001300015F0A1F9686890F8241001F01F012176EC
:1001400090F824000021400984F88C0184F864A010
:1001500084F865A004F130000DF00CFE2868002240
:1001600090F8691084F8661090F8610084F86700D0
:100170009DF80010A868FFF7CCFB022008F021FBD7
:10018000A9480DF1040A08210468686807800DF089
:10019000B5F9002168680DF0A8FB214668680DF0EC
:1001A000B0FB0623002208F10E0168680DF083FB06
:1001B0002868417B68680DF0E3F9494668680DF0EE
:1001C000ECF906230122514668680DF074FB07F034
:1001D0008EFD002818BFFFDF286880F801B077E0A7
:1001E0006DE0FFE76868D5F808804FF001090278F4
:1001F00098F80D10C2F34012114088F80D10D0F895
:100200000F10C8F80E10B0F81310A8F81210417DA6
:1002100088F81410817D88F81510B0F81710A8F828
:100220001610B0F81910A8F80210B0F81B10A8F8B2
:100230000410B0F81D10A8F8061000F11F0108F115
:10024000080015F018F9686890F8241001F01F01F3
:1002500088F8181090F824000021400988F88C01D3
:1002600088F8649088F8659008F130000DF082FD00
:100270002868002290F8691088F8661090F86100EC
:1002800088F867009DF80010A868FFF742FB28680F
:1002900080F86C4090F86E20B0F870100120FEF7E6
:1002A0004BF92868477007F0E8F907F0C7F907F03D
:1002B00088F807F035F9012008F083FA08E090F893
:1002C0002200C0F3001008B1012601E0FEF796FD00
:1002D000286890F8330018B107F0EEF906F037FB04
:1002E00066B100210120FFF7E0F810E0286890F8DF
:1002F0002200C0F300100028E8D0E5E728688178E4
:10030000012904D190F85F10FF2006F042FD286813
:100310004178002919BF4178012903B0BDE8F08F69
:100320004078032818BFFFDF03B0BDE8F08F70B539
:100330003E4C06460D462068807858B106F090FC89
:1003400021680346304691F85F202946BDE8704099
:1003500008F0E2BF06F084FC21680346304691F8BD
:100360005E202946BDE8704008F0D6BF78B50C463F
:1003700000210091082804BF4FF4C87040210DD01F
:10038000042804BF4FF4BF70102107D0022807BF14
:1003900001F11800042101F128000821521D02FB7F
:1003A000010622489DF80010006890F8602062F372
:1003B000050141F040058DF8005090F85F000128DC
:1003C00004BF9DF8020020F0E0002AD0022818BFE8
:1003D000FFDF21D025F080008DF80000C4EB041071
:1003E00000EB80001E2101EB800006FB0404104896
:1003F000844228BFFFDF0F48A0FB0410BDF80110A6
:10040000000960F30C01ADF80110BDF800009DF883
:10041000021040EA014078BD9DF8020020F0E000A3
:1004200020308DF80200D5E7A456020068000020B5
:10043000C4BF0300898888880178406829B190F892
:100440002C1190F88C0038B901E001F0C5BC19B14D
:10045000042901D0012070470020704770B50C4678
:100460000546062102F0C4FB606008B1002006E0EA
:100470000721284602F0BCFB606018B10120207003
:10048000002070BD022070BD2DE9FC470C460646D9
:100490006946FFF7E3FF00287DD19DF8000050B1C9
:1004A000FEF70AF9B0427CD0214630460AF0DAF86D
:1004B000002873D12DE00DF085FDB04271D02146AA
:1004C000304612F05DFD002868D1019D95F8F000DE
:1004D00022E0012000E00020804695F839004FF02E
:1004E000010A4FF00009F0B195F83A0080071AD5DB
:1004F00084F8019084F800A084F80490E68095F8D0
:100500003B102172A98F6181E98FA18185F8399013
:1005100044E0019D95F82C0170350028DBD1287F3F
:100520000028D8D0D5E7304602F0A7FC070000D15C
:10053000FFDF384601F0B5FE40B184F801900F218D
:100540002170E680208184F804A027E0304602F084
:1005500082FC070000D1FFDFB8F1000F21D0384640
:1005600001F0F7FEB8B19DF8000038B90198D0F855
:1005700018014188B14201D180F80090304607F05F
:1005800003FC84F801900C21217084F80490E6802B
:10059000697F217200E004E085F81C900120BDE82D
:1005A000FC870020FBE71CB56946FFF757FF00B149
:1005B000FFDF684601F01CFCFE4900208968A1F8B5
:1005C000F2001CBD2DE9FC4104460E46062002F057
:1005D000B7FA0546072002F0B3FA2844C7B200254F
:1005E000A8463E4417E02088401C80B22080B042DC
:1005F00002D34046A4F8008080B2B84204D3B0428F
:1006000002D20020BDE8FC816946FFF727FF0028E1
:10061000F8D06D1CEDB2AE42E5D84FF6FF702080E9
:100620001220EFE738B54FF6FF70ADF800000DE08F
:100630000621BDF8000002F0EDFA04460721BDF8DE
:10064000000002F0E7FA0CB100B1FFDF00216846BC
:10065000FFF7B8FF0028EBD038BD70B507F002FCFB
:100660000BF0EFFBD44C4FF6FF7600252683668314
:10067000D2A0257001680079A4F14002657042F8AB
:10068000421FA11C1071601C12F097FD1B202081DD
:100690004FF4A4716181A081E18103212177617709
:1006A0002174042262746082A082A4F13E00E1827F
:1006B00005704680BF480C300570A4F1100005702D
:1006C000468084F8205070BD70B5BA4C16460D4671
:1006D0006060217007F03EFBFFF7A4FFFFF7BDFF4E
:1006E000207810F0CCFAB7480DF0B2FD21786068A0
:1006F00012F008FD20780AF0F7FD284608F0E4FB28
:10070000B048FDF7E4FF217860680AF085F83146CB
:10071000207812F0B5FFBDE870400BF092BB10B529
:1007200001240AB1002010BD21B1012903D0002409
:10073000204610BD02210DF04FF9F9E710B50378FE
:100740000446002B406813460A46014608D00120A3
:100750000CF0BBFE6168496A884203D9012010BDD4
:100760000020F5E7002010BD887800B90320C97883
:1007700001B90321107019700020704730B587B09F
:10078000044600886946FFF769FE002806D1A08864
:1007900030B1012804D0022802D0122007B030BDA9
:1007A00004AB03AA21466846FFF7DEFF0400F5D13B
:1007B0009DF80010012000250029019906D081F83C
:1007C000C501019991F8101291BB29E081F82F0120
:1007D000019991F8561139B9019991F82E1119B969
:1007E000019991F8971009B13A2415E006950199FD
:1007F00081F82E01019A9DF80C0082F83001019BCE
:100800009DF8102083F831218DF818008DF81920FB
:1008100006AA00200CF069FD019880F82F5122E013
:10082000019991F8C41119B9019991F8971009B17A
:100830003A2415E00695019981F8C401019A9DF8C2
:100840000C0082F8C601019B9DF8102083F8C72197
:100850008DF818008DF8192006AA01200CF045FD2E
:10086000019880F8C551204698E710B5044600204D
:10087000A17801B90120E2780AB940F0020001F044
:10088000C6FA002803D12046BDE8104076E710BD27
:1008900070B50D4604460189002380880CF01AFDCE
:1008A000696A81421DD2401A401CA1884008091A79
:1008B0008AB2A2802189081A2081668895F864107E
:1008C00010460CF0E5FC864200D230466080E68897
:1008D00095F8651020890CF0DBFC864200D230468A
:1008E000E08070BDF0B585B00D46064603A9FFF760
:1008F000B5FD00282DD19DF80C0060B300220499AD
:10090000FB20B1F84E30FB2B00D30346B1F850402A
:10091000FB20FB2C00D30446DFF8ACC09CE8811020
:1009200000900197CDF808C0ADF80230ADF8064050
:100930006846FFF7ADFF6E80BDF80400E880BDF8A3
:1009400008006881BDF80200A880BDF80600288173
:10095000002005B0F0BD0122D1E72DE9F04186B0BD
:10096000044600886946FFF779FD00287ED1218979
:10097000E08801F066FA00287FD1A188608801F044
:1009800060FA002879D12189E08801F050FA002826
:1009900073D1A188608801F04AFA07006DD12088E0
:1009A00002A9FFF79FFF00B1FFDFBDF810106288BA
:1009B00009200BE07400002014080020FFFFFFFF57
:1009C0001F000000D4060020E0560200914254D3DC
:1009D000BDF80C10E28891424FD3BDF81210BDF85B
:1009E0000E2023891144A2881A44914245D39DF8D0
:1009F0000010019D4FF00008012640F6480041B16B
:100A000085F8BB61019991F8FC1105F5DD7541B9D7
:100A10001AE085F82561019991F84A1105F592755A
:100A200009B13A2726E0E18869806188E980218957
:100A3000814200D30146A980A188814200D20846A4
:100A40002881012201990FE0E18869806188E980AD
:100A50002189814200D30146A980A188814200D228
:100A60000846288101990022284600E005E0FFF7AA
:100A70000FFF2E7085F80180384606B0BDE8F08182
:100A80006BE770B504460DF053FAB0B12078182822
:100A900011D1207901280ED1E088062102F0A8F8B2
:100AA000040008D0208807F06FF92088062102F0A2
:100AB000B1F800B1FFDF012070BDF94D28780028A2
:100AC000FAD0002666701420207020223146201DA6
:100AD000FDF7A7FC022020712E70ECE710B504464C
:100AE000FDF760FD002813D0207817280FD120795A
:100AF00068B1E088072102F07BF840B1008807F078
:100B000043F9E088072102F085F800B1FFDF0120FA
:100B100010BD2DE9F0475FEA000800D1FFDFE04893
:100B200002211A308146FFF74DFD00B1FFDFDC4C9A
:100B30000620678B02F004F80546072002F000F853
:100B40002844C5B2681CC6B2608BB04203D140468F
:100B5000FFF7C4FF58B9608BA84203D14046FFF7A6
:100B600090FF20B9608B4146FFF78EFC38B14046BC
:100B700001F075F90028E7D10120BDE8F0870221D6
:100B80004846FFF71FFD10B9608BB842DCD14046E4
:100B9000BDE8F04712F0B9BD10B501F0C5F808B1D5
:100BA0000C2010BD0BF0A1F9002010BD10B50446BB
:100BB000007818B1012801D0122010BD01F0C5F84D
:100BC00020B10BF043FB08B10C2010BD207801F0E0
:100BD00085F8E21D04F11703611CBDE810400BF01D
:100BE0002ABA10B5044601F09FF808B10C2010BDD8
:100BF000207828B1012803D0FF280BD0122010BD87
:100C000001F06CF8611C0BF030F908B1002010BD48
:100C1000072010BD01200BF062F9F7E710B50BF0CB
:100C200018FB08B1002010BD302010BD10B50446DF
:100C300001F08BF808B10C2010BD20460BF003FB2F
:100C4000002010BD10B501F080F820B10BF0FEFAC5
:100C500008B10C2010BD0BF053FA002010BDFF218D
:100C600081704FF6FF7181808E4949680A788271E0
:100C70008A880281498841810121417000207047A2
:100C80001CB5002412F1080F15D00CDC12F1280F4E
:100C900011D012F1140F0ED012F1100F0BD012F16F
:100CA0000C0F0ED107E012F1040F04D01AB1032A81
:100CB00001D0042A05D1012806D0022808D0032833
:100CC0000AD0122420461CBD1046FEF778F8F9E73A
:100CD00010460DF0B8FAF5E7084614466946FFF7E6
:100CE000BDFB08B10224EDE79DF80000019880F8F3
:100CF00067400024E6E710B5134601220CF08EF998
:100D0000002010BD10B5044610F07EFD052804D06B
:100D100020460FF0A3FF002010BD0C2010BD10B521
:100D2000044601F012F808B10C2010BD2146002045
:100D300007F099F8002010BD10B5044610F01DF81A
:100D400050B108F017FB38B1207808F0C9F82078C6
:100D50000DF03AFD002010BD0C2010BD10B504466A
:100D600000F0F3FF08B10C2010BD2146012007F070
:100D70007AF8002010BD38B504464FF6FF70ADF884
:100D80000000A079E179884216D02079FDF776FB42
:100D900090B16079FDF772FB70B10022A079114625
:100DA00013F0AEF840B90022E079114613F0A8F82C
:100DB00010B9207A072801D9122038BD08F0E7FAC7
:100DC00060B910F021FD48B900216846FFF7FAFB31
:100DD00020B1204605F0B6FF002038BD0C2038BDFC
:100DE0002DE9FC41817805461A2925D00EDC16290B
:100DF0002ED2DFE801F02D2D2D2D2D212D2D2D2D85
:100E00002D2D2D2D2D2D2D2D2D2121212A291FD0A8
:100E10000BDCA1F11E010C291AD2DFE801F019192F
:100E20001919191919191919190D3A3904290FD253
:100E3000DFE801F00E020E022888B0F5706F07D2CD
:100E400001276946FFF70AFB20B10220BDE8FC81BB
:100E50001220FBE79DF8000000F047FF019C10B155
:100E600004F58A7401E004F5C8749DF8000000F0F0
:100E70003CFF019E10B106F2151601E006F2911634
:100E80006846FFF7D9FA08B1207808B10C20DDE7F1
:100E90002770A8783070684600F0AAFF0020D5E7D8
:100EA00014080020740000207CB50D466946FFF749
:100EB000D5FA002618B12E602E7102207CBD9DF857
:100EC000000000F012FF019C9DF80000703400F05B
:100ED0000CFF019884F8426081682960017B2971C8
:100EE00094F842100029F5D100207CBD10B50446CD
:100EF00000F02BFF20B10BF0A9F908B10C2010BDB8
:100F0000207800F0EBFEE279611C0BF020FB08B1C9
:100F1000002010BD022010BD10B5886E60B1002207
:100F200041F8682F0120CA718979884012F0DCFFEE
:100F3000002800D01F2010BD0C2010BD1CB50C4691
:100F40006946FFF78BFA002809D19DF800000028B8
:100F50000198B0F8700000D0401C208000201CBD1B
:100F60001CB5044600886946FFF778FA08B10220EC
:100F70001CBD606828B1DDE90001224600F0C3FF16
:100F80001CBDDDE90001FFF7C7FF1CBD2DE9F041E5
:100F900004460078012804D018B1022801D00328A3
:100FA0001ED1607828B1012803D0022801D003287F
:100FB00016D1E07B10B9A078012811D1A07830F0CB
:100FC00005020DD110F0050F0AD0400801D0112004
:100FD00054E5E078E68862890F4618B1012801D00F
:100FE00012204BE5104600F0CCFF302558B13946B1
:100FF000304600F0D0FF30B1A07B0028F0D00728A9
:10100000EED800203AE5284638E51FB5044600F042
:1010100080FE10B10C2004B010BD022104F10A00C2
:1010200000F0C3FFA0788DF80800A0788DF80000CC
:1010300060788DF8040020788DF80300A07B8DF88F
:101040000500E07B00B101208DF80600A078C00704
:101050000CD0E078012812D098B100208DF8010062
:10106000E088ADF80A006089ADF80C0002A80FF026
:1010700090FE0028CFD168460DF0ABFBCBE70220F5
:10108000ECE70120EAE710B504460121FFF77EFFF7
:10109000002803D12046BDE81040B6E710BD027815
:1010A000012A01D0BAB118E042783AB1012A05D03C
:1010B000022A12D189B1818879B100E059B1418801
:1010C00049B1808838B101EB8101490000EB800013
:1010D000B1EB002F01D2002070471220704770B58D
:1010E000044600780D46012809D010F08DFB052834
:1010F00003D00FF05EFD002800D00C2070BD0DF075
:101100005CFA88B10DF06EFA0DF043FB0028F5D1C2
:1011100025B160780DF0F4FA0028EFD1A18860883D
:10112000BDE870400FF050BE122070BD10B50446EF
:101130000121FFF7B4FF002804D12046BDE810408C
:101140000121CCE710BDF0B5871FDDE9056540F64C
:101150007B44A74213D28F1FA74210D288420ED8D9
:10116000B2F5FA7F0BD2A3F10A00241FA04206D2E7
:10117000521C4A43B2EB830F01DAAE4201D9002080
:10118000F0BD0120F0BD2DE9FC41477A88460446B8
:1011900017F0050F73D0F80871D1780701D5112029
:1011A00054E694F83A0008B9012F68D100252E467C
:1011B000F8071BD088F00105208A294600F0E1FEDF
:1011C00048B36089294600F0E6FE20B3208A618991
:1011D000884254D8A18EE08DCDE90001238D628C28
:1011E000A18BE08AFFF7AFFFA8B10125B8070ED5A4
:1011F00004EB4500828EC18DCDE90012038D428C37
:10120000818BC08AFFF79FFF28B12E466D1CB8F175
:10121000000F02D023E0302018E6228A012119E0D5
:10122000B14203D004EB4100008A024404EB4100C8
:10123000C38A878ABB4222D1838B478BBB421ED194
:10124000438C078CBB421AD1038DC08C834216D1CC
:10125000491CC9B2A942E3D3608990420FD32078D8
:1012600010B101280BD102E0A0780028F9D16078F4
:1012700038B1012805D0022803D0032801D012205C
:10128000E4E50020E2E500217DE70178C90702D00E
:10129000406812F00EBA12F0DBB910B500780128E0
:1012A00000D00020FDF786FD002010BD2DE9F0479D
:1012B00088B00D46AFF6FC02D2E900920146904696
:1012C0002846FFF760FF06000CD100F022FD40B970
:1012D000FE4F387828B90CF075FEA0F57F41FF3934
:1012E00002D00C2008B048E4032105F1100000F002
:1012F0005CFEF64801AA3E380190F5480290F3489A
:1013000006211038039006A801F040FC040037D0F5
:1013100000210BF028FC04F130017B8ABA8ACB83D0
:101320000A84797C0091BA463B7CBA8A798A208803
:1013300001F01AFD00B1FFDF208806F024FD2188AE
:1013400004F10E0000F00BFDE2A004F112070068AA
:1013500000900321684604F0C3FE002069460A5C41
:101360003A54401CC0B20328F9D3A88B6080688C23
:10137000A080288DE080687AC10703D0012706E0AD
:101380000920AFE7800701D5022700E000273A4691
:10139000BAF8160011460FF0ABFD0146A0622046D8
:1013A0000FF0B4FD3A46214600200BF09CFF00B937
:1013B0000926C64A21461C3200200BF096FF002762
:1013C00084F8767084F87770A87800F087FC6076EF
:1013D000D5F80300C4F81A00B5F80700E083C4F894
:1013E000089084F80C80012084F8200101468DF8D3
:1013F0000070684604F074FE9DF8000000F00701DC
:10140000C0F3C1021144C0F3401008448DF800003D
:10141000401D2076092801D208302076012120467F
:101420000BF0A1FB68780DF0D3F8E6BBA97828781B
:10143000EA1C0DF0A0F848B10DF0D4F8A97828788E
:10144000EA1C0DF037F9060002D03AE0122638E027
:10145000687A00F001010020CA0700D00120890746
:1014600001D540F002000DF06FF8060029D12146A9
:1014700003200DF049F9060023D1687A00F001013C
:101480008DF81010C00705D06889ADF81200288AC1
:10149000ADF8140004A80FF07CFC064695F83A005D
:1014A00000B1012000E00CE00DF060F84EB90DF045
:1014B00070F9060005D1A98F20460FF00BFC06003D
:1014C00008D0208806F060FC2088062101F0A2FBED
:1014D00000B1FFDF304605E701460020E6E638B5FB
:1014E0007A48007878B910F08FF9052805D00CF00B
:1014F00069FDA0F57F41FF3905D068460FF0A7FCD4
:10150000040002D00CE00C2038BD0098008806F0E2
:101510003BFC00980621008801F07CFB00B1FFDF56
:10152000204638BD1CB582894189CDE90012038966
:10153000C28881884088FFF706FE08B100201CBDE4
:1015400030201CBD70B50546FFF7ECFF00280ED11A
:101550002888062101F04CFB040007D000F03CFC79
:1015600020B1D4F81801017831B901E0022070BD32
:10157000D4F86411097809B13A2070BD0521817150
:10158000D4F8181100200881D4F81811A8884881CF
:10159000D4F81811E8888881D4F818112889C881EE
:1015A000D4F81801028941898A4204D88279082A2C
:1015B00001D88A4201D3122070BD29884180D4F815
:1015C000181102200870002070BD3EB504460BF0D3
:1015D000B7FCB0B13D480125A0F140024570236839
:1015E00042F8423F23790021137141706946062079
:1015F00001F087FA00B1FFDF684601F060FA10B130
:101600000EE012203EBDBDF80440029880F8205143
:10161000684601F054FA18B9BDF80400A042F4D1AC
:1016200000203EBD70B505460088062101F0E0FAB5
:10163000040007D000F0D0FB20B1D4F818110878CE
:1016400030B901E0022070BDD4F86401007808B11F
:101650003A2070BDB020005D10F0010F1BD0D5F80E
:1016600002004860D5F806008860D4F8180169893E
:1016700010228181D4F8180105F10C010E3004F517
:101680008C74FCF7A4FE2168032008702168288868
:101690004880002070BD0C2070BD38B5044600782D
:1016A000EF2854D86088ADF80000009800F090FC56
:1016B000C0B36188080708D4D4E90120824246D823
:1016C000202A44D3B0F5804F41D805E0140800200B
:1016D0008000002011223300207B18B3072836D861
:1016E000607B28B1012803D0022801D003282ED125
:1016F0004A0703D4022801D0032805D1A07B08B1F2
:10170000012824D1480707D4607D28B1012803D0DF
:10171000022801D003281AD1C806E07D03D501288C
:1017200015D110E013E0012801D003280FD1C8061D
:1017300009D4607E012803D0022801D0032806D1F5
:10174000A07E0F2803D8E07E18B1012801D0122016
:1017500038BD002038BDF8B515460E46044607F0E2
:1017600016FE08B10C20F8BD2046FFF796FF0028B2
:10177000F9D1E07D03280BD0A078C00602D4607EAA
:10178000032805D0FDF720FB3070A07515B10CE0E3
:101790001120F8BDFF208DF8000069460020FDF7FC
:1017A000FDFA69460020FDF7EDFA2046BDE8F84055
:1017B000FDF749BA0022CEE70078C10801D0122017
:1017C0007047FC4981F820000020704710B504469E
:1017D0000078C00704D1608810B1FDF7B6FA80B177
:1017E0002078618800F00102607800F015FC002884
:1017F00006D1FDF792FA01466088884203D9072096
:1018000010BD122010BD6168FDF7C8FA002010BDA0
:1018100010B504460078C00704D1608810B1FCF709
:101820008CFF70B12078618800F00102607800F0D0
:10183000F3FB002804D160886168FDF7A3FA00205B
:1018400010BD122010BD7CB5044640784225012809
:1018500008D8A078FCF769FF20B12078122501286C
:1018600002D090B128467CBDFDF7BAFA20B1A0881D
:101870000028F7D08028F5D8FDF7B9FA60B1607874
:101880000028EFD02078012808D006F09FFB0446FE
:1018900007F077FA00287FD00C207CBDFDF7ECF82C
:1018A00010B9FDF796FA90B307F071FD0028F3D157
:1018B000FCF702FFA0F57F41FF39EDD1FDF7FEF8FF
:1018C000A68842F210704643A079FDF74FFAFCF764
:1018D0003BFFF8B10022072101A801F057F90400ED
:1018E00058D0B5480021846020460AF0F9FF204610
:1018F000FDF7D8FDAF4D04F130006A8AA98AC28392
:101900000184FCF728FF60B1E88A01210DE0FFE7C0
:1019100012207CBD3146002007F0E5FA88B3FFDFD6
:1019200044E0FDF766FA0146E88A07F087FB0146C6
:10193000A0620022204606F04CFBFCF70CFF38B9F1
:10194000FDF757FA0246214601200BF0CCFCD0B13E
:10195000984A21461C3201200BF0C7FC687C00909D
:101960002B7CAA8A698A208801F0FEF900B1FFDF8A
:10197000208806F008FA3146204607F0B4FA00B194
:10198000FFDF13E008E00721BDF8040001F042F991
:1019900000B1FFDF09207CBD44B1208806F0F4F9D6
:1019A0002088072101F036F900B1FFDF00207CBD5F
:1019B000002148E770B50D46072101F019F9040030
:1019C00003D094F8930110B10AE0022070BD94F89E
:1019D0007D00142801D0152802D194F8E00108B147
:1019E0000C2070BD1022294604F5CA70FCF7EFFCEC
:1019F000012084F89301002070BD10B5072101F08B
:101A0000F7F818B190F8931111B107E0022010BD5A
:101A100090F87D10142903D0152901D00C2010BD99
:101A2000022180F89311002010BD2DE9FC410C46E5
:101A30004BF68032122194421CD8DCB16946FEF785
:101A40000DFD002815D19DF8000000F04EF9019E13
:101A50009DF80000703600F048F9019DAD1C2F88FC
:101A60002246394630460AF0F6FE2888B842F6D1BA
:101A7000002005E4084603E47CB504460088694676
:101A8000FEF7ECFC002810D19DF8000000F02DF9C5
:101A9000019D9DF80000703500F027F90198A278AB
:101AA00090F82C10914201D10C207CBD7F2129722D
:101AB000A9720021E972E17880F82D10217980F86F
:101AC0002E10A17880F82C1000207CBD1CB50C468F
:101AD0006946FEF7C3FC00280AD19DF8000000F01B
:101AE00004F9019890F88C0000B1012020700020CA
:101AF0001CBD7CB50D4614466946FEF7AFFC0028B8
:101B000009D19DF8000000F0F0F8019890F82C0041
:101B1000012801D00C207CBD9DF8000000F0E5F804
:101B2000019890F87810297090F8790020700020C2
:101B30007CBD70B50D461646072101F059F818B363
:101B400081880124C388428804EB4104AC4217D841
:101B500042F210746343A4106243B3FBF2F2521ECC
:101B600094B24FF4FA72944200D91446A54200D2BE
:101B70002C46491C641CB4FBF1F24A43521E91B23C
:101B800090F8CC211AB901E0022070BD01843180A7
:101B9000002070BD10B50C46072101F029F868B18E
:101BA00080F8FF4024B190F8FD1009B107F05CFA0D
:101BB000002010BD14080020740000200220F8E767
:101BC000017889B1417879B141881B290CD381888A
:101BD0001B2909D3C188022906D3FC4902680A657A
:101BE00040684865002070471220704710B50446D1
:101BF0000FF07AF9204607F0F0F90020D9E710B588
:101C000007F0EEF90020D4E72DE9F04115460F4624
:101C100006460122114638460FF06AF904460121B2
:101C2000384607F00BFA844200D2044601213046C0
:101C300000F060F806460121002000F05BF8311842
:101C4000012096318C4206D901F19600611AB1FB50
:101C5000F0F0401C80B228800020BDE8F08110B573
:101C6000044600F072F808B10C20A2E7601C0AF0EC
:101C700049FC207800F00100FCF71BFF207800F001
:101C800001000CF0AAFC002093E710B504460720E1
:101C900000F048FF08B10C208BE72078C00711D076
:101CA00000226078114612F02BF908B1122080E76B
:101CB000A06809F022F96078D4F8041009F026F938
:101CC000002076E7002009F018F900210846F5E722
:101CD00010B5006804F0C1FF00206AE718B10228BF
:101CE00001D0012070470020704708B100207047E4
:101CF0000120704710B5012904D0022905D0FFDF6B
:101D0000204656E7C000503001E080002C3084B2FD
:101D1000F6E710B50FF078FD042803D0052801D0B0
:101D2000002046E7012044E710B5FFF7F2FF10B1AD
:101D30000CF0F3FC28B907F02AFB20B1FCF794FE65
:101D400008B1012035E7002033E710B5FFF7E1FFC8
:101D500018B907F01CFB002800D0012029E72DE965
:101D6000FE4300250F4680460A260421404604F023
:101D7000E0F940460BF0C0F8062000F0E1FE044612
:101D800015E06946062000F0BCFE0AE0BDF804003C
:101D9000B84206D00298042241460E30FCF7EAFA17
:101DA00050B1684600F08BFE0500EFD0641E002C99
:101DB00006DD002DE5D005E040460BF0A6F8F5E77E
:101DC00005B9FFDFD8F800000AF04FFD761E01D0FC
:101DD0000028CAD0BDE8FE8390F8F01090F88C007F
:101DE00020B919B1042901D00120704700207047A3
:101DF000017800290AD0416891F8FD20002A05D019
:101E0000002281F8FD20406807F02EB9704770B5B8
:101E100014460546012200F013F9002806D1214698
:101E20002846BDE87040002200F00AB970BDFB28CA
:101E300003D840F64800814201D9112070470020A4
:101E400070471B38E12806D2B1F5A47F03D344F2D2
:101E50009020814201D912207047002070471FB5A1
:101E60005A49403191F82010CA0702D102781D2A40
:101E70000AD08A0702D402781C2A28D049073DD408
:101E80000178152937D039E08088ADF8000002A923
:101E9000FEF7E4FA00B1FFDF9DF80800FFF725FF29
:101EA000039810F8601F8DF8021040788DF8030039
:101EB0000020ADF8040001B9FFDF9DF8030000B970
:101EC000FFDF6846FEF7D1FCD8B1FFDF19E080885C
:101ED000ADF8000040F64801FB20ADF80410ADF865
:101EE0000200ADF80600ADF808106846FEF7C8FD20
:101EF00038B1FFDF05E0807BC00702D0002004B0CE
:101F000057E60120FBE7F8B50746508915460C4611
:101F100040B1B0F5004F05D20022A878114611F06B
:101F2000EFFF08B11220F8BDA06E04F1700630B1C9
:101F3000A97894F86E00814201D00C20F8BD0121EF
:101F400084F86F10A97884F86E106968A1666989B1
:101F5000A4F86C102889B084002184F86F102888B8
:101F60006946FEF7EBFFB08CBDF80010081A00B20E
:101F7000002804DD21463846FEF7CEFFDDE70020CD
:101F8000F8BD042803D321B9B0F5804F01D9002052
:101F9000704701207047042803D321B9B0F5804F62
:101FA00001D9002070470120704710B500224FF47E
:101FB000C84408E030F81230A34200D9234620F884
:101FC0001230521CD2B28A42F4D3F2E5D407002078
:101FD00080B2C1060BD401071CD481064FEAC07140
:101FE00001D5B9B900E099B1800713D410E04106DA
:101FF00010D481060ED4C1074FEA807104D00029A5
:1020000002DB400704D405E0010703D4400701D4F4
:10201000012070470020704770B50C460546FF2927
:1020200004D8FCF798FB18B11F2C01D9122070BD01
:102030002846FCF77AFB08B1002070BD422070BD35
:102040000AB1012200E00222024202D1880802D134
:1020500009B10020704711207047000030B5058895
:1020600025F4004421448CB24FF4004194420AD23A
:10207000121B92B21B339A4201D2A94307E005F426
:102080000041214303E0A21A92B2A9431143018007
:1020900030BD0844083050434A31084480B270478C
:1020A00070B51D4616460B46044629463046049A2E
:1020B000FFF7EFFF0646B34200D2FFDF28220021E0
:1020C0002046FCF7AEF94FF6FF70A082283EB0B272
:1020D00065776080B0F5004F00D9FFDF618805F1BA
:1020E0003C00814200D2FFDF60880835401B343855
:1020F00080B220801B2800D21B2020800020A077E7
